:020000040800F2
:1000000000000220F51B00084D1700084F170008DC
:10001000511700085317000855170008000000008A
:100020000000000000000000000000001187000830
:100030005717000800000000B18700081588000865
:10004000451C0008451C0008451C0008451C00080C
:10005000451C0008451C0008CDFA0008D7FA000826
:10006000E1FA0008EBFA0008F5FA0008451C000860
:10007000451C0008451C00085917000869170008AE
:10008000451C0008451C0008451C0008451C0008CC
:10009000451C0008451C0008451C0008FFFA000824
:1000A000451C0008451C000879170008451C00087D
:1000B000451C0008451C0008451C0008451C00089C
:1000C000451C0008451C0008451C00089117000845
:1000D000A1170008451C0008451C0008451C000825
:1000E00025FB0008451C0008451C0008451C0008AD
:1000F000451C0008451C0008451C0008451C00085C
:10010000451C0008451C0008451C0008451C00084B
:10011000451C0008451C0008B1170008C11700085D
:10012000D1170008451C0008E1170008F117000866
:10013000451C000801180008451C0008451C000863
:10014000451C0008451C0008451C0008451C00080B
:10015000451C0008451C0008451C0008451C0008FB
:10016000451C0008451C0008451C0008451C0008EB
:10017000451C0008451C0008451C00080000000044
:08018000451C0008451C0008A5
:1001900010B5054C237833B9044B13B10448AFF3C1
:1001A00000800123237010BD280200200000000001
:1001B000C85C010808B5034B1BB103490348AFF302
:1001C000008008BD000000002C020020C85C01086F
:1001D00001F0FF01102A2BDB10F0070F08D010F8F8
:1001E000013B013A8B422DD010F0070F42B3F6D1FC
:1001F000F0B441EA012141EA014122F007047FF015
:1002000000070023F0E80256083C85EA010586EA6B
:10021000010685FA47F5A3FA87F586FA47F6A5FAA7
:1002200087F68EB9EED1F0BC01F0FF0102F00702B3
:1002300032B110F8013B013A83EA010313B1F8D15E
:100240000020704701387047002D06BF354603383F
:10025000073815F0010F07D1013015F4807F02BF78
:10026000013015F4C03F0130F0BC0138704700BFC9
:10027000034613F8012B002AFBD1181A01387047E6
:1002800081F0004102E000BF83F0004330B54FEA47
:1002900041044FEA430594EA050F08BF90EA020FB4
:1002A0001FBF54EA000C55EA020C7FEA645C7FEA47
:1002B000655C00F0E2804FEA5454D4EB5555B8BF6A
:1002C0006D420CDD2C4480EA020281EA030382EADB
:1002D000000083EA010180EA020281EA0303362D6D
:1002E00088BF30BD11F0004F4FEA01314FF4801C40
:1002F0004CEA113102D0404261EB410113F0004F52
:100300004FEA03334CEA133302D0524263EB430308
:1003100094EA050F00F0A780A4F10104D5F1200EA6
:100320000DDB02FA0EFC22FA05F2801841F1000101
:1003300003FA0EF2801843FA05F359410EE0A5F1D5
:1003400020050EF1200E012A03FA0EFC28BF4CF006
:10035000020C43FA05F3C01851EBE37101F00045BC
:1003600007D54FF0000EDCF1000C7EEB00006EEBC9
:100370000101B1F5801F1BD3B1F5001F0CD3490853
:100380005FEA30004FEA3C0C04F101044FEA4452AA
:1003900012F5800F80F09A80BCF1004F08BF5FEA31
:1003A000500C50F1000041EB045141EA050130BD11
:1003B0005FEA4C0C404141EB0101013C28BFB1F523
:1003C000801FE9D291F0000F04BF01460020B1FA6E
:1003D00081F308BF2033A3F10B03B3F120020CDA41
:1003E0000C3208DD02F1140CC2F10C0201FA0CF01F
:1003F00021FA02F10CE002F11402D8BFC2F1200C84
:1004000001FA02F120FA0CFCDCBF41EA0C01904039
:10041000E41AA2BF01EB0451294330BD6FEA040482
:100420001F3C1CDA0C340EDC04F11404C4F120026D
:1004300020FA04F001FA02F340EA030021FA04F37F
:1004400045EA030130BDC4F10C04C4F1200220FAD6
:1004500002F001FA04F340EA0300294630BD21FA14
:1004600004F0294630BD94F0000F83F4801306BFDA
:1004700081F480110134013D4EE77FEA645C18BFCE
:100480007FEA655C29D094EA050F08BF90EA020F65
:1004900005D054EA000C04BF1946104630BD91EA5D
:1004A000030F1EBF0021002030BD5FEA545C05D160
:1004B0004000494128BF41F0004130BD14F580049F
:1004C0003CBF01F5801130BD01F0004545F0FE4113
:1004D00041F470014FF0000030BD7FEA645C1ABF48
:1004E000194610467FEA655C1CBF0B46024650EA7F
:1004F000013406BF52EA033591EA030F41F40021AB
:1005000030BD00BF90F0000F04BF0021704730B530
:100510004FF4806404F132044FF000054FF0000105
:1005200050E700BF90F0000F04BF0021704730B5C6
:100530004FF4806404F1320410F0004548BF40429B
:100540004FF000013EE700BF42004FEAE2014FEAF0
:1005500031014FEA02701FBF12F07F4393F07F4FCB
:1005600081F06051704732F07F4208BF704793F0CE
:100570007F4F04BF41F40021704730B54FF46074E1
:1005800001F0004521F000411CE700BF50EA0102E4
:1005900008BF704730B54FF000050AE050EA01028D
:1005A00008BF704730B511F0004502D5404261EBFD
:1005B00041014FF4806404F132045FEA915C3FF43E
:1005C000D8AE4FF003025FEADC0C18BF03325FEADB
:1005D000DC0C18BF033202EBDC02C2F1200300FA8C
:1005E00003FC20FA02F001FA03FE40EA0E0021FAB1
:1005F00002F11444BDE600BF70B54FF0FF0C4CF49F
:10060000E06C1CEA11541DBF1CEA135594EA0C0F50
:1006100095EA0C0F00F0DEF82C4481EA030621EA8B
:100620004C5123EA4C5350EA013518BF52EA0335C6
:1006300041F4801143F4801338D0A0FB02CE4FF078
:100640000005E1FB02E506F00042E0FB03E54FF0A8
:100650000006E1FB03569CF0000F18BF4EF0010EA0
:10066000A4F1FF04B6F5007F64F5407404D25FEA9C
:100670004E0E6D4146EB060642EAC62141EA55514F
:100680004FEAC52040EA5E504FEACE2EB4F1FD0C91
:1006900088BFBCF5E06F1ED8BEF1004F08BF5FEA0F
:1006A000500E50F1000041EB045170BD06F00046C1
:1006B00046EA010140EA020081EA0301B4EB5C046E
:1006C000C2BFD4EB0C0541EA045170BD41F4801166
:1006D0004FF0000E013C00F3AB8014F1360FDEBF8B
:1006E000002001F0004170BDC4F10004203C35DA67
:1006F0000C341BDC04F11404C4F1200500FA05F3EA
:1007000020FA04F001FA05F240EA020001F000428A
:1007100021F0004110EBD37021FA04F642EB060100
:100720005EEA430E08BF20EAD37070BDC4F10C042A
:10073000C4F1200500FA04F320FA05F001FA04F2EE
:1007400040EA020001F0004110EBD37041F10001DA
:100750005EEA430E08BF20EAD37070BDC4F12005E5
:1007600000FA05F24EEA020E20FA04F301FA05F24D
:1007700043EA020321FA04F001F0004121FA04F2F5
:1007800020EA020000EBD3705EEA430E08BF20EAC5
:10079000D37070BD94F0000F0FD101F000464000FF
:1007A00041EB010111F4801F08BF013CF7D041EA81
:1007B000060195F0000F18BF704703F00046520085
:1007C00043EB030313F4801F08BF013DF7D043EA56
:1007D0000603704794EA0C0F0CEA135518BF95EA0C
:1007E0000C0F0CD050EA410618BF52EA4306D1D193
:1007F00081EA030101F000414FF0000070BD50EAB2
:10080000410606BF1046194652EA430619D094EA3B
:100810000C0F02D150EA013613D195EA0C0F05D125
:1008200052EA03361CBF104619460AD181EA030179
:1008300001F0004141F0FE4141F470014FF0000031
:1008400070BD41F0FE4141F4780170BD70B54FF0CC
:10085000FF0C4CF4E06C1CEA11541DBF1CEA13554C
:1008600094EA0C0F95EA0C0F00F0A7F8A4EB05042E
:1008700081EA030E52EA03354FEA013100F0888025
:100880004FEA03334FF0805545EA131343EA1263EE
:100890004FEA022245EA111545EA10654FEA0026A3
:1008A0000EF000419D4208BF964244F1FD0404F55C
:1008B000407402D25B084FEA3202B61A65EB0305B8
:1008C0005B084FEA32024FF480104FF4002CB6EB75
:1008D000020E75EB030E22BFB61A754640EA0C00F5
:1008E0005B084FEA3202B6EB020E75EB030E22BF35
:1008F000B61A754640EA5C005B084FEA3202B6EB76
:10090000020E75EB030E22BFB61A754640EA9C0034
:100910005B084FEA3202B6EB020E75EB030E22BF04
:10092000B61A754640EADC0055EA060E18D04FEAC2
:10093000051545EA16754FEA06164FEAC30343EA62
:1009400052734FEAC2025FEA1C1CC0D111F4801F2F
:100950000BD141EA00014FF000004FF0004CB6E728
:1009600011F4801F04BF01430020B4F1FD0C88BFC7
:10097000BCF5E06F3FF6AFAEB5EB030C04BFB6EBD2
:10098000020C5FEA500C50F1000041EB045170BDC5
:100990000EF0004E4EEA113114EB5C04C2BFD4EBF2
:1009A0000C0541EA045170BD41F480114FF0000E76
:1009B000013C90E645EA060E8DE60CEA135594EAF2
:1009C0000C0F08BF95EA0C0F3FF43BAF94EA0C0FF5
:1009D0000AD150EA01347FF434AF95EA0C0F7FF46A
:1009E00025AF104619462CE795EA0C0F06D152EABE
:1009F00003353FF4FDAE1046194622E750EA4106A2
:100A000018BF52EA43067FF4C5AE50EA41047FF4B2
:100A10000DAF52EA43057FF4EBAE12E74FF0FF3C17
:100A200006E000BF4FF0010C02E000BF4FF0010CE8
:100A30004DF804CD4FEA410C7FEA6C5C4FEA430C61
:100A400018BF7FEA6C5C1BD001B050EA410C0CBFB0
:100A500052EA430C91EA030F02BF90EA020F002012
:100A6000704710F1000F91EA030F58BF994208BF79
:100A700090422CBFD8176FEAE37040F00100704736
:100A80004FEA410C7FEA6C5C02D150EA013C07D18D
:100A90004FEA430C7FEA6C5CD6D152EA033CD3D0D8
:100AA0005DF8040B704700BF8446104662468C46D2
:100AB0001946634600E000BF01B5FFF7B7FF002805
:100AC00048BF10F1000F01BD4DF808EDFFF7F4FF2E
:100AD0000CBF012000205DF808FB00BF4DF808EDB9
:100AE000FFF7EAFF34BF012000205DF808FB00BFDC
:100AF0004DF808EDFFF7E0FF94BF012000205DF8FE
:100B000008FB00BF4DF808EDFFF7CEFF94BF0120B2
:100B100000205DF808FB00BF4DF808EDFFF7C4FFAB
:100B200034BF012000205DF808FB00BF4FEA410CF4
:100B30007FEA6C5C02D150EA013C0AD14FEA430CD7
:100B40007FEA6C5C02D152EA033C02D14FF0000014
:100B500070474FF0010070474FEA410212F5001252
:100B600015D211D56FF47873B3EB625212D94FEAF4
:100B7000C12343F0004343EA505311F0004F23FADE
:100B800002F018BF404270474FF00000704750EA33
:100B9000013005D111F0004008BF6FF000407047F0
:100BA0004FF00000704700BF4A0011D212F500124A
:100BB00011D20DD56FF47873B3EB62520ED44FEAB5
:100BC000C12343F0004343EA505323FA02F0704735
:100BD0004FF00000704750EA013002D14FF0FF3073
:100BE00070474FF0000070474FEA4102B2F1E04316
:100BF00024BFB3F5001CDCF1FE5C0DD901F0004C04
:100C00004FEAC0024CEA5070B2F1004F40EB830053
:100C100008BF20F00100704711F0804F21D113F17F
:100C20003872BCBF01F00040704741F480114FEAB8
:100C30005252C2F11802C2F1200C10FA0CF320FA41
:100C400002F018BF40F001004FEAC1234FEAD3235E
:100C500003FA0CFC40EA0C0023FA02F34FEA4303C8
:100C6000CCE77FEA625307D150EA01331EBF4FF051
:100C7000FE4040F44000704701F0004040F0FE406C
:100C800040F40000704700BF53B94AB9002908BFBB
:100C900000281CBF4FF0FF314FF0FF3000F0A0B92B
:100CA000ADF1080C6DE904CE00F03CF8DDF804E08D
:100CB000DDE9022304B0704738B500220023044662
:100CC0000D46FFF70BFF28B920462946BDE83840FE
:100CD00000F00AB8204605F1004100F005F8404256
:100CE00061EB410138BD00BFD0B50C4B0022064678
:100CF0000F46FFF781FCFFF757FF0446FFF702FCA2
:100D0000074B0022FFF778FC02460B463046394677
:100D1000FFF7BAFAFFF748FF2146D0BD0000F03DCB
:100D20000000F0412DE9F047089D0C46002B4ED104
:100D300094468C458646B2FA82F262D94AB1C2F133
:100D40002003914020FA03F30CFA02FC194300FA45
:100D500002FE4FEA1C471FFA8CF6B1FBF7F44FEA8C
:100D60001E4307FB141143EA014304FB06F19942B9
:100D70000AD91CEB030304F1FF3080F01281994281
:100D800040F20F81023C6344591A1FFA8EF3B1FB03
:100D9000F7F007FB101143EA014300FB06F69E4201
:100DA0000AD91CEB030300F1FF3180F0FC809E4266
:100DB00040F2F980634402389B1B40EA0440002162
:100DC0001DB1D3400022C5E90032BDE8F0878B4257
:100DD00005D90DB1C5E9000100210846F5E7B3FAD0
:100DE00083F1002946D1A34202D39042C0F0F080A3
:100DF000861A64EB03030120002DE6D0C5E90063E9
:100E0000E3E7002A40F09080A1EB0C044FEA1C4875
:100E10001FFA8CF70121B4FBF8F64FEA1E4308FBDA
:100E2000164443EA044307FB06F0984208D91CEB3A
:100E3000030306F1FF3402D2984200F2CD80264629
:100E40001C1A1FFA8EF3B4FBF8F008FB104443EAB7
:100E5000044300FB07F79F4208D91CEB030300F192
:100E6000FF3402D29F4200F2B0802046DB1B40EAF2
:100E70000640A5E7C1F120068B4022FA06F71F4382
:100E800020FA06FC04FA01F343EA0C03F44000FAEA
:100E900001F8380C4FEA1349B4FBF0FE1FFA87FC47
:100EA00000FB1E4449EA04440EFB0CF9A14502FA7A
:100EB00001F20AD93C190EF1FF3A80F08480A14575
:100EC00040F28180AEF1020E3C44A4EB09041FFA0B
:100ED00083F9B4FBF0F300FB134449EA044403FB39
:100EE0000CFCA44507D93C1903F1FF3067D2A44597
:100EF00065D9023B3C4443EA0E40A0FB0293A4EBBD
:100F00000C049C42CE469C4651D34ED055B1B8EB12
:100F10000E0364EB0C0404FA06F6CB401E43CC40EF
:100F2000C5E90064002150E7C2F1200320FA03F173
:100F30000CFA02FC24FA03F394400C434FEA1C48D9
:100F400000FA02FE1FFA8CF7B3FBF8F008FB103131
:100F5000230C43EA014300FB07F1994208D91CEB3B
:100F6000030300F1FF362CD299422AD90238634498
:100F70005B1AA4B2B3FBF8F108FB113344EA034453
:100F800001FB07F3A34208D91CEB040401F1FF366F
:100F900013D2A34211D902396444E41A41EA004150
:100FA00039E70446F0E6084606E7C845AED2B9EB95
:100FB000020E63EB070C0138A8E73146EDE7034664
:100FC00099E73046D4E7D6467FE7634402384DE7D9
:100FD0000646234608460FE7023E634430E700BF5B
:100FE000704700BF08B50548054B036001F062F883
:100FF00000B908BD00F038F9FBE700BF440200204B
:10100000003002400268094B9A4200D0704782B01B
:1010100000230193064B1A6B42F480521A631B6B38
:1010200003F480530193019B02B0704700300240EB
:101030000038024010B582B0002400941E4B1A6B99
:1010400042F480021A631A6B02F480020092009A42
:1010500001941A6B42F400121A631B6B03F4001321
:101060000193019B224605210E2000F0E5FF0E2092
:1010700001F006F8224605210F2000F0DDFF0F20C9
:1010800000F0FEFF22460521382000F0D5FF382071
:1010900000F0F6FF224605213A2000F0CDFF3A206D
:1010A00000F0EEFF224605213B2000F0C5FF3B206B
:1010B00000F0E6FF02B010BD00380240034B0360B1
:1010C000034B0B6080231360704700BF4C0400206B
:1010D0004C02002010B588B00DF1040C074C0FCC69
:1010E000ACE80F0094E807008CE80700002101A895
:1010F00005F04CFB024B186008B010BDE05C010825
:10110000F004002070B58CB0002407940894099472
:101110000A940B9401943E4B1A6B42F010021A632E
:101120001A6B02F010020192019A02941A6B42F0BB
:1011300004021A631A6B02F004020292029A0394E8
:101140001A6B42F080021A631A6B02F0800203925B
:10115000039A04941A6B42F001021A631A6B02F0AC
:1011600001020492049A05941A6B42F002021A6377
:101170001A6B02F002020592059A06941A6B42F06D
:1011800008021A631B6B03F008030693069B214EAB
:1011900022460821304602F01DFD4FF6FF730793EB
:1011A00003250895099407A91B4802F09FFB4FF6F9
:1011B000C17307930895099407A9184802F096FB94
:1011C00049F6191307930895099407A9144802F0E2
:1011D0008DFB4CF2D73307930895099407A9114862
:1011E00002F084FB4FF6F77307930895099407A95B
:1011F000304602F07BFB08230793012308930994F0
:101200000A9407A9304602F071FB0CB070BD00BF14
:1012100000380240000C024000100240000802406A
:10122000000002400004024008B50748074B036075
:10123000012343604FF47A63836002F0F5FC00B948
:1012400008BD00F011F8FBE7F40400200030004076
:1012500008B50268034B9A4200D008BD00F062FE58
:10126000FBE700BF0048014072B6FEE700B595B04D
:101270003022002108A811F049FA002303930493B7
:101280000593069307930193214A116C41F0805115
:101290001164126C02F080520192019A02931D4B6C
:1012A0001A6842F480421A601B6803F48043029378
:1012B000029B092308934FF48033099301230D9374
:1012C00002230E934FF480020F9204221092902278
:1012D000119212930623139308A802F0F5FC98B913
:1012E0000F23039302230493002305934FF4A05389
:1012F00006934FF480530793042103A802F0D2FF12
:1013000020B915B05DF804FBFFF7AEFFFFF7ACFFA7
:10131000003802400070004008B500F0E9FDFFF71A
:10132000A5FFFFF7EFFEFFF785FE00F0F3FB00F0EF
:1013300003FBFFF757FE00F011F800F05DFB00F033
:1013400033FB00F0C1FA00F031F800F053F8FFF77A
:10135000C1FE05F00CFAFEE77047000008B505482D
:10136000054B036003F0F4F800B908BDFFF77CFFFC
:10137000FBE700BF00050020000806500268094B8B
:101380009A4200D0704782B000230193064B5A6BFB
:1013900042F040025A635B6B03F040030193019BF0
:1013A00002B07047000806500038024008B50F48E8
:1013B0000F4B03604FF48273436000238360C3606C
:1013C00002220261012242614FF4007282613022E6
:1013D000C26180220262436283620A23C36203F015
:1013E000F1F900B908BDFFF73FFFFBE7E806002071
:1013F0000030014008B50F480F4B03604FF4827373
:10140000436000238360C3600222026101224261C3
:101410004FF4007282612822C2618022026243621C
:1014200083620A23C36203F0CDF900B908BDFFF758
:101430001BFFFBE790060020003800402DE9F04339
:101440008DB0044600230793089309930A930B93E6
:101450000368794A934205D0784A934278D00DB018
:10146000BDE8F08300250195754B5A6C42F480521B
:101470005A645A6C02F480520192019A02951A6BD6
:1014800042F001021A631A6B02F001020292029A00
:1014900003951A6B42F002021A631B6B03F00203FE
:1014A0000393039B602307934FF00208CDF820803D
:1014B00003270A9705260B9607A9624802F016FA39
:1014C00020230793CDF8208009950A970B9607A94A
:1014D0005D4802F00BFA5D485D4B03604FF0C0635E
:1014E00043608560C5604FF4806303614561856139
:1014F000C5610562456200F079FE18BB534BE36499
:101500009C635448544B03604FF0C06343604023D6
:1015100083600023C3604FF4806202614361836192
:10152000C3610362436200F061FE70B9494BA3647A
:101530009C6300220521232000F07EFD232000F083
:101540009FFD8CE7FFF790FED8E7FFF78DFEEDE7F4
:10155000002504953A4B1A6C42F480421A641A6CC6
:1015600002F480420492049A05951A6B42F0040238
:101570001A631A6B02F004020592059A06951A6B1B
:1015800042F002021A631B6B03F002030693069BF0
:101590000C2307934FF00209CDF820904FF0030879
:1015A000CDF8288005270B9707A92C4802F09EF953
:1015B0004FF480660796CDF820900995CDF82880E5
:1015C0000B9707A9204802F091F92548254B0360A5
:1015D000456040238360C560066145618561C561E2
:1015E0000562456200F002FE00BB1D4BA3649C63D4
:1015F0001D481E4B0360002343608360C3604FF4AB
:101600008062026143618361C3610362436200F0EF
:10161000EDFD70B9144BE3649C6300220521242086
:1016200000F00AFD242000F02BFD18E7FFF71CFE58
:10163000DBE7FFF719FEEDE700300140003800401E
:101640000038024000000240000402403006002042
:1016500010640240D0050020586402400008024097
:1016600070050020706002401005002058600240A4
:1016700000B583B0002200920D4B596C41F48041BB
:101680005964596C01F48041009100990192196CE0
:1016900041F0805119641B6C03F080530193019B4E
:1016A0000F216FF0010000F0C7FC03B05DF804FBF0
:1016B0000038024030B589B00546002401941E4B25
:1016C0005A6C42F480225A645B6C03F480230193C9
:1016D000019B02A903A802F01DFF02F00BFF4300CB
:1016E000164AA2FB03239B0C013B1548154A0260D6
:1016F00040F2E732C260436004618460846103F0B9
:101700003BFF044610B1204609B030BD0C4803F041
:1017100089FD04460028F6D11A2000F0B1FC0F2DF7
:1017200001D90124EFE7002229461A2000F084FCA9
:10173000054B1D60E7E700BF0038024083DE1B4316
:10174000400700200048014008000020FEE7FEE7B7
:10175000FEE7FEE7FEE7704708B5024800F0EEFE40
:1017600008BD00BF1005002008B5024800F0E6FEE5
:1017700008BD00BF7005002008B5034803F0DAFD7E
:10178000024803F0D7FD08BD640800204007002090
:1017900008B5024803F080FC08BD00BFE806002041
:1017A00008B5024803F078FC08BD00BF9006002091
:1017B00008B5024803F0BEFD08BD00BFD4070020F5
:1017C00008B5024803F0B6FD08BD00BF8C07002035
:1017D00008B5024800F0B2FE08BD00BF3006002088
:1017E00008B5024800F0AAFE08BD00BFAC08002002
:1017F00008B5024800F0A2FE08BD00BFD0050020D9
:1018000008B5024801F05EFC08BD00BFE4090020F5
:1018100001207047024B16221A604FF0FF307047CC
:10182000301A012008B54FF0FF31FFF7F3FFFEE754
:1018300070B50C461646002506E0AFF30080214641
:1018400001F8010B01350C46B542F6DB304670BDA0
:101850004FF0FF3070474FF400534B60002070474B
:10186000012070470020704710B403460C4A0D4910
:101870000D48006850B10C4800680344521A934266
:1018800008D8094A13605DF8044B70470648074CB6
:101890000460F0E7064B0C221A604FF0FF30F2E7CD
:1018A000000002200010000088070020381A0120E4
:1018B000301A0120034AD2F8883043F47003C2F88A
:1018C0008830704700ED00E000B587B00023029338
:1018D000039304930593009301931548154A0260FE
:1018E0008F224260836042F20F72C26003614361E3
:1018F000836103F041FE90B94FF48053029302A933
:101900000B4803F0DFFE68B900230093019369469A
:10191000074804F057F940B907B05DF804FBFFF73A
:10192000A3FCE9E7FFF7A0FCEEE7FFF79DFCF3E778
:10193000640800200000014000B587B00023029336
:10194000039304930593009301931548154A02608D
:1019500047224260836042F20F72C260036183617A
:1019600003F00AFE90B94FF48053029302A90C4889
:1019700003F0A8FE68B90023009301936946084864
:1019800004F020F940B907B05DF804FBFFF76CFCE8
:10199000E9E7FFF769FCEEE7FFF766FCF3E700BF56
:1019A0001C0800200004004000B583B00023009311
:1019B00001930F480F4A02604722426083604FF64E
:1019C000FF72C260836103F0D7FD50B9002300931A
:1019D00001936946064804F0F5F828B903B05DF8AC
:1019E00004FBFFF741FCF1E7FFF73EFCF6E700BF21
:1019F000D40700200010004000B583B000230093FE
:101A000001930F480F4A02605122426083604FF6F3
:101A1000FF72C260836103F0AFFD50B900230093F1
:101A200001936946064804F0CDF828B903B05DF883
:101A300004FBFFF719FCF1E7FFF716FCF6E700BF20
:101A40008C0700200014004000B585B003682C4AC4
:101A500093420BD02B4A93421CD02B4A934226D060
:101A60002A4A934237D005B05DF804FB0022009269
:101A7000274B596C41F0010159645B6C03F0010381
:101A80000093009B0F211A2000F0D6FA1A2000F0D4
:101A9000F7FAE8E7002301931D4B1A6C42F00202AB
:101AA0001A641B6C03F002030193019BDBE7002225
:101AB0000292174B196C41F0100119641B6C03F072
:101AC00010030293029B0521362000F0B5FA362060
:101AD00000F0D6FAC7E7002203920D4B196C41F0D3
:101AE000200119641B6C03F020030393039B052161
:101AF000372000F0A1FA372000F0C2FAB3E700BFA8
:101B000000000140000400400010004000140040AC
:101B10000038024008B50A480A4B03604FF4E1233D
:101B2000436000238360C36003610C2242618361D0
:101B3000C36104F0D1F900B908BDFFF795FBFBE7DD
:101B40000C0900200010014030B589B00023039338
:101B50000493059306930793026803F1804303F50A
:101B600088339A4201D009B030BD04460025019562
:101B700003F594335A6C42F010025A645A6C02F026
:101B800010020192019A02951A6B42F001021A6347
:101B90001B6B03F001030293029B4FF4C06303939A
:101BA00002230493032306930723079303A90E48F4
:101BB00001F09CFE0D480E4B03604FF00063436044
:101BC0008560C5604FF48063036145618561C561CF
:101BD0000562456200F00AFB18B9044BA3639C63DD
:101BE000C1E7FFF741FBF8E700000240AC08002026
:101BF00040640240DFF834D00D480E490E4A0023FD
:101C000002E0D458C4500433C4188C42F9D30B4AB0
:101C10000B4C002301E013600432A242FBD3FFF718
:101C200049FE10F043FEFFF777FB704700000220EB
:101C300000000020280200202C8B01082802002030
:101C4000341A0120FEE708B510B10246002307E070
:101C500072B6FFF709FBFEE7002142F823100133BB
:101C6000012BF9D90023137208BD08B590B10346C2
:101C7000027A012A12D8511C0172EFF311814FF040
:101C8000500080F31188BFF36F8FBFF34F8F43F87D
:101C9000221008BD72B6FFF7E7FAFEE772B6FFF74B
:101CA000E3FAFEE708B550B1037A013BDBB20372F9
:101CB000012B08D850F8233083F3118808BD72B681
:101CC000FFF7D2FAFEE772B6FFF7CEFAFEE70000A2
:101CD00048B110B504460C200FF0C6FB206030B1AF
:101CE000FFF7B1FF10BD044B16221A60704772B6A1
:101CF000FFF7BAFAFEE700BF301A012008B510B1AD
:101D0000FFF7B3FF08BD72B6FFF7AEFAFEE708B5FE
:101D100010B1FFF7C7FF08BD72B6FFF7A5FAFEE7DF
:101D200088B1CA6892B18A689AB10A69A2B10A6890
:101D300082604A68C260CA6842618A6802610A6950
:101D40008261002070474FF0FF3070474FF0FF3046
:101D500070474FF0FF3070474FF0FF30704770B55D
:101D600082B00546002301934468002C4AD1836861
:101D700003B1984720232B60002602E06FF0040691
:101D800001341F2C0DD86B6901AA122120469847F7
:101D90000028F3DB019B03F01F03A342F0D12C606A
:101DA000002628681F2826D8002E37D12B694FF42B
:101DB000004200219847002833DB6B6901AA00210B
:101DC0002868984700282FDBAB6998470446019B99
:101DD00013F4004F11D0AB699847001BB0F5FA7FA0
:101DE0000DD86B6901AA0021286898470028EEDA0F
:101DF0006FF0040601E06FF002067EB903E06FF0B9
:101E00000106FAE70026AB6998470446AB69984794
:101E1000031BB3F5FA6FF9D901236B60304602B0AA
:101E200070BD6FF00306F9E76FF00406F6E710B532
:101E300082B0044600230193436901AA012100688E
:101E40009847002839DB636901AA01212068984777
:101E5000002835DB019B13F0040F34D0636901AA1D
:101E6000002120689847002830DB019B13F4805F35
:101E70000CD103F40452B2F5045F2AD013F4005FCE
:101E800029D113F4807F28D004201DE0636901AAC2
:101E90001F2120689847002821DB019B13F4805FF5
:101EA00020D003F01C03182B1ED0082B1ED0142B9F
:101EB00001D0052008E0042006E06FF0040003E0F4
:101EC0006FF0040000E0012002B010BD6FF00400CC
:101ED000FAE70220F8E70320F6E70520F4E76FF0C1
:101EE0000400F1E70620EFE70220EDE70320EBE72F
:101EF00008B50B4B1A6842F400721A601A6842F473
:101F000080621A601A6842F480721A60032000F03E
:101F100075F80F20FFF7CEFBFFF7AAFB002008BDE6
:101F2000003C0240034A1168034B1B780B441360CA
:101F3000704700BF6809002004000020014B1868AA
:101F4000704700BF6809002038B50446FFF7F6FF68
:101F50000546B4F1FF3F02D0044B1B781C44FFF749
:101F6000EDFF401BA042FAD338BD00BF04000020A3
:101F7000002808DB0901C9B200F1604000F56140AA
:101F800080F80013704700F00F000901C9B2014B3F
:101F90001954704714ED00E000B500F00700C0F1DF
:101FA000070CBCF1040F28BF4FF0040C031D062BD7
:101FB0000FD9C31E4FF0FF3E0EFA0CF021EA0001CC
:101FC00099400EFA03FE22EA0E0241EA02005DF891
:101FD00004FB0023EEE70000BFF34F8F0549CA68FA
:101FE00002F4E062044B1343CB60BFF34F8F00BF9A
:101FF000FDE700BF00ED00E00400FA0510B504465F
:10200000C31E042B0FD80A4AD36823F4E0631B04D1
:102010001B0C240204F4E064234343F0BF6343F445
:102020000033D36010BD90210248FFF795F9EAE72D
:1020300000ED00E0C85D010870B506460C46154687
:102040000F2A0ED80F2C11D80B4BD8682A462146E0
:10205000C0F30220FFF7A0FF01463046FFF788FFDC
:1020600070BDA8210548FFF777F9EBE7A9210348E0
:10207000FFF772F9E8E700BF00ED00E0C85D010876
:1020800008B5002808DB00F01F0240090123934037
:10209000044A42F8203008BDBC210348FFF75CF930
:1020A000F9E700BF00E100E0C85D010808B5FFF7EF
:1020B00093FF0000A0B110B504460268094B9A4294
:1020C00003D068210848FFF747F963791BB1012362
:1020D0006371002010BD23712046FEF793FFF6E7E1
:1020E0000120704700300240045E010830B40568EA
:1020F0002C6824F480242C60046863608368402B7F
:1021000005D0036899600368DA6030BC70470368E3
:102110009A600368D960F8E710B40368D9B210393F
:102120000C4AA2FB014212090B4CA25CC2655F295A
:1021300009D923F47F7323F0030304338365806D8F
:102140005DF8044B704723F47F7323F0030383652A
:10215000F5E700BFABAAAAAA745E0108836A826988
:1021600092B9012B0AD0022B02D00BB1002070478C
:10217000C36A13F0807F28D100207047C36AB3F18F
:10218000C07F24D000207047B2F5005F09D0022B39
:1021900025D9032B25D1C36A13F0807F23D10020DA
:1021A0007047032B03D8DFE803F01404140A00205F
:1021B0007047C36A13F0807F0DD100207047C36A57
:1021C000B3F1C07F09D00020704701207047012083
:1021D000704701207047012070470120704701209F
:1021E00070470020704701207047000070B504461A
:1021F000FFF7A4FE002C00F03E8105462368954AB7
:10220000934231D0183293422ED0183293422BD0C1
:102210001832934228D01832934225D01832934274
:1022200022D0183293421FD0183293421CD002F5AC
:102230005672934218D01832934215D018329342F6
:1022400012D0183293420FD0183293420CD0183269
:10225000934209D01832934206D01832934203D0E9
:10226000B7217D48FFF778F86368A3B1B3F1007F29
:1022700011D0B3F1806F0ED0B3F1C06F0BD0B3F1BA
:10228000006F08D0B3F1206F05D0B3F1406F02D0DA
:10229000B3F1606F6DD1A3681BB1402B01D0802BCF
:1022A0006CD1E368B3F5007F01D0002B6BD12369BB
:1022B000B3F5806F01D0002B6AD163692BB1B3F500
:1022C000006F02D0B3F5805F67D1A3692BB1B3F57E
:1022D000005F02D0B3F5804F64D1E36923B1B3F559
:1022E000807F01D0202B62D1236A43B1B3F5803FB8
:1022F00005D0B3F5003F02D0B3F5403F5CD1636A2F
:102300000BB1042B5DD1636AC3B1A36A032B5DD803
:10231000E36A43B1B3F5000F05D0B3F1807F02D07B
:10232000B3F1C07F57D1236B43B1B3F5001F05D084
:10233000B3F5800F02D0B3F5C00F51D1022384F85A
:102340003530002384F834302268136823F0010309
:10235000136023681A6812F0010F46D0FFF7EEFDF4
:10236000401B0528F5D920236365032084F8350038
:1023700070BDB8213848FEF7EFFF8CE7B921364829
:10238000FEF7EAFF8DE7BA213348FEF7E5FF8EE757
:10239000BB213148FEF7E0FF8FE7BC212E48FEF756
:1023A000DBFF92E7BD212C48FEF7D6FF95E7BE2163
:1023B0002948FEF7D1FF97E7BF212748FEF7CCFF5A
:1023C0009DE7C0212448FEF7C7FF9CE7C5212248AE
:1023D000FEF7C2FF9CE7C6211F48FEF7BDFFA2E73C
:1023E000C7211D48FEF7B8FFA8E71A681B4911402E
:1023F0006268A0680243E0680243206902436069A2
:102400000243A0690243E0690243206A02430A438F
:10241000616A042924D01A602668756925F00705C9
:10242000636A1D43042B07D1A36A1D43E36A1BB1F2
:102430002046FFF793FEC0B975612046FFF76CFE9A
:10244000E26D3F239340836000206065012384F8A0
:1024500035308DE7106002403C5E01083F8010F08F
:10246000E16A206B01430A43D5E7402363650120FD
:1024700084F835007CE701207AE700BF2DE9F041C0
:1024800004460E4617461D46D0F858805A1E4FF691
:10249000FE739A4211D894F83430012B36D00123C0
:1024A00084F8343094F83530DBB2012B0BD00023A4
:1024B00084F834300220BDE8F08140F2CB1114489A
:1024C000FEF74AFFE7E7022384F83530002363650F
:1024D0002B463A4631462046FFF708FEE26D3F2381
:1024E0009340C8F808302268136843F0160313605D
:1024F000236C23B12268136843F008031360226839
:10250000136843F0010313600020D4E70220D2E7F0
:102510003C5E010890F83530DBB2022B03D08023FB
:10252000436501207047052380F835300268136841
:1025300023F001031360002070470000F0B583B062
:10254000044600230193724B1D68724BA3FB0535B3
:10255000AD0A876D3E68C26D08239340334210D0A8
:1025600003681A6812F0040F0BD01A6822F00402F4
:102570001A60C26D08239340BB60436D43F00103B2
:102580004365E26D01239340334209D022685269CA
:1025900012F0800F04D0BB60636D43F002036365EB
:1025A000E26D04239340334209D02268126812F08E
:1025B000020F04D0BB60636D43F004036365E26DFA
:1025C00010239340334224D02268126812F0080F7F
:1025D0001FD0BB6023681A6812F4802F0DD01B68CF
:1025E00013F4002F04D1236C9BB12046984710E0D0
:1025F000A36C73B1204698470BE01A6812F4807FF1
:1026000003D11A6822F008021A60236C0BB120462D
:102610009847E26D20239340334255D022681268D8
:1026200012F0100F50D0BB6094F83530DBB2052BA0
:102630000ED023681A6812F4802F33D01B6813F46D
:10264000002F2AD1636C002B3ED0204698473BE0F8
:102650002268136823F0160313602268536923F07D
:1026600080035361236CA3B12268136823F008032D
:102670001360E26D3F239340BB60012384F8353043
:10268000002384F83430236D002B3FD02046984738
:102690003CE0A36C002BE7D1EBE7E36BA3B1204652
:1026A000984711E01A6812F4807F09D11A6822F065
:1026B00010021A60012384F83530002384F8343086
:1026C000E36B0BB120469847636DFBB1636D13F06C
:1026D000010F17D0052384F835302268136823F0E2
:1026E00001031360019B01330193AB4204D82368BB
:1026F0001B6813F0010FF5D1012384F83530002356
:1027000084F83430E36C0BB12046984703B0F0BD39
:1027100000000020B5814E1B2DE9F04182B0074634
:1027200000230193D0F8688008F1120350F8234089
:10273000C56E012613E001A803F0C8FF019B13B189
:102740002362A36010E000260EE04FF48C43636028
:1027500011E003F1120257F82240013D9846BDB145
:10276000B6B1236A002BE6D0002EF8D0BB6D002B4B
:10277000EBD10E4B6360BFF35F8F236843F00043E0
:10278000236008F10103032BE3D9A8F10303E0E779
:10279000FB6EAB4207D03B6803F5805300229A6082
:1027A000C7F86880FD6602B0BDE8F0810046008091
:1027B0005079137943EA002307480B50D078937877
:1027C0001B0443EA0063507843EA00231278134362
:1027D000024A8B50704700BF408002404480024054
:1027E00030B4002208E0C468DC6051F80C3043F4D7
:1027F000400341F80C300132032A1FD8C16802EBB4
:1028000082034FEAC30C01EBC303002441F80C40E0
:102810005C609C60DC60941D40F8243051F80C40F2
:1028200044F4801441F80C40022ADCD8541C04EB18
:102830008404C56805EBC404DC60D6E7002383622A
:10284000C268036803F580531A6130BC704700B555
:102850004FF0000E03E00269DA600EF1010EBEF1E6
:10286000030F29D801690EEB8E034FEAC30C01EB6D
:10287000C303002241F80C205A609A60DA601A62A1
:102880005A624FF0004241F80C204FF48C425A60DB
:102890005A6822F000425A600EF1120240F82230CB
:1028A000BEF1020FD7D801690EF1010202EB8202DC
:1028B00001EBC201D960D0E70023C36503668366DC
:1028C000C36683650269036803F58053DA605DF8C7
:1028D00004FBF0B5856A00EB85039B698C681E6874
:1028E000002EC0F2AF802E1D00EB8606F669002E8A
:1028F00040F0AA8026689E605E6826F4FF5626F0A7
:102900001F0667683E435E600E6816F0010F05D033
:102910001E6826F440064F693E431E600E6816F09E
:10292000200F05D01E6826F040660F693E431E60EA
:10293000096811F0040F03D0196841F08001196093
:10294000196841F080511960BFF35F8F196841F039
:10295000004119602F4600264FF0010E29E019684A
:1029600021F08041196030E000EB8C039B6919680D
:1029700021F080511960196800292EDB0CF1040147
:1029800000EB8101C96941BB0EF1010EA468216809
:102990009960596821F4FF5121F01F01676839439C
:1029A00059600136BFF35F8F196841F0004119602B
:1029B0006746A16851B3196821F000511960002AD7
:1029C000CDD0196841F08041196007F1010CBCF1CC
:1029D000030FC9D9A7F1030CC6E700EB850399697A
:1029E000002204E000EB8301896901321D46724533
:1029F0000AD2BFF35F8F0B6823F000430B606B1CA0
:102A0000032BEFD9EB1EEDE70220F0BDAAB11A6847
:102A100042F080421A601A6842F000521A60C26B9B
:102A20003B1D00EB8303DA61876272B6036C3344AB
:102A30000133036462B60020E7E71A6822F080429F
:102A40001A60E8E70220E0E70220DEE770B50546FD
:102A50000C46026813683B491940237C002B60D167
:102A60004FF40003607C00285DD14FF480000343E5
:102A7000A0680343E07F43EA004360690343A07F0B
:102A8000002852D14FF400500343207F43EA003323
:102A9000A0690343207943EA802394F820000028AA
:102AA00045D14FF400700343E07B43EAC013606AF2
:102AB000034394F8280043EA00130B4313602B6888
:102AC0001E680120FFF740FA2B681E6029688A699A
:102AD00022F0BE021204120CA36C1B0494F84C00EA
:102AE00038BB80200343206D034394F85500012830
:102AF00021D00020034394F8560001281DD0002067
:102B0000034394F85400012819D0002003431343D1
:102B10008B612B689C690120FFF716FA2B689C617A
:102B200070BD00239EE70020A1E70020ACE7002055
:102B3000B9E70020D6E70820DCE70420E0E7022020
:102B4000E4E700BF0F8120FF70B505460C46026820
:102B500002F580539B692B491940237B002B4DD1F3
:102B60004FF08063607B43EA4063607F002847D179
:102B70004FF480100343A07B43EA40536069034352
:102B8000207F43EAC013A07F43EA8013206A0343F7
:102B900094F8240043EA80030B4302F580529361CA
:102BA0002B6803F580539E690120FFF7CDF92B6850
:102BB00003F580539E612279A36843EA4263A269C8
:102BC00013432269134394F8252043EAC213A26AEF
:102BD00043EA8203226813432A6843F4000302F5A0
:102BE000805213602B6803F580531C680120FFF7A7
:102BF000ABF92B6803F580531C6070BD0023B1E76F
:102C00000020B7E7233FDEF870B5A4B006460125E3
:102C10008DF83C508DF83D5000240D948DF84B40BC
:102C20008DF84A508DF848408DF830508DF84C4062
:102C30008DF83B4014948DF854401D948DF87840E5
:102C40001F948DF882408DF880404FF4804310939C
:102C50004FF4006311938DF881400BA9FFF7F6FE46
:102C60008DF80C508DF80D508DF81D508DF80E50CC
:102C700005948DF81C408DF81E4008948DF8245062
:102C80008DF804504FF4803302934FF48003069381
:102C90004FF4005304938DF825500A94009469462C
:102CA0003046FFF751FF24B070BD10B582B0044626
:102CB00000230193036803F580539A6942F480125C
:102CC0009A61036803F580539B6901930120FFF724
:102CD0003BF92368019A03F580539A6102B010BD55
:102CE000002857D030B583B00446D0F88430002B8C
:102CF00034D000230193284B5A6C42F480425A642A
:102D00005B6C03F480430193019B244B5A6822F4CB
:102D100000025A605A68A1680A435A605B682368D7
:102D200003F580531A6842F001021A60FFF706F9B2
:102D30000546236803F580531B6813F0010F13D079
:102D4000FFF7FCF8401BB0F5FA7FF2D90423C4F872
:102D50008830E023C4F88430012019E02323C0F830
:102D6000843003F0BDFBC4E72046FFF74DFF20464B
:102D7000FFF736FD2046FFF76AFD62680021204616
:102D8000FFF716FD0020C4F888001023C4F8843033
:102D900003B030BD012070470038024000380140C8
:102DA000F8B5D0F88430102B01D00120F8BD0446CE
:102DB0002325C0F88450012686650268D36B43F44E
:102DC0000273D3630268D2F80C3143F4003343F04A
:102DD0006003C2F80C310268D2F8103143F40313D7
:102DE000C2F810310423C366FFF796FC226813680B
:102DF00043F00803136023681F683046FFF7A4F808
:102E000023681F602268136843F00403136023687B
:102E10001F683046FFF798F823681F602046FFF7C9
:102E200044FF236803F580539A6942F400529A6183
:102E3000236803F580539A6942F002029A6122687E
:102E400002F58052D36943F4D03343F0C103D36118
:102E5000C4F884500020A9E738B5D0F88430232B7B
:102E600001D0012038BD0446C0F88430026802F564
:102E70008052D36923F4D03323F0C103D3610368B4
:102E800003F580539A6922F400529A61036803F5AE
:102E900080539A6922F002029A610268136823F053
:102EA0000403136003681D680120FFF74DF82368D1
:102EB0001D602046FFF7F9FE2268136823F008031F
:102EC000136023681D680120FFF73EF823681D602A
:102ED000002308E003F1120254F822104A6842F07D
:102EE00000424A600133032BF4D90020A06510236F
:102EF000C4F88430B6E710B5044629B1D4F884305C
:102F0000232B09D0012010BDD0F8883043F00103F5
:102F1000C0F888300120F6E74B6BE36301222046BE
:102F2000FFF7D7FC38B1D4F8883043F00203C4F877
:102F300088300120E7E7BFF34F8FA36A5A1CA262D3
:102F4000032A01D9033BA362236803F58052526927
:102F500012F0040F08D003F5805304225A6123684D
:102F600003F5805300225A600020CCE72DE9F84F8A
:102F7000044689B18B46D0F88430232B72D1D0F827
:102F80005C8008F1120350F82350C36EC3F1040AA9
:102F90004FF000094F4638E0D0F8883043F0010385
:102FA000C0F8883001205EE02B6813F4007F02D067
:102FB00000232366636666692B6813F4807F07D05D
:102FC0002E68C6F30D46043E2B6823674FF00109B7
:102FD000AA682A62B3B204F1800104F17C0003F014
:102FE0009BFB236E01332366636E334463660023C9
:102FF0002B6208F10103032B01D9A8F1030303F1AC
:10300000120254F82250013798462B68002B14DB2B
:10301000574512D2B9F1000F0FD12B6813F4807FFE
:1030200003D0AB69A367EB6963672B6813F4007F78
:10303000BAD1E36F002BB7D1DBE7E36E3B44E36625
:1030400033B9C4F85C80B9F1000F05D101200AE062
:103050002046FFF761FBF4E7E36FCBF80030002078
:10306000E06700E00120BDE8F88FF8B50646056C82
:10307000446C012702E0013404F00304EDB1E7B130
:10308000013D231D06EB8303D8690028F3D0F268C5
:1030900004EB8403DB00D358002B01DA0027EDE7B3
:1030A00003F055FB231D06EB83030022DA61013494
:1030B00004F0030435647464E0E70020F8BD704751
:1030C0007047000010B50446036803F5805252694A
:1030D00012F0400F05D003F58052D26912F0400F74
:1030E00047D1236803F58052526912F0010F05D0D1
:1030F00003F58052D26912F0010F41D1236803F524
:103100008052526912F4004F28D003F58052D269E0
:1031100012F4004F22D0D4F8882042F00802C4F8FC
:10312000882003F58052526912F4005F31D003F514
:1031300080535A6922F07F4222F4010222F45F4256
:1031400022F0FF02C4F88C20DA6922F4C032DA617E
:10315000E023C4F88430204603F088F923689A6B92
:1031600012F0080F1FD11A4B5B6913F4002F26D100
:1031700010BD03F58053174A5A6103F067F9B0E7B1
:1031800003F580534FF001125A61204603F066F9AF
:10319000B4E703F580535A6948F280610A40C4F8E5
:1031A0008C205961D7E7DB6A03F06003C4F89430E0
:1031B0002046FFF784FF0023C4F89430D3E7044B84
:1031C0004FF400225A612046FFF77AFFD0E700BF94
:1031D000003C014040000100F8B505461E4600686D
:1031E000036903F01C03C90289B21943940104F472
:1031F000F8640C4344F001040461FEF79FFE0746A7
:1032000001E02B681C6914F0010F07D0FEF796FE51
:10321000C01BB0F5803FF4D3012004E02B685B694C
:103220009BB233600020F8BD70B505460668306972
:1032300000F01C00C90289B20143940104F4F8644F
:103240000C4344F003049BB273612B681C61FEF7CE
:1032500075FE064601E02B681C6914F0010F07D0CB
:10326000FEF76CFE801BB0F5803FF4D3012000E038
:10327000002070BD002974D002681268C2F30012E9
:1032800081F828200268126802F060024A6202682F
:10329000126812F4007F0CBF0122002281F8202066
:1032A00002681268C2F30042CA770268126812F418
:1032B000005F0CBF012200228A7702681268C2F305
:1032C00000320A770268126802F400628A610268BA
:1032D000126802F480424A610268126812F4800F98
:1032E0000CBF012200224A740268126812F4000F17
:1032F0000CBF012200220A7402681268C2F3C012D5
:10330000CA730268126802F460228A600268126856
:10331000C2F380220A7102689269C2F3400281F806
:1033200054200268926912F0800F0CBF0122002223
:1033300081F84C200268926902F030020A65026846
:103340009269120C8A6402689269C2F3800281F861
:10335000562002689269C2F3C00281F8552000200D
:1033600070470120704751B108B5D0F88430102B58
:1033700001D0012008BDFFF769FB0020FAE701201A
:103380007047000038B5054603681C6924F01C042A
:1033900001F09AF8104B0344104A934204D244F0CF
:1033A00008042B681C6138BD0D4B03440D4A934241
:1033B00002D844F00C04F4E70B4B03440B4A93424D
:1033C000EFD30B4B03440B4A934202D844F004045E
:1033D000E7E744F01004E4E700D3CEFEC0E1E400E8
:1033E00040F1E9FD3F787D0100796CFC005A6202F2
:1033F000001F0AFA7FF0FA02D0F88C007047000034
:10340000204BDB6813F0100F07D01F4AD36943F03D
:103410001003D3611B4B1022DA601A4BDB6813F0E8
:10342000200F07D0184AD36943F00803D361154B26
:103430002022DA60134BDB6813F0400F07D0124AEA
:10344000D36943F00403D3610E4B4022DA600D4B85
:10345000DB6813F0800F07D00B4AD36943F00203F7
:10346000D361084B8022DA60064BDB6813F0020F51
:1034700007D0054AD36943F02003D361014B0222F0
:10348000DA607047003C02406C09002038B5044601
:103490000D4600F17843B3F5801F06D300F1604379
:1034A00003F50843B3F5047F0CD2094B1A6922F4E3
:1034B00040721A611A691A611A6942F001021A61AE
:1034C000257038BD40F2B9210248FDF745FFECE711
:1034D000003C02407C5E010838B504460D4600F110
:1034E0007843B3F5801F06D300F1604303F508432A
:1034F000B3F5047F0ED20A4B1A6922F440721A61A6
:103500001A6942F480721A611A6942F001021A6162
:10351000258038BD4FF428710248FDF71DFFEAE70A
:10352000003C02407C5E010838B504460D4600F1BF
:103530007843B3F5801F06D300F1604303F50843D9
:10354000B3F5047F0ED20A4B1A6922F440721A6155
:103550001A6942F400721A611A6942F001021A6192
:10356000256038BD40F287210248FDF7F5FEEAE705
:10357000003C02407C5E010870B5044616461D46BC
:1035800000F17843B3F5801F06D300F1604303F5E3
:103590000843B3F5047F11D20B490B6923F4407340
:1035A0000B610B6943F440730B610B6943F001033A
:1035B0000B612660BFF36F8F656070BD40F26521BF
:1035C0000248FDF7C9FEE7E7003C02407C5E0108C7
:1035D000094B1B69002B01DB00207047064B074A93
:1035E0005A6002F188325A601B69002B01DB00200F
:1035F00070470120704700BF003C0240230167452F
:10360000034A136943F0004313610020704700BF71
:10361000003C024038B50446144B0022DA61FEF744
:103620008DFC0546124BDB6813F4803F0AD0B4F1E1
:10363000FF3FF7D024B1FEF781FC401BA042F1D937
:1036400003200DE00A4BDB6813F0010F02D0084B9A
:103650000122DA60064BDB6813F0F20F01D1002083
:1036600038BDFFF7CDFE0120FAE700BF6C0900204E
:10367000003C0240F8B516461E4A127E012A37D099
:1036800004460D461F461B4B01221A7603281BD801
:103690004CF25030FFF7BEFF90B9D4B1012C1DD0D1
:1036A000022C20D032463B462846FFF765FF4CF2FD
:1036B0005030FFF7AFFF104A136923F00103136185
:1036C0000C4B00221A76F8BDA2210C48FDF744FEEF
:1036D000DEE7F1B22846FFF7D9FEE8E7B1B22846A7
:1036E000FFF7FAFEE3E731462846FFF71DFFDEE766
:1036F0000220E8E76C090020003C02407C5E0108E3
:1037000038B504460D46032811D8012D15D10E4BAE
:103710001A6922F440721A611A6942F004021A61AD
:10372000186940EA042040F48030186138BD40F246
:10373000BA310648FDF710FEE7E740F2BB31034817
:10374000FDF70AFEE3E700BF003C0240B85E010857
:1037500038B505460C460B2809D8032C0DD8ACB15A
:10376000012C2BD0022C0ED04FF440710FE040F210
:10377000D9311448FDF7F0FDEFE740F2DA31114896
:10378000FDF7EAFDEBE74FF4007100E000210E4B7E
:103790001A6922F440721A611A690A431A611A6995
:1037A00022F0F8021A61186940EAC50040F00200F0
:1037B00018611A6942F480321A6138BD4FF4807181
:1037C000E5E700BFB85E0108003C0240164B1B68ED
:1037D00013F4007F10D0144B1A6822F400721A60A0
:1037E0001A6842F400621A601A6822F400621A60D1
:1037F0001A6842F400721A600B4B1B6813F4806F56
:1038000010D0094B1A6822F480621A601A6842F4D8
:1038100080521A601A6822F480521A601A6842F4C0
:1038200080621A60704700BF003C0240F8B52C4B24
:103830001B7E012B52D004460E46294B01221A76DC
:103840000368934229D84CF25030FFF7E3FE074655
:1038500000283ED14FF0FF3333602368012B21D085
:10386000E368A2681344013B0B2B2AD8A568E368E0
:10387000A2681344AB422AD9217C2846FFF768FF8F
:103880004CF25030FFF7C6FE164A136923F0FA03D4
:1038900013610746D0B90135E9E7A9211248FDF7C0
:1038A0005BFDD0E76168207CFFF72AFF4CF25030C7
:1038B000FFF7B0FE07460B4A136923F004031361B8
:1038C00005E0C1210848FDF747FDCFE73560FFF768
:1038D0007DFF034B00221A763846F8BD0227FBE72E
:1038E0006C090020003C0240B85E01082DE9F0415F
:1038F00082B007460E46A84B984223D003F580635A
:1039000098421FD003F5806398421BD003F5806373
:10391000984217D003F58063984213D003F5806373
:1039200098420FD003F5806398420BD003F5806373
:10393000984207D003F58063984203D0AC219748A2
:10394000FDF70AFD33689AB212B1B3F5803F03D395
:10395000AD219248FDF700FD7368012B10D9B3F536
:10396000041F0DD011D8B3F5881F09D003D9B3F5C2
:10397000901F05D012E0032B04D9113B012B0DD869
:10398000002486E0022B09D3FAE7B3F5441FF7D0F1
:10399000B3F5481FF4D0B3F5081FF1D0AE217F482E
:1039A000FDF7DAFCECE7F368032B13D8BA68610083
:1039B00003238B4022EA0302F3688B401343BB606E
:1039C0007A6822EA05027368C3F30013A340134325
:1039D0007B606FE0C0217148FDF7BEFCE6E7D121B6
:1039E0006E48FDF7B9FC6DE033694BB10D2B05D87E
:1039F00033B9DE216948FDF7AFFC01E00F2BF8D1A8
:103A0000E208083257F8220004F0070189000F236A
:103A10008B4020EA030033698B40034347F8223090
:103A20005FE0072300E000238B40034302325C4940
:103A300041F822305B4B9A686FEA080322EA0801DA
:103A4000706810F4801F01D048EA0201554A916065
:103A5000D26803EA0201706810F4001F01D048EA3E
:103A60000201504AD160526803EA0201706810F402
:103A7000003F01D048EA02014A4A516012681340EF
:103A8000716811F4803F01D048EA0203454A13608F
:103A900001340F2C7CD80125A540336803EA0508C2
:103AA00035EA0303F4D1736803F00303013B012BF0
:103AB0007FF679AF736803F00303032B0CD0B36870
:103AC000022B8CD8FA68610003238B4022EA0302A0
:103AD000B3688B401343FB60736803F00303022B4E
:103AE00082D03A68610003238B4022EA03027368A4
:103AF00003F003038B4013433B60736813F4403FB0
:103B0000C6D000230193284B5A6C42F480425A6479
:103B10005B6C03F480430193019BA208911C204B32
:103B200053F8210004F0030189000F238B4020EAA1
:103B30000300194B9F423FF476AF03F580639F4229
:103B40001AD003F580639F4218D003F580639F422B
:103B500016D003F580639F4214D003F580639F4223
:103B600012D003F580639F4210D003F580639F421B
:103B70003FF457AF082357E7012355E7022353E7E4
:103B8000032351E704234FE705234DE706234BE7C3
:103B900002B0BDE8F08100BF00000240F85E0108FD
:103BA00000380140003C01400038024038B504466E
:103BB0000D4621B123691D4207D0012038BD4FF4C5
:103BC000BE710348FDF7C8FBF4E70020F6E700BF2D
:103BD000F85E010870B5054614460E4621B1012C69
:103BE00008D86CB1AE6170BD40F29D110648FDF77A
:103BF000B3FBF4E74FF4CF710348FDF7ADFBF0E7FB
:103C00003604AE61EFE700BFF85E010808B5054B6A
:103C10005B69034200D108BD024B58610CF096FC71
:103C2000F9E700BF003C0140002841D038B5044608
:103C30000268204B9A4203D0AE211F48FDF78CFB4F
:103C40006368062B25D8A368B3F5805F26D2236866
:103C50004CF6CC421A60236845F255521A6023682C
:103C600062685A602368A2689A60FEF767F90546A1
:103C70002368DA6812F0030F15D0FEF75FF9401BD6
:103C80003128F5D92368DB6813F0030FF0D0032047
:103C90000DE0AF210848FDF75FFBD4E7B0210648EF
:103CA000FDF75AFBD3E74AF6AA221A60002038BD76
:103CB0000120704700300040345F010803684AF675
:103CC000AA221A6000207047002800F0608270B5B8
:103CD00082B0044603680F2B39D8236813F0010F14
:103CE0004DD063682BB1B3F5803F02D0B3F5A02F60
:103CF00032D1804B9B6803F00C03042B36D07D4BF4
:103D00009B6803F00C03082B2BD06368B3F5803F4E
:103D10005FD0B3F5A02F62D0764B1A6822F48032C0
:103D20001A601A6822F480221A606368002B60D03F
:103D3000FEF704F905466F4B1B6813F4003F1ED1D4
:103D4000FEF7FCF8401B6428F5D9032026E2E621A3
:103D50006948FDF701FBC0E7EB216748FDF7FCFA76
:103D6000C7E7644B5B6813F4800FCED0614B1B68D0
:103D700013F4003F03D06368002B00F00A8223682D
:103D800013F0020F66D0E368012B41D823691F2B83
:103D900044D8584B9B6813F00C0F4AD0554B9B6886
:103DA00003F00C03082B3FD0E368002B77D0534B74
:103DB00001221A60FEF7C2F805464E4B1B6813F04D
:103DC000020F63D1FEF7BAF8401B0228F5D9032091
:103DD000E4E1484A136843F480331360A5E7454B98
:103DE0001A6842F480221A601A6842F480321A601B
:103DF0009BE7FEF7A3F805463E4B1B6813F4003F14
:103E0000BDD0FEF79BF8401B6428F5D90320C5E11F
:103E100040F21D113848FDF79FFAB7E74FF48F7154
:103E20003548FDF799FAB4E7324B5B6813F4800F1D
:103E3000BAD1304B1B6813F0020F03D0E368012B9B
:103E400040F0A9812B4A136823F0F803216943EA63
:103E5000C1031360236813F0080F51D06369012B6D
:103E60002FD863699BB3254B0122C3F8802EFEF740
:103E700065F805461F4B5B6F13F0020F40D1FEF74C
:103E80005DF8401B0228F5D9032087E1194A136821
:103E900023F0F803216943EAC1031360DAE7174B03
:103EA00000221A60FEF74AF80546124B1B6813F011
:103EB000020FCFD0FEF742F8401B0228F5D90320AD
:103EC0006CE14FF4AF710C48FDF746FAC9E70B4BB4
:103ED0000022C3F8802EFEF731F80546054B5B6FD4
:103EE00013F0020F0CD0FEF729F8401B0228F5D979
:103EF000032053E100380240705F01080000474290
:103F0000236813F0040F7CD0A368012B01D9052B83
:103F100038D1A54B1B6C13F0805F39D1002301937E
:103F2000A14B1A6C42F080521A641B6C03F0805350
:103F30000193019B01259D4B1B6813F4807F29D0C1
:103F4000A368012B3AD0052B3ED0974B1A6F22F075
:103F500001021A671A6F22F004021A67A368002B85
:103F60003CD0FDF7EBFF06468F4B1B6F13F0020FA3
:103F700045D1FDF7E3FF801B41F288339842F3D926
:103F800003200BE14FF4C5718948FDF7E5F9C0E75F
:103F90000025D0E7854A136843F480731360FDF76A
:103FA000CDFF0646814B1B6813F4807FC8D1FDF717
:103FB000C5FF801B0228F5D90320EFE07A4A136F72
:103FC00043F001031367C9E7774B1A6F42F004020D
:103FD0001A671A6F42F001021A67BFE7FDF7AEFFDA
:103FE0000646714B1B6F13F0020F08D0FDF7A6FFBA
:103FF000801B41F288339842F3D90320CEE0002D94
:104000003ED1A369022B41D8A369002B00F0C580E3
:10401000654A926802F00C02082A00F09380022B95
:104020007CD1E36913B1B3F5800F35D1236A3F2BFF
:1040300038D8636A323BB3F5BF7F39D8A36A022B05
:1040400008D0082B3AD84FF4A87222FA03F313F0E1
:10405000010F33D0E36A023B0D2B35D8554B0022BC
:104060001A66FDF76BFF05464F4B1B6813F0007F88
:1040700030D0FDF763FF401B0228F5D903208DE007
:10408000494A136C23F080531364BAE740F2CD1110
:104090004748FDF761F9B7E74FF4EB714448FDF786
:1040A0005BF9C3E740F2D7114148FDF755F9C0E786
:1040B0004FF4EC713E48FDF74FF9BFE740F2D911DC
:1040C0003B48FDF749F9C5E74FF4ED713848FDF776
:1040D00043F9C3E7E369226A1343626A43EA82133E
:1040E000A26A5208013A43EA0243E26A43EA0263DF
:1040F0002D4A53602F4B01221A66FDF71FFF04461D
:10410000294B1B6813F0007F06D1FDF717FF001B3A
:104110000228F5D9032041E000203FE0254B002292
:104120001A66FDF70BFF04461F4B1B6813F0007F58
:1041300006D0FDF703FF001B0228F5D903202DE070
:1041400000202BE0012B2BD0174B5B6803F4800180
:10415000E269914226D103F03F02216A8A422BD1C3
:10416000616A47F6C0721A40B2EB811F26D103F490
:104170004031A26A5208013AB1EB024F20D103F05C
:104180007063E26AB3EB026F1CD1002006E00120ED
:104190007047012002E0012000E0002002B070BD65
:1041A0000120FBE70120F9E70038024000700040E1
:1041B000705F0108000047420120EFE70120EDE7B2
:1041C0000120EBE70120E9E708B5334B9B6803F0DA
:1041D0000C03042B5BD0082B5BD12F4B5A6802F0E9
:1041E0003F025B6813F4800F2CD02B4B5868C0F350
:1041F00088104FEA401CBCEB000C6EEB0E0E4FEA31
:104200008E1343EA9C634FEA8C11B1EB0C0163EB14
:104210000E03DB0043EA5173C90011EB000C43F1BC
:104220000003590200234FEA4C2041EADC51FCF71D
:104230002BFD194B5B68C3F3014301335B00B0FBFB
:10424000F3F027E0144B5868C0F388104FEA401C85
:10425000BCEB000C6EEB0E0E4FEA8E1343EA9C6330
:104260004FEA8C11B1EB0C0163EB0E03DB0043EA68
:104270005173C90011EB000C43F1000399020023B4
:104280004FEA8C2041EA9C51FCF7FEFCD1E7034841
:1042900000E0034808BD00BF0038024000127A0069
:1042A0000024F400002800F0FA8070B50D460446A2
:1042B0000368013B0E2B30D8072D34D87C4B1B688C
:1042C00003F00703AB4208D2EBB2794A13701368CC
:1042D00003F00703AB4240F0E480236813F0020FC1
:1042E00032D013F0040F04D0724A936843F4E053C1
:1042F0009360236813F0080F04D06E4A936843F468
:1043000060439360A368C3B1C02B16D049D8A02BDB
:1043100013D00ED9B02B10D049E040F25A21664894
:10432000FDF71AF8C8E740F25B216348FDF714F87F
:10433000C4E7802B01D0902B39D15E4A936823F0DB
:10434000F003A1680B439360236813F0010F48D07A
:104350006368032B31D86368012B34D09A1E012A7D
:1043600038D9544A126812F0020F00F09C8051496B
:104370008A6822F0030213438B60FDF7DFFD0646D7
:104380004C4B9B6803F00C036268B3EB820F28D0A0
:10439000FDF7D4FD801B41F288339842F0D9032009
:1043A00070E0E02BC9D0F02BC7D0D02BC5D040F2A5
:1043B0007E214148FCF7D0FFBFE740F285213E480F
:1043C000FCF7CAFFC7E73B4A126812F4003FCED1A0
:1043D000012057E0374A126812F0007FC7D1012050
:1043E00050E0334B1B6803F00703AB4207D9EAB236
:1043F0002F4B1A701B6803F00703AB4255D123689B
:1044000013F0040F14D0E3685BB1B3F5805F08D0FC
:10441000B3F5A05F05D0B3F5C05F02D0B3F5E05FA0
:1044200031D1244A936823F4E053E1680B4393604D
:10443000236813F0080F15D023695BB1B3F5805FD3
:1044400008D0B3F5A05F05D0B3F5C05F02D0B3F5D7
:10445000E05F1ED1174A936823F46043216943EA61
:10446000C1039360FFF7B0FE124B9B68C3F30313C5
:10447000124AD35CD840124B1860124B1868FDF7F3
:1044800019F9002070BD40F2C3210B48FCF764FF0E
:10449000C7E740F2CA210848FCF75EFFDAE70120CF
:1044A00070470120EEE70120ECE70120EAE700BFBA
:1044B000003C024000380240705F0108B85D01080E
:1044C0000000002008000020014B1868704700BF62
:1044D0000000002008B5FFF7F7FF044B9B68C3F30B
:1044E0008223034AD35CD84008BD00BF0038024095
:1044F000B05D010808B5FFF7E7FF044B9B68C3F305
:104500004233034AD35CD84008BD00BF00380240A4
:10451000B05D01080F2303600B4B9A6802F00302A1
:1045200042609A6802F0F00282609A6802F4E052F7
:10453000C2609B68DB0803F4E0530361034B1B6814
:1045400003F007030B60704700380240003C024054
:10455000E0B110B5044602680D4B9A4203D0A32186
:104560000C48FCF7F9FE63795BB1022363712268A2
:10457000136843F004031360012363710020A060FB
:1045800010BD23712046FCF7F9FEEEE701207047CD
:1045900000080650A85F0108F8B50379012B30D058
:1045A00004460E46012303714579EDB29D4206D0C3
:1045B000042383600125002323712846F8BD0223CC
:1045C0004371FDF7BBFC074623685A6812F0010FE0
:1045D00010D1FDF7B3FCC01B0228F5D923685B6836
:1045E00013F0010FF0D1012363710223A3600023B4
:1045F0002371E2E79B68E360336001236371002568
:10460000D9E70225D9E700002DE9F04782B0054639
:10461000884617461E46FDF791FC0A9B1B1A03EBC2
:104620000609FDF78BFC8246284B1B68C3F3CB338E
:1046300009FB03F301932B689C6838EA04040CBF60
:1046400001230023BB423DD0B6F1FF3FF3D0FDF77D
:1046500075FCA0EB0A00484507D2019A02B14A4610
:10466000019B013B01939146E5E72A68536823F0DB
:10467000E00353606B68B3F5827F0BD0AB6AB3F590
:10468000005F14D0012385F85130002385F85030A5
:10469000032018E0AB68B3F5004F02D0B3F5806F8C
:1046A000ECD12A68136823F040031360E6E72A6818
:1046B000136823F4005313602A68136843F400530B
:1046C0001360DFE7002002B0BDE8F08700000020A3
:1046D00010B584B00446164B1868164BA3FB003087
:1046E000400D4FF47A7303FB00F003906368B3F559
:1046F000827F0BD0039BBBB1039B013B03932368D9
:104700009B6813F0800FF5D100200EE000920B465D
:10471000002280212046FFF777FF30B1636D43F020
:1047200020036365032000E0002004B010BD00BF3B
:1047300000000020819F5E1610B582B004460B4633
:104740004168B1F5827F14D06168B1F5827F2AD1CA
:10475000A168B1F5806F19D0009200228021204617
:10476000FFF752FF30B3636D43F02003636503200E
:1047700020E08168B1F5004F02D0B1F5806FE3D140
:104780002068016821F040010160DDE7009200220D
:1047900001212046FFF738FF60B1636D43F020032D
:1047A0006365032006E00092002201212046FFF706
:1047B0002BFF08B902B010BD636D43F020036365A1
:1047C0000320F7E7002800F0228110B504460368B3
:1047D000904A93420CD0A2F57842934208D002F559
:1047E0008062934204D04FF4A0718B48FCF7B4FD73
:1047F000636813B1B3F5827F43D1A3682BB1B3F5DE
:10480000806F02D0B3F5004F41D1E368B3F5006F7C
:1048100001D0002B41D1A369B3F5007F03D013B1C0
:10482000B3F5802F3FD1E36993B1182B41D9382BD1
:1048300009D8202B07D3203B4FF0013222FA03F393
:1048400013F0010F04D140F245117348FCF784FDC9
:10485000236A0BB1802B35D1636A0BB1102B37D192
:10486000636A002B65D123690BB1022B36D16369D2
:10487000012B39D86368B3F5827F3BD00023E36115
:104880006FE040F241116448FCF766FDB5E74FF474
:10489000A1716148FCF760FDB7E740F243115E4843
:1048A000FCF75AFDB7E74FF4A2715B48FCF754FDE3
:1048B000B9E7082BC7D3594A22FA03F313F0010FC3
:1048C000C1D0C5E74FF4A3715348FCF745FDC3E7DA
:1048D00040F247115048FCF73FFDC1E74FF4A57186
:1048E0004D48FCF739FDC2E740F24B114A48FCF74E
:1048F00033FDBFE7E369A3B3182B11D9382B09D8CF
:10490000202B07D3203B4FF0013222FA03F313F0A0
:10491000010F26D140F24F113F48FCF71DFD20E06A
:10492000082BF7D33D4A22FA03F313F0010FF1D01D
:1049300017E0E36993B1182B5AD9382B09D8202BEB
:1049400007D3203B4FF0013222FA03F313F0010F9B
:1049500004D140F259113048FCF7FEFC00232361DA
:1049600063610023A36294F85130002B49D00223E5
:1049700084F851302268136823F0400313606368A1
:1049800003F48273A26802F404421343E26802F45F
:1049900000621343226902F002021343626902F0CB
:1049A00001021343A26902F400721343E26902F0A8
:1049B00038021343226A02F080021343A26A02F40F
:1049C0000052216813430B60638B03F00403626A97
:1049D00002F01002216813434B602268D36923F46C
:1049E0000063D36100206065012384F8513010BD5D
:1049F000082BAED3094A22FA03F313F0010FA8D013
:104A0000ACE784F850302046FCF718FDAFE70120F2
:104A1000704700BF00300140E05F01080001010164
:104A20002DE9F04383B00446884691461F460A9D0F
:104A30008368002B59D194F85030012B00F013817A
:104A4000012384F85030FDF779FA064694F8513086
:104A5000DBB26268012B0AD0B2F5827F40F0E980B8
:104A6000A268002A40F0EF80042B40F0EE80B8F1FD
:104A7000000F00F0EC80B9F1000F00F0EA80002F89
:104A800000F0E98094F85130DBB2042B02D005230A
:104A900084F8513000236365C4F83890E787A7870E
:104AA000C4F83080E786A7862364636423681A68A5
:104AB00012F0400F03D11A6842F040021A60E36816
:104AC000B3F5006F17D063680BB1012F0BD1226BC8
:104AD000236812781A73236B01332363E38E9BB22E
:104AE000013B9BB2E386012771E040F27C415F48C5
:104AF000FCF732FC9FE763680BB1012F0BD1226BEF
:104B000023681288DA60236B02332363E38E9BB23F
:104B1000013B9BB2E38601271CE023689A6812F0F0
:104B2000010F0ED0E28F92B25AB1DA68A36B1A80ED
:104B3000A36B0233A363E38F9BB2013B9BB2E3877A
:104B40000127FDF7FBF9801BA84203D3B5F1FF3F16
:104B500040F08380E38E9BB21BB9E38F9BB2002BA6
:104B600053D023689A6812F0020FD6D0E28E92B228
:104B7000002AD2D0002FD0D0226B1288DA60236BAB
:104B800002332363E38E9BB2013B9BB2E386002793
:104B9000C3E723689A6812F0010F0ED0E28F92B239
:104BA0005AB1DA68A36B1A70A36B0133A363E38F66
:104BB0009BB2013B9BB2E3870127FDF7BFF9831B43
:104BC000AB4202D3B5F1FF3F49D1002D49D0E38E6E
:104BD0009BB213B9E38F9BB2BBB123689A6812F002
:104BE000020FD6D0E28E92B2002AD2D0002FD0D0BF
:104BF000226B12781A73236B01332363E38E9BB20B
:104C0000013B9BB2E3860027C3E732462946204694
:104C1000FFF75EFD48B9A36863B901932368DA68BA
:104C200001929B680193019B04E0202363650120AE
:104C300000E00220012384F85130002384F8503032
:104C400003B0BDE8F0830220F4E70220F2E7012080
:104C5000F0E70120EEE70120ECE70320EAE703207C
:104C6000E8E70320E6E70220EAE700BFE05F01088B
:104C70002DE9F04383B00446884691461D464068BE
:104C8000B0F5827F38D094F85030012B00F0AE8020
:104C9000012384F85030FDF751F9074694F851602C
:104CA000F6B2012E40F08F80B8F1000F00F08C803A
:104CB000B9F1000F00F08880042384F851300023FC
:104CC0006365C4F83880A4F83C90A4F83E90236350
:104CD000A386E38623646364A368B3F5004F19D009
:104CE00023681A6812F0400F03D11A6842F040029C
:104CF0001A60E3681BB341E0A368002BC3D104230F
:104D000084F85130009513460A462046FFF788FE86
:104D100006465FE02268136823F0400313602268B0
:104D2000136823F480431360DAE7FDF707F9C01B2B
:104D3000A84202D3B5F1FF3F50D1002D50D0E38FF0
:104D40009BB2002B33D023689A6812F0010FECD08D
:104D5000A26B1B7B1370A36B0133A363E38F9BB226
:104D6000013B9BB2E387EAE7FDF7E8F8C01BA842E6
:104D700002D3B5F1FF3F35D1002D35D0E38F9BB283
:104D8000ABB123689A6812F0010FEDD0DA68A36B1B
:104D90001A80A36B0233A363B4F83EC01FFA8CFCE5
:104DA0000CF1FF3C1FFA8CFCA4F83EC0E6E73A4643
:104DB00029462046FFF7C0FC08B120236365636DD8
:104DC00013B9002600E00226012384F851300023A5
:104DD00084F85030304603B0BDE8F0830326F3E793
:104DE0000326F1E70326EFE70326EDE70226F1E7C6
:104DF000F8B504460E4617461D46C36C002B5BD023
:104E0000A36C002B5ED0A368002B61D194F85030C6
:104E1000012B00F0AC80012384F8503094F851301D
:104E2000DBB26268012B0AD0B2F5827F40F090803D
:104E3000A268002A40F09180042B40F09080002E60
:104E400000F08F80002F00F08E80002D00F08D800C
:104E500094F85130DBB2042B02D0052384F8513092
:104E6000002363652663A586E586A763A587E58796
:104E70002364636494F85130DBB2042B2ED0E36CCE
:104E80003C4A1A64E36C3C4ADA63E36C3B4ADA64FA
:104E9000E36C00221A652168E38F9BB2A26B0C3190
:104EA000E06CFDF7EBFA00B3636D43F0100363654C
:104EB000012084F851004CE040F23E713048FCF78C
:104EC0004BFA9DE740F23F712D48FCF745FA9AE70F
:104ED00040F242712A48FCF73FFA97E7E36C294A0F
:104EE0001A64E36C284ADA63CFE72268536843F018
:104EF00001035360A26C00231364A26CD363A26C01
:104F0000D364A26C13652268E38E9BB20C32216BD2
:104F1000A06CFDF7B3FA98B923681A6812F0400F35
:104F200003D11A6842F040021A602268536843F0C5
:104F3000200353602268536843F00203536008E083
:104F4000636D43F010036365012084F8510000E0B5
:104F50000220002384F85030F8BD0220F9E7022037
:104F6000F7E70120F5E70120F3E70120F1E7022050
:104F7000F2E700BF9F4F00083B500008AB4F00080E
:104F8000E05F0108934F0008CD4F0008704770475D
:104F9000704708B5806BFFF7FBFF08BD704708B589
:104FA000806BFFF7FBFF08BD704708B5806B026898
:104FB000536823F003035360436D43F010034365CC
:104FC000012380F85130FFF7EFFF08BD38B50546E3
:104FD000846BFCF7B3FF2B681B6813F4807F1ED132
:104FE000024621684B6823F020034B60A3681BB97D
:104FF0006368B3F5827F16D021684B6823F0010304
:105000004B6064212046FFF797FB08B120236365BE
:105010000023E387012384F85130636D4BB92046A8
:10502000FFF7B4FF38BD21684B6823F003034B60E2
:10503000E7E72046FFF7B8FFF4E738B50546846B8D
:10504000FCF77CFF2B681B6813F4807F1BD10246A2
:1050500021684B6823F020034B6064212046FFF752
:1050600037FB18B1636D43F0200363652268536812
:1050700023F0030353600023E386E387012384F8CE
:105080005130636D1BB92046FFF781FF38BD2046C4
:10509000FFF78AFFFAE7000010B584B00446026803
:1050A0005168936803F04100012867D013F0020FA4
:1050B00002D011F0800F68D113F4B07F68D011F0E6
:1050C000200F65D013F0400F0FD094F85100C0B2FC
:1050D00003285FD0606D40F0040060650020009000
:1050E000D068009090680090009813F0200F0CD0CA
:1050F000606D40F0010060650020029090680290B1
:10510000106820F040001060029A13F4807F09D0EC
:10511000636D43F0080363650023039323689B6872
:105120000393039B636D002B32D02268536823F0F6
:10513000E0035360012384F8513011F0030F31D0A4
:105140002268536823F003035360E36C4BB1174AA2
:105150001A65E06CFDF7DEF918B1636D43F04003AA
:105160006365A36CA3B1114A1A65A06CFDF7D2F96F
:1051700070B1636D43F04003636509E011F0400FC7
:1051800094D0236C2046984702E0636C20469847F1
:1051900004B010BD00230193D36801939368019379
:1051A000019BF5E72046FFF7FFFEF1E7B15100084C
:1051B00008B5806B0023C387C386FFF7F5FE08BDE3
:1051C00090F85100704710B4036A046A24F0010497
:1051D0000462846924F0F00C4CEA021223F00A0302
:1051E0000B43826103625DF8044B704710B4036A9D
:1051F00023F0100303628469036A24F4704C4CEAC0
:10520000023223F0A00343EA0113826103625DF8D6
:10521000044B7047836823F070030B4343F007038C
:105220008360704710B5044603683E4A934237D006
:10523000B3F1804F34D0A2F57C42934230D002F5D6
:10524000806293422CD002F58062934228D002F50E
:105250008062934224D002F58062934220D002F50E
:10526000704293421CD002F57052934218D002F55E
:105270008062934214D002F58062934210D0A2F56E
:10528000983293420CD002F58062934208D002F526
:105290008062934204D040F2CF112348FCF75CF8BF
:1052A00094F83D30DBB2012B37D1022384F83D3036
:1052B0002268D36843F00103D3602368194A9342FC
:1052C00020D0B3F1804F1DD0A2F57C42934219D07B
:1052D00002F58062934215D002F58062934211D0AC
:1052E00002F5784293420DD002F57052934209D0F4
:1052F000A2F59432934205D01A6842F001021A6076
:1053000000200BE09A6802F00702062A07D01A680C
:1053100042F001021A60002000E0012010BD0020D0
:10532000FCE700BF000001401860010870477047AB
:105330007047704710B5044603681A6912F0020FEF
:1053400011D0DA6812F0020F0DD06FF002021A616C
:105350000123037703689B6913F0030F70D0FFF7F5
:10536000E6FF0023237723681A6912F0040F12D096
:10537000DA6812F0040F0ED06FF004021A610223F3
:10538000237723689B6913F4407F5FD02046FFF7A3
:10539000CEFF0023237723681A6912F0080F12D07A
:1053A000DA6812F0080F0ED06FF008021A610423B9
:1053B00023772368DB6913F0030F4ED02046FFF7F5
:1053C000B6FF0023237723681A6912F0100F12D05A
:1053D000DA6812F0100F0ED06FF010021A61082375
:1053E00023772368DB6913F4407F3DD02046FFF725
:1053F0009EFF0023237723681A6912F0010F03D060
:10540000DA6812F0010F36D123681A6912F0800FA2
:1054100003D0DA6812F0800F34D123681A6912F0D1
:10542000400F03D0DA6812F0400F32D123681A69B6
:1054300012F0200F03D0DA6812F0200F30D110BD27
:10544000FFF774FF2046FFF773FF8AE72046FFF758
:105450006DFF2046FFF76CFF9BE72046FFF766FFD6
:105460002046FFF765FFACE72046FFF75FFF2046C9
:10547000FFF75EFFBDE76FF001021A612046FBF700
:10548000E7FEC1E76FF080021A61204600F027FCBA
:10549000C3E76FF040021A612046FFF74AFFC5E7F5
:1054A0006FF020021A61204600F018FCC7E70000E8
:1054B0000368304A904212D0B0F1804F0FD0A2F56D
:1054C0007C4290420BD002F58062904207D002F5F8
:1054D0008062904203D002F57842904203D123F0DB
:1054E00070034A681343234A90422AD0B0F1804F98
:1054F00027D0A2F57C42904223D002F580629042F0
:105500001FD002F5806290421BD002F57842904293
:1055100017D002F57052904213D002F5806290428B
:105520000FD002F5806290420BD0A2F598329042E3
:1055300007D002F58062904203D002F5806290426B
:1055400003D123F44073CA68134323F080034A69EC
:10555000134303608B68C3620B688362054B9842F8
:1055600003D003F58063984201D10B6903630123E3
:105570004361704700000140002800F08E8010B5A4
:1055800004460368464A934237D0B3F1804F34D083
:10559000A2F57C42934230D002F5806293422CD037
:1055A00002F58062934228D002F58062934224D0B3
:1055B00002F58062934220D002F5704293421CD0E3
:1055C00002F57052934218D002F58062934214D0D3
:1055D00002F58062934210D0A2F5983293420CD02B
:1055E00002F58062934208D002F58062934204D0B3
:1055F00040F213112B48FBF7AFFEA3683BB1102B11
:1056000005D0202B03D0402B01D0602B2DD1236956
:105610002BB1B3F5807F02D0B3F5007F2BD1A36906
:105620000BB1802B2DD194F83D3083B3022384F845
:105630003D30214651F8040BFFF73AFF012384F86F
:10564000463084F83E3084F83F3084F8403084F8A7
:10565000413084F8423084F8433084F8443084F890
:10566000453084F83D30002010BD4FF48A710D485C
:10567000FBF772FECBE740F215110A48FBF76CFE10
:10568000CDE74FF48B710748FBF766FECBE784F854
:105690003C302046FCF7D8F9C8E70120704700BF2E
:1056A000000001401860010810B4846824F47F4CA5
:1056B00042EA03220A4342EA0C0282605DF8044B8C
:1056C0007047000038B590F83C30012B00F0748230
:1056D00004460D46012380F83C30022380F83D301B
:1056E0000B68B3F5805F18D0602B16D010D8402B14
:1056F00013D0502B11D083B1102B0ED0202B0CD0F7
:10570000302B0AD041F2B7419648FBF725FE04E062
:10571000702B02D0B3F5005FEDD12268936823F4BB
:105720007F4323F0770393602B68602B00F09A810E
:1057300000F28180402B00F0DC813ED9502B78D1E3
:105740002368894A93421FD0B3F1804F1CD0A2F541
:105750007C42934218D002F58062934214D002F545
:105760008062934210D002F5784293420CD002F549
:105770007052934208D0A2F59432934204D041F281
:10578000F6417848FBF7E8FD6B68B3F5004F05D0AC
:1057900023B1022B02D00A2B40F05881EB680F2B6B
:1057A00000F25A81EA6869682068FFF70CFD502111
:1057B0002068FFF72FFD002005E0202B0DD009D930
:1057C000302B0AD00120012384F83D30002384F8D7
:1057D0003C3038BD0BB1102B29D12368624A93426B
:1057E0001FD0B3F1804F1CD0A2F57C42934218D059
:1057F00002F58062934214D002F58062934210D089
:1058000002F5784293420CD002F57052934208D0D0
:10581000A2F59432934204D041F229515148FBF74A
:105820009BFD29682068FFF7F5FC0020CBE70120ED
:10583000C9E70120C7E7B3F5805F00F09780B3F5B3
:10584000005F42D12368484A934217D0B3F1804F9A
:1058500014D0A2F57C42934210D002F580629342AC
:105860000CD002F58062934208D002F57842934250
:1058700004D041F2E2413B48FBF76EFDAB684BB10F
:10588000B3F5805F06D0B3F5005F03D0B3F5405F9A
:1058900040F0CA806B68B3F5004F05D023B1022BEE
:1058A00002D00A2B40F0C680EB680F2B00F2C880B4
:1058B000EB686A68A9682068FFF7F6FE22689368BB
:1058C00043F48043936000207DE7702B47D1236829
:1058D000254A93421FD0B3F1804F1CD0A2F57C42E1
:1058E000934218D002F58062934214D002F5806290
:1058F000934210D002F5784293420CD002F57052D8
:10590000934208D0A2F59432934204D041F2CA41A6
:105910001448FBF721FDAB6843B1B3F5805F05D0B8
:10592000B3F5005F02D0B3F5405F6BD16B68B3F5A0
:10593000004F04D01BB1022B01D00A2B68D1EB68B9
:105940000F2B6BD8EB686A68A9682068FFF7ACFE7C
:105950002268936843F077039360002033E70120C7
:1059600031E700BF18600108000001402368934A36
:10597000934200F00581B3F1804F00F00381A2F55E
:105980007C42934200F0008102F58062934200F075
:10599000FD8002F58062934200F0FA8002F5806299
:1059A000934200F0F78002F58062934200F0F480A9
:1059B00002F57042934200F0F18002F5705293427A
:1059C00000F0EE8002F58062934200F0EB8002F579
:1059D0008062934200F0E880A2F59832934200F092
:1059E000E58002F58062934200F0E28002F5806279
:1059F000934200F0DF8041F2C3417148FBF7ACFCF9
:105A00000020E0E641F2CD416D48FBF7A5FC8DE7B3
:105A100041F2CE416A48FBF79FFC90E741F2CF414B
:105A20006748FBF799FC8DE741F2E5416448FBF7D5
:105A300093FC2FE741F2E6416148FBF78DFC33E729
:105A400041F2E7415E48FBF787FC31E741F2F9415B
:105A50005B48FBF781FCA1E641F2FA415848FBF7AD
:105A60007BFC9FE62368554A93421FD0B3F1804FD9
:105A70001CD0A2F57C42934218D002F5806293427A
:105A800014D002F58062934210D002F5784293421E
:105A90000CD002F57052934208D0A2F59432934292
:105AA00004D041F206514648FBF756FC6B68B3F54B
:105AB000004F04D01BB1022B01D00A2B0DD1EB6893
:105AC0000F2B10D8EA6869682068FFF78FFB602108
:105AD0002068FFF79FFB002075E641F20951384826
:105AE000FBF73AFCEBE741F20A513548FBF734FC8F
:105AF000E8E72368314A93421FD0B3F1804F1CD0AE
:105B0000A2F57C42934218D002F58062934214D0F1
:105B100002F58062934210D002F5784293420CD095
:105B200002F57052934208D0A2F59432934204D009
:105B300041F216512248FBF70FFC6B68B3F5004F9A
:105B400004D01BB1022B01D00A2B0DD1EB680F2B17
:105B500010D8EA6869682068FFF735FB40212068A3
:105B6000FFF758FB00202EE641F219511448FBF7CD
:105B7000F3FBEBE741F21A511148FBF7EDFBE8E7C5
:105B8000002020E600201EE600201CE600201AE689
:105B9000002018E6002016E6002014E6002012E699
:105BA000002010E600200EE600200CE600200AE6A9
:105BB000002008E6002006E602200AE60000014078
:105BC0001860010838B504460D460368414A9342FF
:105BD0001FD0B3F1804F1CD0A2F57C42934218D065
:105BE00002F58062934214D002F58062934210D095
:105BF00002F5806293420CD002F58062934208D095
:105C000002F57042934204D040F2B1713248FBF782
:105C1000A3FB2B68A3B1402B12D00BD8202B0FD0A5
:105C2000302B0DD0102B0BD040F2B2712A48FBF76D
:105C300093FB05E0602B03D0702B01D0502BF3D1E8
:105C40006B68802B01D0002B3CD194F83C30012BA9
:105C50003ED0012384F83C30022384F83D30236891
:105C60005968986821F070012A680A435A602368CD
:105C7000184A93421AD0B3F1804F17D0A2F57C4254
:105C8000934213D002F5806293420FD002F58062F6
:105C900093420BD002F57842934207D002F570523E
:105CA000934203D0A2F59432934204D120F08000B5
:105CB0006A6802439A60012384F83D30002084F82A
:105CC0003C0038BD40F2B3710348FBF745FBBCE72D
:105CD0000220F6E70000014050600108704770475D
:105CE00010B504464268574B9A423FD8E36813B157
:105CF000B3F5005F40D123692BB1B3F5806F02D0BB
:105D0000B3F5C06F3ED163694FF6F372134200D111
:105D100023B940F664614C48FBF71EFB2268136907
:105D200023F44053E1680B431361A36822691A43CB
:105D300063691A43E3691A432168CB6823F4164365
:105D400023F00C031343CB602268536923F44073A0
:105D5000A1690B43536123683C4A934218D002F572
:105D60008062934214D0FEF7B5FB13E040F6616108
:105D70003548FBF7F1FAB9E740F662613248FBF7C4
:105D8000EBFAB8E740F663612F48FBF7E5FABAE7AC
:105D9000FEF7B0FBE369B3F5004F29D000210318EB
:105DA00049411B1841F10001C90041EA5371DB0070
:105DB000181863684FEA83024FEA937341F10001B8
:105DC000FAF762FF224AA2FB00314909642303FB70
:105DD00011031B013233A2FB03235B0903F0F00222
:105DE00002EB011203F00F03216813448B6010BD16
:105DF0000023021843EB0301121841F10001C9000E
:105E000041EA5271D200101841F100016268921803
:105E10005B41FAF739FF0E4AA2FB003149096423BE
:105E200003FB1103DB003233A2FB03235B095A009F
:105E300002F4F87202EB011203F007032168134425
:105E40008B60D4E7A037A0008C60010800100140EF
:105E50001F85EB512DE9F84305460F461646994636
:105E6000DDF820802B681C6837EA04040CBF01248D
:105E70000024B4422DD1B8F1FF3FF3D0B8F1000FA8
:105E800005D0FCF75BF8A0EB09004045EAD92A6889
:105E900002F10C0353E8003F23F4D0730C3242E8C4
:105EA00000310029F3D12A6802F1140353E8003FBE
:105EB00023F00103143242E800310029F3D12023FA
:105EC00085F83D3085F83E30002385F83C300320CE
:105ED00000E00020BDE8F883002800F08B8010B5BA
:105EE00004468369002B55D00368434A934210D07F
:105EF000A2F54C4293420CD002F58062934208D046
:105F000002F54C42934204D040F273113B48FBF738
:105F100023FAA36943B1B3F5807F05D0B3F5007FC1
:105F200002D0B3F5407F2FD1A36813B1B3F5805FE2
:105F30004ED1E36913B1B3F5004F4FD194F83D3022
:105F4000002B51D0242384F83D302268D36823F4F9
:105F50000053D3602046FFF7C3FE2268136923F481
:105F6000904313612268536923F02A035361226826
:105F7000D36843F40053D36000202064202384F8C6
:105F80003D3084F83E3010BD4FF4BA711B48FBF72A
:105F9000E3F9C9E70368184A9342C5D0A2F54C4219
:105FA0009342C1D002F580629342BDD002F5806277
:105FB0009342B9D002F580629342B5D002F54442D3
:105FC0009342B1D04FF4BC710C48FBF7C5F9ABE775
:105FD0004FF4BD710948FBF7BFF9AAE740F27B1106
:105FE0000648FBF7B9F9A9E784F83C302046FBF7EF
:105FF000ABFDA7E701207047001001408C6001084D
:106000002DE9F04182B01E4690F83D30DBB2202BE6
:1060100054D104460D469046002953D0002A53D04F
:1060200090F83C30012B51D0012380F83C30002304
:106030000364212380F83D30FBF780FF0746A4F876
:106040002480A4F82680A368B3F5805F05D04FF0C4
:106050000008002384F83C3012E0236913B14FF0AC
:106060000008F6E7A8460025F3E738F8023B226867
:10607000C3F308035360E28C92B2013A92B2E28415
:10608000E38C9BB273B100963B46002280212046F0
:10609000FFF7E0FEE0B9002DE7D015F8012B2368EB
:1060A0005A60E8E700963B46002240212046FFF771
:1060B000D1FE78B9202384F83D3000E0022002B000
:1060C000BDE8F0810120FAE70120F8E70220F6E7B9
:1060D0000320F4E70320F2E70020704730B58DB0CD
:1060E0000C4630252A46002168460CF00FFB2A4654
:1060F000002168460CF00AFB2246002303E01168E9
:10610000F1B10133126822B3032B3BD8516803EB82
:10611000430C0CA800EB8C0C4CF8301C51894CF84B
:106120002C1C002BEBD003F1FF3C03EB43010DEBE8
:1061300081010CEB4C0C00EB8C0C4CF8281CDEE7BE
:1061400003EB43010CA800EB8101002041F8280C6F
:10615000D7E723890D4D6B60C5F808D06C632046E6
:1061600005F020F829460A48FCF7C5FE20B108488A
:10617000FCF77BFF002007E00A21064B186800F0BF
:1061800031FCF4E76FF00B000DB030BDAC0900201E
:10619000E4090020940A00202DE9F043A3B004464E
:1061A0006422002109A80CF0B1FA634D634B2B6007
:1061B00000268DF81C6080238DF81D30E1238DF8BA
:1061C0001E308DF81F608DF820604FF001088DF8AB
:1061D000218007AB6B604FF40003AB60584BEB6062
:1061E000584B2B614FF4C0636B61574B1A788DF895
:1061F0001C205A788DF81D209A788DF81E20DA78A8
:106200008DF81F201A798DF820205B798DF82130C8
:106210002846FCF765FD0746DFF8489138223146ED
:1062200048460CF073FA2123C9F800304FF44003BC
:10623000C9F81430454804F009FA062384F83C30C4
:106240006B681A7884F836205A7884F837209A7860
:1062500084F83820DA7884F839201A7984F83A20DA
:106260005B7984F83B3040F2DC53A38694F83D30F0
:1062700043F00A0384F83D3003223146404600F0E3
:1062800045FE334B186003223146404600F03EFE87
:10629000304B1860EC46304D0FCDACE80F0095E860
:1062A00007008CE807002146684600F06FFA2B4D86
:1062B0002B492846FBF734FD2846FBF750FDAFBBC2
:1062C0002846FBF7B4FD40451EDD042827D00528ED
:1062D00029D003281FD04FF480464FF40067164D95
:1062E00009A92846FCF7C6FF0F970E9609A928466C
:1062F000FDF739F82846FCF753FD204604F04AFC28
:10630000204604F0A7FC13E0204604F0D7FC20460A
:1063100004F06CFC0CE04FF480460027DFE7002619
:106320004FF40067DBE700263746D8E7FAF79CFF13
:1063300023B0BDE8F08300BFE409002000800240E4
:106340009C0A00203C0B0020C01401202C61010895
:10635000980A0020940A0020FC5C01088C090020A7
:106360000C000020AC09002000B583B0002301938D
:10637000054B1B781BB1019803B05DF804FB01A924
:106380000248FCF7F3FDF6E7DC0B0020E4090020EF
:1063900038B505464FF0FF310B4B186800F022FB73
:1063A0000028F7D101E0002CF4D02846FFF7DCFFED
:1063B00004460028F7D02B69294698470028F2D0D8
:1063C000204604F07DFDEEE7980A002008B501465E
:1063D000074804F08FF9074B1B78012B00D008BD4C
:1063E000044B00221A70044B186800F02AFBF6E7F1
:1063F0002C610108DC0B0020980A002008B5FBF78F
:106400009DFD08BD08B50248FCF7BCFF002008BD93
:10641000E409002008B513460A4601460348FCF784
:10642000DBFE00B908BD4FF0FF30FBE7E4090020B8
:1064300008B513460A4601460348FCF7F5FE00B9C5
:1064400008BD4FF0FF30FBE7E409002008B5024B20
:10645000186800F0F6FA08BD980A002008B5024B4B
:10646000186800F0EEFA08BD940A002008B5FCF7A1
:10647000C3FF10F0800F00D108BD024B186800F078
:10648000E0FAF9E7980A002010B5044680B10C4BF9
:106490002363732384F83E30742384F83F30094B20
:1064A0006361094BA3612046FFF776FE002010BD13
:1064B000064B4FF4F572064906480CF07DF8E6E706
:1064C0001C61010821DE0008DD600008C8600108C9
:1064D000E4600108F460010808B5FBF72FFD08BD72
:1064E0002DE9F0418CB000230793089309930A9398
:1064F0000B9302683F4B9A4202D00CB0BDE8F0818A
:1065000000240194A3F590431A6B42F000721A63C1
:106510001A6B02F000720192019A02941A6B42F017
:1065200080621A631A6B02F080620292029A0394EC
:106530001A6B42F000621A631A6B02F00062039257
:10654000039A04941A6B42F004021A631A6B02F065
:1065500004020492049A05941A6B42F001021A6331
:106560001A6B02F001020592059A06941A6B42F02A
:1065700002021A631B6B03F002030693069B4FF0A3
:106580003208CDF81C800227089703260A960B25AF
:106590000B9507A91848FDF7A9F9862307930897D3
:1065A00009940A960B9507A91448FDF79FF94FF433
:1065B00060530793089709940A960B9507A910480A
:1065C000FDF794F9224605213D20FBF735FD3D20DE
:1065D000FBF756FD0B4D224608212846FDF7FAFA37
:1065E0004046FBF7B1FC012208212846FDF7F2FAEC
:1065F00083E700BF00800240000802400000024024
:1066000000040240000C02402DE9F0419AB004461B
:106610006422002101A80CF079F8236A20469847EB
:106620000026374635460BE02648FCF715FC204689
:1066300004F0DCFA204604F041FB642000F0D9F8B5
:106640002148FBF7F4FB94F83D3013F0040F01D020
:106650000128E9DD13F0040FEFD10128EDDD023848
:10666000032816D8DFE800F01002070C00264FF4CC
:10667000804701250DE04FF400660027012508E062
:1066800000263746012504E04FF400664FF48047AA
:106690000125002DD1D0DFF82C8001A94046FCF760
:1066A000E9FD0796069701A94046FCF75CFE4046C7
:1066B000FCF776FB204604F06DFA204604F0CAFA97
:1066C000BBE700BFE40900208C09002010B582B0B0
:1066D00004460E4803F0DEFF88B1034600F12002B5
:1066E00022600B4A02614FF4C0620192226800925C
:1066F00041220021084604F07DFB02B010BD054B8D
:1067000001221A7000232360F7E700BF2C61010803
:10671000CD630008DC0B002030B4A2F1200400257A
:1067200042F8205C22F8185C22F8163C026822B17C
:106730000A6814600C60026805E00460FAE71189D9
:10674000194411811268002AF9D130BC704708B58C
:1067500004F0B6FB08BD842801D003307047002048
:106760007047EFF30580003818BF0120704708B567
:1067700001F052FA002008BD08B5FFF7F2FF10B192
:1067800001F09AFA08BD01F091FAFBE72DE9F04318
:1067900087B00E464469C4B18569B5B14768D0F881
:1067A0000080D0F81090B0F90800FFF7D4FF0295F0
:1067B0000194009033464A464146384601F0BEF9FE
:1067C0000590059807B0BDE8F0834468056807693F
:1067D000B0F90800FFF7BFFF05AB01930090334607
:1067E000BAB22946204601F0E4F90128E9D0002098
:1067F000E8E708B500B9012001F06EFB002008BDF4
:1068000030B585B004460D46002303930293FFF78D
:10681000A8FFB0B103AB009302AB0122294620468A
:1068200001F086FE012817D1039B93B14FF0E023BE
:106830004FF08052C3F8042DBFF34F8FBFF36F8F1B
:1068400007E002AB01222946204601F0EDFD0128B8
:1068500005D1029805B030BD4FF00040FAE74FF087
:106860000040F7E770B584B004460E461546002395
:106870000293FFF776FF48B18223019304AB13E93B
:10688000070084E80700204604B070BD2B4602AA2A
:106890003146002001F076FD012806D015B900230D
:1068A0000193EBE740230193E8E7029B002B02DB17
:1068B00008230193E2E786230193DFE708B54168E7
:1068C00019B1012000F062FC08BD012000F053FC6A
:1068D000FAE730B583B00023019310B30C460546A8
:1068E000FFF73FFFA0B101AA0021284600F0DFFE1C
:1068F000012818D1019BC3B14FF0E0234FF0805223
:10690000C3F8042DBFF34F8FBFF36F8F002006E055
:106910002146284600F0D8FD012808D1002003B008
:1069200030BD8020FBE7FF20F9E70020F7E7FF20DC
:10693000F5E710B582B0044600230193FFF711FF7D
:1069400098B101A9204600F0B7FC01281AD1019B9B
:10695000D3B14FF0E0234FF08052C3F8042DBFF3C2
:106960004F8FBFF36F8F002008E000231A461946AF
:10697000204600F030FB012802D0FF2002B010BDFD
:106980000020FBE7FF20F9E70020F7E710B582B011
:10699000426892B1012906D0084600F0DBFA0446AD
:1069A000204602B010BD0323009313460022114677
:1069B000012000F061FA0446F2E7012904D00846FC
:1069C00000F0EBFA0446EBE703220021012000F07F
:1069D0009DFA04460028E3D000231A46194600F029
:1069E000FAFADDE770B582B00023019318B30C46C4
:1069F0000646FFF7B6FE0546A0B101AA00213046C3
:106A000000F055FE012818D1019D8DB14FF0E02313
:106A10004FF08052C3F8042DBFF34F8FBFF36F8F39
:106A2000002505E02146304600F04EFD012806D144
:106A3000284602B070BD8025FAE7FF25F8E7FF255C
:106A4000F6E710B582B0044600230193FFF789FEF4
:106A500098B101A9204600F02FFC01281AD1019B12
:106A6000D3B14FF0E0234FF08052C3F8042DBFF3B1
:106A70004F8FBFF36F8F002008E000231A4619469E
:106A8000204600F0A8FA012802D0FF2002B010BD75
:106A90000020FBE7FF20F9E70020F7E710B50446E8
:106AA000FFF75FFE20B9204600F08EFE002010BDEB
:106AB0008220FCE700B583B0826842B1C36833B17D
:106AC000002100914168006800F0D6F904E000223E
:106AD0004168006800F01AFA03B05DF804FB30B5B5
:106AE00085B00446019100230393154602B90125A0
:106AF000FFF737FEA8B1002303AA01A9204600F042
:106B000074FB012818D1039BC3B14FF0E0234FF071
:106B10008052C3F8042DBFF34F8FBFF36F8F002057
:106B200008E000232A4601A9204600F054FA012873
:106B300006D1002005B030BDFF20FBE70020F9E7BB
:106B4000FF20F7E770B584B004460291002301935B
:106B5000E1B10D46164600230393FFF702FE00B392
:106B600003AA01A9284600F0A2FD012816D000239F
:106B70000093039BFBB14FF0E0234FF08052C3F82A
:106B8000042DBFF34F8FBFF36F8F14E0802300936A
:106B90006B4693E8070084E8070011E01023009398
:106BA000E7E7324601A9284600F0DFFB01280AD0BA
:106BB00006B1402600966B4693E8070084E807007C
:106BC000204604B070BD10230093F4E710B50446CE
:106BD000FFF7C7FD18B1204600F0D3FD10BD2046D9
:106BE00000F0BCFDFAE710B50446FFF7BAFD20B986
:106BF000204600F0E9FD002010BD8220FCE700F1F6
:106C0000080343604FF0FF328260C36003610023DA
:106C10000360704700230361704743684B609A68C4
:106C20008A605160996008610368013303607047AE
:106C300030B40D68B5F1FF3F11D000F108031C46D8
:106C40005B681A68AA42FAD963684B6099608C60E5
:106C50006160086103680133036030BC70470469F8
:106C6000F2E70369416882688A60416851605A6846
:106C7000824206D0002202611A68013A1A6018683E
:106C8000704782685A60F5E70346406A18B11B6B8B
:106C90001868C0F10700704710B5044601F04AFDBE
:106CA000A26BE36B9A4204D0002401F065FD2046FC
:106CB00010BD0124F9E710B5044601F03BFDA36BBC
:106CC00023B9012401F058FD204610BD0024F9E746
:106CD00070B504461546866B026C5AB903681BB141
:106CE00000200136A66370BD806801F08BFA002396
:106CF000A360F6E76DB940680BF0FCFD6368226C99
:106D000013446360A268934219D3236863602846E2
:106D1000E7E7C0680BF0EEFDE368226C51429B1A76
:106D2000E3602268934202D2A3680B44E360022D21
:106D300001D00020D5E726B1013E0020D1E728464A
:106D4000CFE70020CDE70346026C6AB110B50846D4
:106D5000D9681144D9609C68A14201D31968D960EF
:106D6000D9680BF0C7FD10BD704738B5054601F076
:106D7000E1FC95F8454064B201E0013C64B2002CAE
:106D80000ADD6B6A43B105F1240001F035F90028F2
:106D9000F3D001F0C5F9F0E7FF2385F8453001F0A5
:106DA000EBFC01F0C7FC95F8444064B201E0013C03
:106DB00064B2002C0ADD2B6943B105F1100001F02B
:106DC0001BF90028F3D001F0ABF9F0E7FF2385F8B9
:106DD000443001F0D1FC38BD38B5E0B10D46044671
:106DE00001F0A8FC2368E26B216C01FB0230A0607B
:106DF0000020A0636360013A02FB0133E360FF23DC
:106E000084F8443084F84530FDB9236963B901F052
:106E1000B3FC012038BD4FF0500383F31188BFF35A
:106E20006F8FBFF34F8FFEE704F1100001F0E4F81D
:106E30000028ECD04FF0E0234FF08052C3F8042D2F
:106E4000BFF34F8FBFF36F8FE1E704F11000FFF73F
:106E5000D6FE04F12400FFF7D2FED8E710B50346B2
:106E600002980C4631B90060C36304640121FFF746
:106E7000B3FF10BD0260F7E740B94FF0500383F352
:106E80001188BFF36F8FBFF34F8FFEE710B584B04B
:106E90001C46844653B192B189B94FF0500383F335
:106EA0001188BFF36F8FBFF34F8FFEE74FF0500392
:106EB00083F31188BFF36F8FBFF34F8FFEE76AB183
:106EC00048230393039B482B13D04FF0500383F3C5
:106ED0001188BFF36F8FBFF34F8FFEE70029EFD00C
:106EE0004FF0500383F31188BFF36F8FBFF34F8FC1
:106EF000FEE7039B012384F8463000949DF8183088
:106F00006046FFF7ABFF204604B010BD40B94FF01C
:106F1000500383F31188BFF36F8FBFF34F8FFEE7EA
:106F2000F0B583B00D461446064601FB00F048302C
:106F300001F0BAFD074650B1002380F846300090BA
:106F4000234600F1480229463046FFF787FF3846BE
:106F500003B0F0BD40B94FF0500383F31188BFF385
:106F60006F8FBFF34F8FFEE710B582B00C4688429B
:106F700008D24FF0500383F31188BFF36F8FBFF334
:106F80004F8FFEE702230093134600221146FFF7BE
:106F900073FF00B1846302B010BD40B94FF05003DD
:106FA00083F31188BFF36F8FBFF34F8FFEE710B5E8
:106FB0000C46884208D24FF0500383F31188BFF388
:106FC0006F8FBFF34F8FFEE702220021FFF79EFF76
:106FD00000B1846310BDF0B585B0019288B10F4651
:106FE0001D460446B1B1022D20D1E36B012B1DD00B
:106FF0004FF0500383F31188BFF36F8FBFF34F8FB0
:10700000FEE74FF0500383F31188BFF36F8FBFF398
:107010004F8FFEE7036C002BE5D04FF0500383F356
:107020001188BFF36F8FBFF34F8FFEE701F084F835
:10703000064658B9019B002B48D04FF0500383F30C
:107040001188BFF36F8FBFF34F8FFEE700263DE03F
:107050002A4639462046FFF73BFE636A7BB948B1B2
:107060004FF0E0234FF08052C3F8042DBFF34F8F51
:10707000BFF36F8F01F080FB012005B0F0BD04F17C
:10708000240000F0B9FF0028F4D04FF0E0234FF0C7
:107090008052C3F8042DBFF34F8FBFF36F8FE9E722
:1070A00001F06AFB0020E8E702A800F0EBFF0126F0
:1070B00019E0002384F8443021E0002384F84530AF
:1070C00023E02046FFF751FE00F08AFE01F032FB7C
:1070D000A26BE36B9A42BBD3022DB9D0019B002B6C
:1070E000DED0002EE0D001F047FB00F0D7FD01F02C
:1070F00021FB94F8442052B2B2F1FF3FD9D094F86A
:10710000452052B2B2F1FF3FD7D001F035FB01A9C3
:1071100002A800F0C3FFD8B92046FFF7BDFD002844
:10712000CFD0019904F1100000F04EFF2046FFF788
:107130001CFE00F055FE0028C8D14FF0E0234FF0B0
:107140008052C3F8042DBFF34F8FBFF36F8FBDE79D
:107150002046FFF70AFE00F043FE00208DE748B10D
:1071600008B5002181600160C1600B460A46FFF747
:1071700032FF08BD704710B5024600210120FFF71D
:10718000C5FE0446FFF7EBFF204610BD10B582B0E8
:107190000B460090002211460120FFF76DFE0446C9
:1071A000FFF7DDFF204602B010BD38B538B1044608
:1071B000856800F0BBFF85420AD0002038BD4FF043
:1071C000500383F31188BFF36F8FBFF34F8FFEE738
:1071D000E368013BE3600BB10120EFE71A46194673
:1071E0002046FFF7F8FE0120E8E72DE9F84390B1CB
:1071F0000F4616461C460546B1B1022C20D1EB6B5A
:10720000012B1DD04FF0500383F31188BFF36F8F14
:10721000BFF34F8FFEE74FF0500383F31188BFF3A6
:107220006F8FBFF34F8FFEE7036C002BE5D04FF05D
:10723000500383F31188BFF36F8FBFF34F8FFEE7C7
:1072400001F09EFBEFF311884FF0500383F3118898
:10725000BFF36F8FBFF34F8FAA6BEB6B9A4206D3CE
:10726000022C04D0002088F31188BDE8F88395F83B
:1072700045904FFA89F9AB6B224639462846FFF70D
:1072800027FDB9F1FF3F06D009F101035BB285F894
:1072900045300120E7E76B6A0BB90120E3E705F110
:1072A000240000F0A9FE18B126B101203060DAE711
:1072B0000120D8E70120D6E768B170B50C46054635
:1072C000036C8BB14FF0500383F31188BFF36F8FC2
:1072D000BFF34F8FFEE74FF0500383F31188BFF3E6
:1072E0006F8FBFF34F8FFEE70368EBB101F048FBF0
:1072F000EFF311864FF0500383F31188BFF36F8FC4
:10730000BFF34F8FAA6BEB6B934226D995F84530AC
:107310005BB20132AA63B3F1FF3F11D001335BB21C
:1073200085F84530012019E08368002BDED04FF04E
:10733000500383F31188BFF36F8FBFF34F8FFEE7C6
:107340006B6A0BB9012009E005F1240000F054FE3E
:1073500038B144B10120206000E0002086F311889C
:1073600070BD0120FAE70120F8E7F0B585B0019281
:1073700090B10F460446C1B100F0DEFE064600BBE8
:10738000019B002B5ED04FF0500383F31188BFF3B5
:107390006F8FBFF34F8FFEE74FF0500383F31188D9
:1073A000BFF36F8FBFF34F8FFEE7036C002BE3D06B
:1073B0004FF0500383F31188BFF36F8FBFF34F8FEC
:1073C000FEE700263EE039462046FFF7BCFC013DC3
:1073D000A563236923B901F0CFF9012005B0F0BD01
:1073E00004F1100000F008FE0028F4D04FF0E02374
:1073F0004FF08052C3F8042DBFF34F8FBFF36F8F50
:10740000E9E701F0B9F90020E8E702A800F03AFE48
:10741000012621E0002384F8443029E0002384F889
:1074200045302BE02046FFF7A0FC00F0D9FC09E036
:107430002046FFF79AFC00F0D3FC2046FFF73BFC08
:1074400000283FD101F076F9A56B002DBBD1019B3F
:10745000002BD6D0002ED8D001F08EF900F01EFC03
:1074600001F068F994F844305BB2B3F1FF3FD1D03A
:1074700094F845305BB2B3F1FF3FCFD001F07CF917
:1074800001A902A800F00AFE0028D1D12046FFF78A
:1074900012FC0028C6D0019904F1240000F094FDEC
:1074A0002046FFF762FC00F09BFC0028CAD14FF099
:1074B000E0234FF08052C3F8042DBFF34F8FBFF38A
:1074C0006F8FBFE7002089E770B584B0019158B194
:1074D0000446036C8BB14FF0500383F31188BFF364
:1074E0006F8FBFF34F8FFEE74FF0500383F3118888
:1074F000BFF36F8FBFF34F8FFEE700F01DFE054611
:1075000050B9019B5BB14FF0500383F31188BFF377
:107510006F8FBFF34F8FFEE70026354655E00646D6
:1075200053E0013BA36323683BB123694BB901F0EE
:1075300023F90126304604B070BD00F015FFA060AD
:10754000F3E704F1100000F057FD0028EFD04FF0F2
:10755000E0234FF08052C3F8042DBFF34F8FBFF3E9
:107560006F8FE4E746B14FF0500383F31188BFF308
:107570006F8FBFF34F8FFEE701F0FEF8DAE702A846
:1075800000F080FD01252AE0002384F8443032E039
:10759000002384F8453034E001F0CCF8A06800F016
:1075A000DBFD064601F0E8F83BE02046FFF7DDFB97
:1075B00000F016FC09E02046FFF7D7FB00F010FCB6
:1075C0002046FFF778FB002842D101F0B3F8A36B07
:1075D000002BA6D1019B002BC4D0002DCFD001F0F1
:1075E000CBF800F05BFB01F0A5F894F844305BB2F7
:1075F000B3F1FF3FC8D094F845305BB2B3F1FF3F21
:10760000C6D001F0B9F801A902A800F047FD002892
:10761000D1D12046FFF74FFB0028C6D02368002BAE
:10762000BAD0019904F1240000F0CEFC2046FFF707
:107630009CFB00F0D5FB0028C7D14FF0E0234FF0B2
:107640008052C3F8042DBFF34F8FBFF36F8FBCE799
:107650000EB900266EE701F06DF82046FFF714FB27
:107660000146A06800F026FE01F086F8F1E780B13F
:1076700070B50C460546866800F058FD864211D06C
:1076800021462846FFF720FF80B1EB680133EB600D
:107690000CE04FF0500383F31188BFF36F8FBFF3FB
:1076A0004F8FFEE7EB680133EB60012070BD2DE9E1
:1076B000F843B0B10D4690460446D9B101F060F9E7
:1076C000EFF311874FF0500383F31188BFF36F8FEF
:1076D000BFF34F8FA66BCEB9002087F31188BDE8AA
:1076E000F8834FF0500383F31188BFF36F8FBFF31C
:1076F0004F8FFEE7036C002BE0D04FF0500383F375
:107700001188BFF36F8FBFF34F8FFEE794F844905B
:107710004FFA89F929462046FFF715FB731EA3632C
:10772000B9F1FF3F06D009F101035BB284F84430A0
:107730000120D2E723690BB90120CEE704F1100044
:1077400000F05AFC30B1B8F1000F05D00120C8F8A4
:107750000000C2E70120C0E70120BEE740B110B53C
:10776000044600F0E7FFA46B01F006F8204610BDC8
:107770004FF0500383F31188BFF36F8FBFF34F8F28
:10778000FEE708B1806B70474FF0500383F3118818
:10779000BFF36F8FBFF34F8FFEE700000023072B6F
:1077A0000FD8084A02EBC3025268824201D001336B
:1077B000F5E7044A002142F8331002EBC30251609E
:1077C000704770476855002038B110B50446FFF780
:1077D000E5FF94F846304BB110BD4FF0500383F3F2
:1077E0001188BFF36F8FBFF34F8FFEE7204601F084
:1077F000DDF9F1E7084B1B681B6823B9074B4FF015
:10780000FF321A607047044B1B68DB68DB685A68FC
:10781000024B1A60704700BF18560020B055002078
:107820002DE9F04707469846089DDDF824900A9C0C
:10783000266B02F18042013A06EB820626F007062B
:107840006664002945D008464FF0000CBCF10F0FCC
:1078500009D810F80C2004EB0C0383F8342012B183
:107860000CF1010CF2E7002384F84330062D00D917
:107870000625E562A5644FF0000AC4F84CA0201D5F
:10788000FFF7C8F904F11800FFF7C4F92461C5F146
:107890000705A5616462C4F89CA084F8A0A04C22EE
:1078A000514604F150000AF031FF0C4B636503F1BF
:1078B0006802A265D033E36542463946304600F09F
:1078C00011FF2060B9F1000F01D0C9F80040BDE8F8
:1078D000F087002384F83430C8E700BFF418012093
:1078E00038B5002407E004EB840293000E481844E6
:1078F000FFF785F90134062CF5D90C4D2846FFF722
:107900007EF90B4C2046FFF77AF90A48FFF777F922
:107910000948FFF774F90948FFF771F9084B1D6032
:10792000084B1C6038BD00BF445600203056002074
:107930001C56002000560020EC550020D455002095
:10794000185600201456002010B5044600F0F2FE30
:10795000214A136801331360204B1B685BB1204B35
:107960001B686BB91D4B1B68DA6AE36A9A4207D839
:107970001A4B1C6004E0194B1C601368012B28D0C3
:10798000184A136801331360E06A01238340164AE2
:1079900011680B43136000EB8000211D134B03EBB8
:1079A0008000FFF73AF900F0E7FE0D4B1B687BB152
:1079B0000A4B1B68DA6AE36A9A4209D24FF0E02365
:1079C0004FF08052C3F8042DBFF34F8FBFF36F8F7A
:1079D00010BDFFF785FFD3E7D0550020D05600201B
:1079E000C4550020B4550020C8550020445600203E
:1079F00010B5044650300AF0B7FE94F8A13063B1D8
:107A0000012B11D0022B0ED04FF0500383F31188BD
:107A1000BFF36F8FBFF34F8FFEE7206B01F0C6F807
:107A2000204601F0C3F810BD204601F0BFF8FAE788
:107A30000F4B1B68D3B110B500F07CFE0D4BDB681B
:107A4000DC68201DFFF70DF90B4A1368013B13603A
:107A5000074A1368013B136000F08EFE2046FFF7D3
:107A6000C7FF034B1B68002BE6D110BD704700BF5A
:107A7000E8550020EC550020D055002008B5FFF750
:107A8000D7FF074B1B68012BF9D94FF0E0234FF0CC
:107A90008052C3F8042DBFF34F8FBFF36F8FEEE713
:107AA0004456002070B504460D461D4B1E681D4B04
:107AB00018680430FFF7D5F848B91A4B1B68DB6A21
:107AC00001229A4018490B6823EA02030B60B4F1C3
:107AD000FF3F0DD03444134B1B685C60A64210D9A5
:107AE000124B18680F4B19680431FFF7A1F870BDED
:107AF000002DEFD00B4B196804310D48FFF78DF8BE
:107B0000F5E70C4B1868074B19680431FFF790F83C
:107B1000094B1B68A342EAD9074B1C60E7E700BF8B
:107B2000CC550020D0560020C85500201456002007
:107B3000D455002018560020B055002030B587B02D
:107B40000B9C7CB10C9DB5B1A4250495049DA42D7E
:107B50001AD04FF0500383F31188BFF36F8FBFF338
:107B60004F8FFEE74FF0500383F31188BFF36F8F01
:107B7000BFF34F8FFEE74FF0500383F31188BFF33D
:107B80006F8FBFF34F8FFEE7049D0C9D2C63022483
:107B900085F8A14000240394029505AC01940A9C49
:107BA0000094FFF73DFE0C98FFF7CEFE059807B056
:107BB00030BD2DE9F04385B00746884614461E4681
:107BC000900000F071FF08B38146A42000F06CFF24
:107BD0000546A8B1C0F83090002380F8A130039387
:107BE00002900D9B01930C9B009333462246414625
:107BF0003846FFF715FE2846FFF7A6FE012007E0EE
:107C0000484600F0D3FF4FF0FF3001E04FF0FF3067
:107C100005B0BDE8F083000010B588B000240594DD
:107C2000069407AA06A905A8F9F748FA059B029346
:107C3000069B019300942346079A10491048FFF7CA
:107C40007DFF104B1860B8B14FF0500383F31188DB
:107C5000BFF36F8FBFF34F8F0B4B1B6850330B4A33
:107C600013600B4B4FF0FF321A600A4B01221A606F
:107C7000094B1C6000F0F8FD08B010BD3861010828
:107C80007D7A0008AC550020D05600206C00002002
:107C9000B0550020C4550020CC550020024A13687E
:107CA00001331360704700BFA8550020014B1868CE
:107CB000704700BFCC55002008B500F061FE014BB5
:107CC000186808BDCC550020F8B53A4B1B68002B4E
:107CD00069D1394B1D6801351D60C5B9374B1B682B
:107CE0001B6843B14FF0500383F31188BFF36F8FCC
:107CF000BFF34F8FFEE7314A1168314B18681060AF
:107D00001960304A136801331360FFF773FD2E4B7F
:107D10001B68AB423DD900272C4B1B68DB6A03EB89
:107D200083039A002A4B9B58012B00D90127294B2A
:107D30001B68002B3CD001273AE001271F4B1B6832
:107D40001B6843B31D4B1B68DB68DC6863689D429E
:107D500026D3261D3046FEF784FFA36A1BB104F12B
:107D60001800FEF77EFFE36A01229A401A4908686C
:107D700002430A6003EB83039A003146144810441F
:107D8000FEF74BFFE26A114B1B68DB6A9A42D4D2C2
:107D9000D4E70027D2E70C4B4FF0FF321A60BBE765
:107DA000094A1360B8E70D4A1368013313600027CE
:107DB0003846F8BDA8550020CC55002018560020A4
:107DC00014560020B8550020B0550020D056002091
:107DD00044560020BC550020C8550020C055002046
:107DE00038B5354B1B6843B94FF0500383F3118806
:107DF000BFF36F8FBFF34F8FFEE700F09BFC2E4B5E
:107E00001A68013A1A601B68002B4FD12B4B1B6874
:107E10000BB900244BE00024294B1B681BB3284BF3
:107E2000DB68DC6804F11800FEF71BFF251D2846FF
:107E3000FEF717FFE06A01238340224A11680B43D3
:107E4000136000EB800029461F4B03EB8000FEF718
:107E5000E4FEE26A1D4B1B68DB6A9A42DCD31C4BD2
:107E600001221A60D8E70CB1FFF7C4FC194B1C685B
:107E700084B9174B1C68D4B14FF0E0234FF0805207
:107E8000C3F8042DBFF34F8FBFF36F8F01240EE0B3
:107E9000013C07D0FFF718FF0028F9D00C4B012256
:107EA0001A60F5E70B4B00221A60E2E7002400F0AD
:107EB00063FC204638BD00BFA8550020D0550020E7
:107EC00000560020C855002044560020D0560020FF
:107ED000BC550020C055002010B5A8B10446104B79
:107EE0001B6843B14FF0500383F31188BFF36F8FCA
:107EF000BFF34F8FFEE7FFF7D1FE00212046FFF7CB
:107F0000D1FDFFF76DFF48B94FF0E0234FF08052ED
:107F1000C3F8042DBFF34F8FBFF36F8F10BD00BFA9
:107F2000A8550020224B1B681BB1224B01221A606E
:107F30007047204B00221A601F4B1B68B3FA83F373
:107F4000DBB2C3F11F0303EB83018A001B498A588C
:107F500042B94FF0500383F31188BFF36F8FBFF323
:107F60004F8FFEE7154803EB83018A0002445168F6
:107F70004968516003EB830C4FEA8C0208320244DB
:107F800091420DD003EB83039A000C4B13445B68C2
:107F9000DA680B4B1A601B6850330A4A136070474B
:107FA000486862469100054A0A445060EAE700BF0B
:107FB000A8550020BC550020C8550020445600207C
:107FC000D05600206C00002058B110B50C46094A6C
:107FD00011681831FEF72CFE01212046FFF762FDE3
:107FE00010BD4FF0500383F31188BFF36F8FBFF3C1
:107FF0004F8FFEE7D056002038B5C368DC6824B345
:1080000004F118052846FEF72CFE184B1B682BBB05
:10801000251D2846FEF725FEE06A01238340144A09
:1080200011680B43136000EB80002946114B03EBF2
:108030008000FEF7F2FDE26A0F4B1B68DB6A9A4292
:1080400011D901200D4B186038BD4FF0500383F358
:108050001188BFF36F8FBFF34F8FFEE729460848A3
:10806000FEF7DBFDE7E70020EEE700BFA8550020A4
:10807000C855002044560020D0560020BC55002092
:1080800000560020034B1B680360034B1B684360D2
:10809000704700BFB8550020CC550020F8B5C8B1D6
:1080A0000C460546F9B100F045FB1B4B19686B689F
:1080B000C81A2268B2F1FF3F26D0184E36682F68E2
:1080C000B74201D08B4224D9824215D800232360C5
:1080D00001241AE04FF0500383F31188BFF36F8F30
:1080E000BFF34F8FFEE74FF0500383F31188BFF3C8
:1080F0006F8FBFF34F8FFEE75B1A13442360284650
:10810000FFF7C0FF002400E0002400F035FB20460C
:10811000F8BD0124F9E700BFCC550020B855002078
:10812000014B01221A607047BC550020014B1868B2
:10813000704700BFD0560020054B1B6833B1054B7C
:108140001B680BB100207047022070470120704768
:10815000C4550020A8550020002848D038B5044652
:10816000C36A254A1268D26A934238D28269002AC9
:1081700005DB214A1268D26AC2F107028261616995
:1081800003EB83031D4A02EB8303994205D01A4B8C
:108190001B68DB6AE362012038BD251D2846FEF717
:1081A00060FD38B9E36A01229A4015490B6823EA59
:1081B00002030B60104B1B68D86AE062012404FACA
:1081C00000F30F4A11680B43136000EB800029464F
:1081D0000A4B03EB8000FEF720FD2046DCE7826CB3
:1081E000054B1B68DB6A9A4203D30020D4E70020CA
:1081F00070470120D0E700BFD05600204456002031
:10820000C855002000284BD038B50446264B1B68C3
:10821000834208D04FF0500383F31188BFF36F8F70
:10822000BFF34F8FFEE7C36C43B94FF0500383F3A6
:108230001188BFF36F8FBFF34F8FFEE7013BC3641D
:10824000C16A826C91422DD00BB1002038BD051D52
:108250002846FEF706FD68B9E36A03EB8302920045
:1082600012498A5832B901229A4011490B6823EA0F
:1082700002030B60A06CE062C0F10703A36101245C
:1082800004FA00F30A4A11680B43136000EB800004
:108290002946064B03EB8000FEF7BFFC2046D5E7DE
:1082A000002070470020D1E7D0560020445600201F
:1082B000C855002000284FD038B50446C36C43B9D8
:1082C0004FF0500383F31188BFF36F8FBFF34F8FCD
:1082D000FEE7826C8A4200D20A46E16A914201D0EE
:1082E000012B00D038BD1D4B1B68A3422BD0E2628E
:1082F000A369002B02DBC2F10702A261626901EBF4
:108300008101174B03EB81039A42EBD1251D2846CF
:10831000FEF7A7FC38B9E36A01229A4011490B68BD
:1083200023EA02030B60E06A012383400D4A1168CF
:108330000B43136000EB80002946094B03EB8000E0
:10834000FEF76BFCCEE74FF0500383F31188BFF3C9
:108350006F8FBFF34F8FFEE7704700BFD0560020EE
:1083600044560020C8550020054B1B6823B1044B20
:108370001A68D36C0133D364014B1868704700BF8F
:10838000D0560020F8B506460F4614461D4600F0AC
:10839000D1F9244B1B6893F8A020D2B2022A0CD04A
:1083A000204A1168D1F89C3023EA0603C1F89C30BA
:1083B0001368012283F8A020D5B900F0DDF900F0A0
:1083C000B9F924B1174B1B68D3F89C302360154BC7
:1083D0001B6893F8A030DBB2022B18D00024114B9D
:1083E0001B68002283F8A02000F0C6F92046F8BDE3
:1083F00011462846FFF756FB4FF0E0234FF080521E
:10840000C3F8042DBFF34F8FBFF36F8FD5E7054B34
:108410001A68D2F89C3023EA0703C2F89C30012482
:10842000DDE700BFD0560020F8B5B0B10E461446C7
:108430001D46074600F07EF915B1D7F89C302B6039
:1084400097F8A030DBB2022287F8A020042C27D8AE
:10845000DFE804F0110C181E21004FF0500383F3E5
:108460001188BFF36F8FBFF34F8FFEE7D7F89C20C3
:108470003243C7F89C20012B20D0012400F07CF966
:108480002046F8BDD7F89C200132C7F89C20F2E7BF
:10849000C7F89C60EFE7022B40D0C7F89C60EAE782
:1084A000D7F89C20B2F1FF3FE5D04FF0500383F3A3
:1084B0001188BFF36F8FBFF34F8FFEE73C1D20463F
:1084C000FEF7CFFBF86A01238340164A11680B437D
:1084D000136000EB80002146134B03EB8000FEF796
:1084E0009CFBBB6A43B14FF0500383F31188BFF389
:1084F0006F8FBFF34F8FFEE7FA6A0C4B1B68DB6A86
:108500009A420DD94FF0E0234FF08052C3F8042D6A
:10851000BFF34F8FBFF36F8F0124AFE70024ADE7A8
:108520000124ABE7C855002044560020D056002057
:1085300018B32DE9F0410E4614461D46074600F0DB
:108540001FFAEFF311834FF0500282F31188BFF34B
:108550006F8FBFF34F8F984615B1D7F89C302B60C3
:1085600097F8A030DBB2022287F8A020042C27D88D
:10857000DFE804F0110C181E21004FF0500383F3C4
:108580001188BFF36F8FBFF34F8FFEE7D7F89C20A2
:108590003243C7F89C20012B20D0012088F311889A
:1085A000BDE8F081D7F89C200132C7F89C20F2E7A3
:1085B000C7F89C60EFE7022B46D0C7F89C60EAE75B
:1085C000D7F89C20B2F1FF3FE5D04FF0500383F382
:1085D0001188BFF36F8FBFF34F8FFEE7BB6A43B1C4
:1085E0004FF0500383F31188BFF36F8FBFF34F8FAA
:1085F000FEE7174B1B680BBB3C1D2046FEF731FB0B
:10860000F86A01238340134A11680B43136000EB9F
:1086100080002146104B03EB8000FEF7FEFAFA6A59
:108620000E4B1B68DB6A9A4210D9069B13B10123DB
:10863000069A136001200A4B1860AFE707F1180192
:108640000848FEF7EAFAEAE70020A7E70120A5E7D5
:10865000A8550020C855002044560020D0560020C0
:10866000BC5500200056002082B0002301930D4B22
:108670001B68B3F1FF3F08D04FF0500383F311881C
:10868000BFF36F8FBFF34F8FFEE74FF0500383F3BD
:108690001188BFF36F8FBFF34F8F019B002BFCD06E
:1086A00002B070472000002008480068006880F38E
:1086B00008884FF0000080F3148862B661B6BFF3FB
:1086C0004F8FBFF36F8F00DF00BF000008ED00E0A9
:1086D000DFF80C00016841F4700101607047000090
:1086E00088ED00E04FF0807340F8043C21F0010178
:1086F00040F8081C054B40F80C3C40F8202C6FF06B
:10870000020340F8243C4438704700BF69860008E3
:10871000074B19680868B0E8F04F80F30988BFF389
:108720006F8F4FF0000080F311887047AFF3008027
:10873000D05600204FF0500383F31188BFF36F8FA2
:10874000BFF34F8F0B4A136801331360012B00D026
:1087500070474FF0E023D3F8043D13F0FF0FF7D03C
:108760004FF0500383F31188BFF36F8FBFF34F8F28
:10877000FEE700BF20000020094B1B6843B94FF003
:10878000500383F31188BFF36F8FBFF34F8FFEE762
:10879000013B034A13600BB983F31188704700BF94
:1087A0002000002000000000000000000000000089
:1087B000EFF30980BFF36F8F154B1A681EF0100F8F
:1087C00008BF20ED108A20E9F04F10602DE9090064
:1087D0004FF0500080F31188BFF34F8FBFF36F8FBE
:1087E000FFF7A0FB4FF0000080F3118809BC196867
:1087F0000868B0E8F04F1EF0100F08BFB0EC108A08
:1088000080F30988BFF36F8F704700BFAFF300801C
:10881000D056002008B54FF0500383F31188BFF302
:108820006F8FBFF34F8FFFF74FFA28B14FF0E02360
:108830004FF08052C3F8042D002383F3118808BD44
:108840004FF0E022002313619361054B1B6805493B
:10885000A1FB03139B09013B53610723136170477D
:1088600000000020D34D62104FF0E023D3F8002D1C
:108870003D4B9A421CD04FF0E023D3F8002D3B4BE8
:108880009A421ED030B583B0394B1A78D2B20192D9
:10889000FF221A701B78DBB28DF803309DF803308D
:1088A00003F05003334A1370334B07221A601BE066
:1088B0004FF0500383F31188BFF36F8FBFF34F8FD7
:1088C000FEE74FF0500383F31188BFF36F8FBFF3C0
:1088D0004F8FFEE7284A1368013B13609DF8033071
:1088E0005B00DBB28DF803309DF8033013F0800F8E
:1088F000F0D1214B1B68032B08D04FF0500383F3BA
:108900001188BFF36F8FBFF34F8FFEE71B021A4A28
:10891000136003F4E0631360019BDBB2144A13702D
:108920004FF0E024D4F8203D43F47003C4F8203D18
:10893000D4F8203D43F07043C4F8203DFFF780FF9A
:1089400000250E4B1D60FFF7C3FED4F8343F43F003
:108950004043C4F8343FFFF7A7FEFFF7E3FAFFF701
:1089600083FE284603B030BD71C20F4170C20F4173
:1089700000E400E0D8560020D4560020200000205B
:10898000EFF305830F2B0FD9114A9B5CDBB2114A21
:1089900012789A4208D94FF0500383F31188BFF33D
:1089A0006F8FBFF34F8FFEE74FF0E023D3F80C3DFE
:1089B00003F4E063084A1268934208D94FF0500369
:1089C00083F31188BFF36F8FBFF34F8FFEE77047BC
:1089D000F0E300E0D8560020D4560020134A12F0ED
:1089E000070F1FD0D11D21F00701C1F5EA43303335
:1089F00013440A460E480260002141601344083BBC
:108A000023F007030B48036059601960991A5160FD
:108A10001360094B1960094B1960094B4FF0004274
:108A20001A60704747F23053E4E700BFFC5600205D
:108A3000F4560020F0560020E8560020EC560020A6
:108A4000DC560020164B1A461B688342FBD3516844
:108A500002EB010C844509D0416800EB010C634531
:108A600009D00360904219D01060704740680144FB
:108A700051601046F0E710B40A4C2468A3420BD0B2
:108A80005B681944416013681B680360904200D022
:108A900010605DF8044B70470460F7E7704700BF53
:108AA000F4560020F056002038B50446FFF7F6F8DB
:108AB000384B1B68B3B1384B1B681C4250D1002C9B
:108AC00050D004F1080214F0070F02D022F0070280
:108AD0000832002A55D0314B1B68934253D330499A
:108AE0000C6804E0FFF77AFFE5E721461C4663685F
:108AF000934202D22368002BF7D1264B1B68A34276
:108B000043D00D68083523680B6063689B1A102BEF
:108B100010D9A01810F0070F08D04FF0500383F3BE
:108B20001188BFF36F8FBFF34F8FFEE74360626022
:108B3000FFF788FF626819490B689B1A0B60194997
:108B400009688B4201D217490B60134B1B68134312
:108B5000636000232360144A13680133136002E04A
:108B6000002500E00025FFF73BF915F0070F0ED0B8
:108B70004FF0500383F31188BFF36F8FBFF34F8F14
:108B8000FEE70025EFE70025EDE70025EBE72846A7
:108B900038BD00BFF0560020DC560020EC56002007
:108BA000F4560020E8560020E4560020002834D077
:108BB00038B50446A0F1080550F8043C174A12687D
:108BC000134208D14FF0500383F31188BFF36F8F26
:108BD000BFF34F8FFEE750F8081C41B14FF0500330
:108BE00083F31188BFF36F8FBFF34F8FFEE723EA44
:108BF000020340F8043CFFF751F854F8041C084AFB
:108C000013680B4413602846FFF71CFF054A1368DE
:108C100001331360FFF7E4F838BD7047DC560020DD
:108C2000EC560020E056002010B50C460A680C32C5
:108C300001F052F900B110BD94F90400FBE7000007
:108C400070B58AB00C46114600F016FA054638B1E8
:108C50008DF80C40019001A91A48FFF7E5FF10B903
:108C600028460AB070BD6B682BB1174BA322174979
:108C7000174809F0A1FC05F11004204606F0C4FADB
:108C800088B105F10C06304606F0EAFA90B130469C
:108C900006F0E1FA204606F065FA2946042001F0C4
:108CA0003DFD0025DCE7084BA4220A49084809F0ED
:108CB00083FCE6E7044BA9220749054809F07CFC40
:108CC000E5E700BF6390000840610108906101087A
:108CD000F4600108B4610108CC61010848B100B535
:108CE0008BB0019001A90448FFF79EFF0BB05DF81F
:108CF00004FB0020704700BF5591000838B550B103
:108D00000546FFF7EBFF044608B1204638BD28466C
:108D100000F0F2F9F9E70024F7E7000000B58BB0A6
:108D200060B10346A1B101930391ADF8102001A9F0
:108D30000848FFF779FF0BB05DF804FB064B4FF4D2
:108D40009D720649064809F037FC6FF00F00F2E704
:108D50000449E8E7F591000840610108E86101086D
:108D6000F4600108C47A010800B58BB040B10190ED
:108D7000039101A90748FFF757FF0BB05DF804FB0B
:108D8000054B4FF46D720549054809F015FC6FF06D
:108D90000F00F2E721920008406101080462010817
:108DA000F460010838B550B1044606F0A3FA94F90E
:108DB00008500023237206F0A9FA284638BD002582
:108DC000FBE70000F0B583B000230193002933D006
:108DD000044617460E4600230B60002836D000F1EB
:108DE0001005284606F010FA002839D094F82030F3
:108DF00013F0020F09D117F0040F06D113F0010F81
:108E000003D194F90830002B3FD001A9284606F081
:108E1000E8F9B0F1FF3F2BD0019B002B40D0019B24
:108E20001B681A89636A13B1012120469847019B88
:108E30003360002003B0F0BD1F4B40F24A221F49AF
:108E40001F4809F0B9FB6FF00F00F3E71A4B4FF41E
:108E500013721C491A4809F0AFFB6FF00F00E9E7E5
:108E60002046FFF79FFF0028E4D16FF00A00E1E7FA
:108E70002046FFF797FF0028DCD194F8203013F04C
:108E8000010F15D06FF00A00D4E7E26901A9284666
:108E900006F07BF9B0F1FF3FBED16FF00200C9E7E9
:108EA000054B40F293220849054809F085FBB6E7D7
:108EB0006FF00600BEE700BF4061010820620108B4
:108EC000F4600108406201085C62010808B538B12D
:108ED000037803F0F003102B02D0FFF773FF08BDF7
:108EE000044B40F24E320449044809F065FB6FF030
:108EF0000F00F4E74061010868620108F4600108AE
:108F000038B5044603685B6833B1144B40F2652200
:108F10001349144809F050FB25682B7803F0F0033F
:108F2000202B02D0FA23237138BD002002F008FF65
:108F3000686023685A683AB11B78222B0BD02268EC
:108F40000949506802F0B0FE23685B68002BEBD142
:108F5000FF232371E8E701231374F0E7946201080B
:108F6000C8620108F46001086D8F00082DE9F04126
:108F70000446154698460E4669B3002C32D0636805
:108F8000B34205D0244BEE222449254809F014FBB6
:108F900004F11007384606F037F968B3032001F0F2
:108FA0008FFB064668B305604560B8F1000F2CD012
:108FB000D8F80030B360BDF81830B3812D89314640
:108FC000384606F0D8F810BB636AC3B12A460021C0
:108FD0002046984713E0104BE5221249104809F04B
:108FE000EBFACAE70C4BE6220F490D4809F0E4FA08
:108FF000284601F065FF02E0284601F061FFBDE868
:10900000F081284601F05CFFF9E70023D2E7304603
:1090100000F03AF9F3E700BF946201082C630108FD
:10902000F4600108E86201080C63010810B582B021
:1090300000F11004204606F0E7F820B902B010BD98
:10904000019800F021F901A9204606F0CAF8B0F114
:10905000FF3FF5D1204606F085F8204606F0DAF805
:10906000ECE708B50023037103685B6803B108BD32
:10907000FFF746FFFBE7000070B505460E460420EB
:1090800001F01EFB044658B30023037205704360D1
:1090900005F0F005202D17D100F110050621284616
:1090A00006F04CF8B8B9002104F10C0006F0B5F850
:1090B000C0B9002363704FF0FF3262616662A36142
:1090C000E36184F820300BE0084B40F2E5220849C8
:1090D000084809F071FA2146042001F01FFB002422
:1090E000204670BD284606F03DF8F4E7946201087A
:1090F0004C630108F460010838B50446436833B195
:10910000104B4FF447721049104809F055FA04F11A
:10911000100006F079F860B904F10C05284606F055
:109120009AF8284606F0A2F82146042001F0F6FA43
:1091300038BD044B40F223320549044809F03CFA9B
:10914000EAE700BF9462010874630108F460010853
:10915000A463010838B5044603685D7815BB032D88
:1091600034D0002323712068FFF760FF23685A681A
:109170003AB11B7803F0F003202B2ED02368002295
:109180005A602068436A13B100221146984720684C
:10919000436A13B100220221984720680C3006F080
:1091A0005FF838BD1B7803F0F003102B06D1022DB9
:1091B000D7D0032D0AD0FB232371EEE70A4B40F2F0
:1091C0005E420A490A4809F0F7F9F0E7236893F884
:1091D000203013F0040FC4D1EDE70023D3612368DE
:1091E000586802F075FDC9E794620108E063010860
:1091F000F460010810B504460368586868B11B782C
:1092000003F0F003202B03D06FF00500207110BD98
:10921000A289A16802F02EFBF8E76FF00500F5E7E0
:1092200010B504460068FFF7BDFD034648B9236842
:109230005868C0B11B7803F0F003202B03D06FF007
:109240000A03237110BDA1688B6823B9096802F075
:10925000BBFC0346F5E78B8901F10802096802F0BF
:109260006DFC0346EDE76FF00A03EAE700F1100337
:10927000DBB2102B04D84042024B53F82000704759
:1092800005207047F463010868B110B50446006812
:1092900020B101F015FE0023636023602146032006
:1092A00001F03CFA10BD704710B540B104460068AB
:1092B00008B101F005FE00236360236010BD034B7D
:1092C00081220349034809F077F9F7E73864010878
:1092D000AC640108F460010870B5B0B10E461546E3
:1092E0000446006808B101F0EBFD41220021362060
:1092F00001F04EFE206088B1466023681D8123681E
:109300005D8123686360002070BD074B9922074987
:10931000074809F051F96FF00F00F5E7002363608B
:109320004FF0FF30F0E700BF38640108C86401085F
:10933000F4600108032803D8024B03EB00107047C8
:109340000020704730CC002008B5FFF7F3FF08BDC0
:1093500008B5FFF7F9FF034608B102680AB11846DD
:1093600008BD1346FBE7000008B5FFF7F1FF00B1A9
:1093700008BD024B09221A60FAE700BF301A01202B
:1093800030B5039D4FF0000C02E0F5B90CF1010C73
:109390008469644515D9446904EBCC0E54F83C400B
:1093A0008C42F3D122B1BEF9044014F0010F0AD16E
:1093B000002BEAD0BEF9044014F0020FE5D00120E2
:1093C00000E0002030BD0120FCE70120FAE70000AA
:1093D00008280DD020280BD0042809D008B5054B4B
:1093E00040F639320449054809F0E6F8002008BD86
:1093F000704700BFE064010814650108F4600108CB
:10940000F8B506460D460024032C31DC05F072FF4A
:109410002301194AD3581BB105F078FF0134F3E753
:10942000230102EB0417D65005F070FF00237B6088
:10943000BB7B8BB9104B03EB041300221A813378EA
:1094400003F0F003102B0FD001250B4B03EB04139B
:109450005D8100229A810DE0084B40F20E220849FE
:10946000084809F0A9F8E5E7002DEED00125ECE762
:109470004FF0FF342046F8BD30CC0020E0640108F6
:109480002C650108F4600108F0B585B016461C464D
:109490000A9D0F46D1B10CB345B310238DF80030AF
:1094A00002238DF80130304600F068FDADF802006F
:1094B0003B6801930023029303932A689DF80030D0
:1094C0009A421BD323D92B60002618E0114B40F29F
:1094D00007421149114809F06FF8DCE70D4B4FF4D2
:1094E00081620F490D4809F067F8D5E7094B40F252
:1094F00009420C49094809F05FF8CEE701262A68BD
:109500006946204609F0F6F9304605B0F0BD002660
:10951000F5E700BFE06401084C650108F46001084C
:1095200060650108706501082DE9F04F85B081463E
:10953000884616469A4693686BB118F0080F17D004
:109540000422D9F804300393A3B1039B1B681F893D
:109550000025AB462EE0D368002BEEDD324B40F207
:1095600049423249324809F027F86FF00F0045E0D0
:109570000022E6E703A9D9F80000FFF7A7FC0028BE
:109580003CD1039B1BB1039BC9F80430DDE7264B9C
:1095900040F25E422749264809F00EF8F3E75B46A1
:1095A000224609580398006801F0EAFE5C441FFA5D
:1095B00084FB0135F368AB420DDDBB450BD2A7EB55
:1095C0000B04A4B2B168E80001EBC5035B68A342D9
:1095D000E5D89CB2E3E733680BB172688AB900231F
:1095E000B36133690BB10023736118F0010F12D01E
:1095F000BAF1000F16D0AAF80070002005B0BDE83F
:10960000F08F03998A89301D00900831D9F8000045
:10961000FFF73AFFE3E70023C9F804300398FFF7A8
:1096200033FEE5E70020E9E7E06401088065010812
:10963000F46001085C6201082DE9F04182B0054642
:109640000E4690461F462E4B1C683EE096B1A2681F
:109650008AB12B46002D0ADB5B1152F8233005F04E
:109660001F02D34013F0010F05D0012003E005F1E4
:109670001F03F1E73046B8F1000F0FD070B9E26870
:1096800062B12B46002D31DB5B1152F8233005F01F
:109690001F02D34013F0010F00D001201FB368B99F
:1096A000226902B32B46002D23DB5B1152F82330D5
:1096B00005F01F02D34013F0010F14D00123E36122
:1096C00004F1200005F0C2FD2468ACB1E069002877
:1096D000FAD16369002BB9D0009743463246294638
:1096E0002046FFF74DFE0028EED0E7E705F11F0307
:1096F000CAE705F11F03D8E702B0BDE8F08100BF5B
:109700002CCC002000286DD02DE9F0410C460546F8
:109710004669002E0EDB3046FFF726FE054668B38D
:1097200005F0E8FD0746042C38D8DFE804F0111CEA
:109730002931340005F0DEFD6E69002E02DB05F0F4
:10974000E5FDE8E70CB9013E6E6105F0DFFD15E0CF
:10975000B5F9083001331BB22B81012B01DD002349
:1097600006E0012304E0B5F90830013B2B8100231A
:10977000AA7B02B1DBB9384605F0C8FDBDE8F0812F
:109780006B891BB9012301226A81F1E70023FAE703
:1097900000236B81ECE70123AB81E9E7124B4FF427
:1097A0001F621249124808F007FF0123E0E7B5F9EC
:1097B0000840002CD4BF00240124B5F80A80B8F179
:1097C000000818BF4FF00108AD89003D18BF012502
:1097D000384605F09BFD2B46424621463046FFF7B2
:1097E0002BFFCBE7704700BFE0640108AC650108C0
:1097F000F4600108F8B50C4615461E46FFF7A8FDB3
:10980000002800F0DC800746002C00F0BC8040F609
:10981000FF739C4240F0D58041F20B039D4200F360
:10982000D28041F205039D420EDBA5F58052053A38
:10983000062A00F2CA80DFE812F033004D00C800AB
:10984000C800C80066008100082D01D0202D1FD15E
:10985000202D06D13B681B7803F0F003202B40F04D
:10986000B6802846FFF7B4FD0346069A032A40F265
:10987000B0803A68002A00F0AE805268002A00F0FA
:10988000AC80306830B1517A0B435372002099E0BC
:109890005C2097E0517ADB435BB20B40537291E05E
:1098A000069B0F2B40F29B800168002900F09980F5
:1098B0003068B3685D4A82FB0342DB17C3EBA21337
:1098C0004FF47A7202FB0033002BC0F28C808B6164
:1098D000002077E0069B0F2B40F28780016800296B
:1098E00000F085803068B368504A82FB0342DB1782
:1098F000C3EBA2134FF47A7202FB0033002B78DB28
:10990000CB6100205EE0069B032B74D90368002B1B
:1099100073D05A68002A72D01B7803F0F003202B12
:109920006FD1306828B1137C43F001031374002019
:1099300048E0137C03F0FE03137443E0069B052B01
:1099400061D90368002B60D033787BB900213A6875
:10995000137803F0F003202B10D0354B40F67D52E6
:109960003449354808F028FE00202BE0304600F04E
:10997000BBFF01460028EAD1132023E0506802F023
:1099800047F900201EE0012D0ED0022D3FD1069B8D
:10999000032B3ED90368002B3DD05B68002B3CD0E5
:1099A0003278DA7220460DE0069B032B37D9036824
:1099B000BBB35B68BBB332789A72204602E00920E1
:1099C00000E05C20F8BD5C20FCE75C20FAE75C204E
:1099D000F8E71620F6E71620F4E71620F2E716203F
:1099E000F0E71620EEE71620ECE71620EAE716204F
:1099F000E8E71620E6E71620E4E71620E2E716205F
:109A0000E0E75C20DEE71620DCE71620DAE75C20E2
:109A1000D8E71620D6E71620D4E71620D2E716207E
:109A2000D0E71620CEE71620CCE700BFD34D62105A
:109A3000E0640108BC650108F460010870B582B0FB
:109A40000C461546FFF790FC78B30646102D13D14F
:109A50006378022B10D114F0030F0DD163680193CA
:109A6000608800F08BFA024601A93068FFF756F9CA
:109A700098B9002002B070BD0D4B40F2E2220D49B2
:109A80000D4808F099FD6FF00F00FFF7EFFB08B1EC
:109A90000A4A10604FF0FF30ECE7FFF7E7FB08B130
:109AA000064A10604FF0FF30E4E74FF0FF30E1E787
:109AB000E0640108E8650108F4600108301A01203B
:109AC0002DE9F0418CB00746884614461E46139D8A
:109AD000FFF74AFC002833D00022ADF80A20CDF869
:109AE0000C80049409920A920B9203AB0793012312
:109AF0000893129B0593CDB12B68069300970DF147
:109B00000A0305AA3146FFF70FFD88B9BDF80A0020
:109B1000A04228BF20466FF00043984200D3184669
:109B20000DB1069B2B600CB0BDE8F0810023E4E78B
:109B3000FFF79CFB08B1044A10604FF0FF30F2E7DA
:109B40004FF0FF30EFE700BF301A01202DE9F0435E
:109B500085B00E4614460C9D0D9FFFF705FC0028AE
:109B600068D0804603681B7803F0F003102B33D0D5
:109B7000B4F5803F3AD21FFA84F9002D3CD0102F63
:109B80003DD1002D3BD06B78022B38D115F0030F5F
:109B900035D1002301930093002D41D06B680293CF
:109BA000688800F0EBF9ADF80C004A46314668468B
:109BB000FFF792FB0546002835D06846FFF774FB97
:109BC0002846FFF753FB08B11D4A1060002D34D121
:109BD000A0B205B0BDE8F0836FF00F00FFF746FBC1
:109BE00008B1174A10604FF0FF30F2E7144B5A22C9
:109BF0001A604FF0FF30ECE7002FCAD0BFE7114BDF
:109C000040F252621049114808F0D6FC6FF00F0084
:109C1000FFF72CFB08B10A4A10604FF0FF30D8E77D
:109C200000200290BFE76946D8F80000FFF79CF8D3
:109C30000546C2E74FF0FF30CBE74FF0FF30C8E7F3
:109C4000301A0120E064010804660108F46001088C
:109C500038B5134602291BD0032907D0012922D089
:109C60001B4B16221A604FF0FF340FE0194AD9B28D
:109C70004020FEF7E5FF0546E5B100212846FFF745
:109C8000BFFB0446B0F1FF3F1AD06861204638BDE3
:109C9000882A06D020200F4A0021FEF7D1FF054672
:109CA000EAE72120F7E70B4A00211020FEF7C8FF62
:109CB0000546E1E7064B69221A604FF0FF34E5E7FD
:109CC0002846FFF71BF8024B17221A60DEE700BF99
:109CD000301A0120059700082DE9F04182B00546B1
:109CE000884616461C46FFF73FFB00B3A4B1114F50
:109CF000384605F0DCFA089B00932346324641467D
:109D00002846FFF777FD0446384605F0D7FA4CB9E8
:109D1000204602B0BDE8F081074B0E221A604FF0DA
:109D2000FF34F5E7044B1C604FF0FF34F0E74FF0D1
:109D3000FF34EDE770CC0020301A0120F8B506465C
:109D40000F460EE0144C204605F0B8FA00223946C2
:109D5000304605F01AFA204605F0A9FAF8BD01F0E0
:109D6000FFFB01F01DFC0446B0F1FF3FEAD00028E4
:109D7000F5D0094D284605F0A1FA2246394630466D
:109D800005F003FA0446284605F091FAB4F1FF3FC6
:109D9000E4D101F0E5FBE4E770CC002010B5044607
:109DA0000378012B17D0022B1DD033B1104BCF22DB
:109DB0001049114808F000FC08E0C3688168406859
:109DC000984720B92146062000F0A8FC10BD606825
:109DD00001F076F8F6E74368806898472146052049
:109DE00000F09CFCF2E7436880689847EEE700BF0C
:109DF0002466010854660108F460010800B583B0C8
:109E00000C4805F054FA0C4B1B682BB10B4A106838
:109E1000984701E0FFF7C2FF01A90948FFF78EFF4D
:109E200001980028F6D1074B91220749074808F00E
:109E3000C3FBF1E770CC00207CCC002078CC002064
:109E400074CC00202466010854660108F4600108FF
:109E5000F8B507460E461546124805F0D5F978B113
:109E6000062000F02DFC0446C0B1002303704760BB
:109E70008660C56001460B4805F07DF938B9F8BD2C
:109E8000094BFC2209490A4808F096FBE8E72146FD
:109E9000062000F043FC4FF0FF30F0E74FF0FF30BA
:109EA000EDE700BF74CC0020246601087466010849
:109EB000F460010808B591F83D3013F0180F03D095
:109EC000034AFFF7C5FF08BD024AFFF7C1FFFAE7E3
:109ED00025F0000885E2000870B504460D46054EE1
:109EE000304605F0E4F92846A047304605F0E6F98B
:109EF000002070BD70CC002030B583B005460C4604
:109F000000F04DF8134B1D60134B1C6006211348E5
:109F100005F014F968B9124805F0B8F988B90022BB
:109F200000924FF480630F490F4805F0CCF903B05D
:109F300030BD0E4B40F261220D490E4808F03CFB4B
:109F4000E9E70A4B40F265220B490A4808F034FB66
:109F5000E5E700BF7CCC002078CC002074CC00204A
:109F600070CC0020FD9D0008CC6601082466010825
:109F700084660108F4600108A8660108030A43EA40
:109F8000002080B27047030203F47F0343EA0063BA
:109F9000020A02F47F42134343EA1060704708B597
:109FA00005F068F900F0C4F800F064FB00F07CFCF8
:109FB00001F090FB01F0C0FA08BD0000014B1B68E6
:109FC00018447047A4CC0020024B1B68C01A80B212
:109FD000704700BFA4CC0020F8B50446FFF7F4FF9B
:109FE000074625882846FFF7E9FF0646648820468D
:109FF000FFF7E4FFB5F5486F10D8B4F5486F0FD8F8
:10A00000BC4202D00388BB420CD1094B1B68B3424F
:10A010000AD07388BB4209D1012000E00020F8BDBE
:10A020000020FCE70020FAE70120F8E70020F6E72F
:10A03000A0CC002038B50446344B1B6883423ED880
:10A04000334B1B68A34242D92379002B47D1238885
:10A05000B3F5486F4BD82088FFF7B0FF844215D086
:10A0600003799BB92A4B1B6883420FD0294B1B688D
:10A07000834244D000882080B0F5486F06D0FFF7B7
:10A080009DFF05462046FFF79FFF68806088FFF729
:10A0900095FF0546844211D003797BB91D4B1B689F
:10A0A000A3422FD020882880B0F5486F06D0FFF754
:10A0B00085FF04462846FFF787FF608038BD164BB2
:10A0C00040F2DF121549164808F076FAB8E7124B4D
:10A0D0004FF4F0721349124808F06EFAB4E70E4BD1
:10A0E00040F2E11210490E4808F066FAAFE70A4B59
:10A0F0004FF4F2720D490A4808F05EFAABE7054BDF
:10A100001C60B7E7034B1860CCE700BFA4CC00206D
:10A11000A0CC002098CC0020DC6601080C67010868
:10A12000F460010824670108406701085C670108C2
:10A1300038B5114C24F00304104B1C604FF44865F3
:10A1400025800023638023712846FFF737FF0C4BDF
:10A15000186001230371058045800A4B1C600A4882
:10A1600005F094F800B938BD084B40F21F220849A9
:10A17000084808F021FAF6E7ABCC0020A4CC002078
:10A18000A0CC002098CC00209CCC0020DC660108EC
:10A1900088670108F4600108002860D038B50446DB
:10A1A00010F0030F17D1A0F108052D4B1B68AB422F
:10A1B00005D800F10C032B4A1268934217D92A4B99
:10A1C00040F27F2229492A4808F0F6F905F092F872
:10A1D00005F09CF838BD244B40F2732225492448F1
:10A1E00008F0EAF905F086F805F090F8F2E7224861
:10A1F00005F05DF814F8043C9BB12846FFF7ECFE2F
:10A20000F0B1002304F8043C1C4B1B68AB4201D99D
:10A210001A4B1D602846FFF70DFF174805F04EF852
:10A22000D8E7114B4FF423721549114808F0C4F9CF
:10A23000114805F043F805F05DF805F067F8C9E747
:10A24000094B40F295220F49094808F0B5F90A4830
:10A2500005F034F805F04EF805F058F8BAE7704705
:10A26000A4CC0020A0CC0020DC660108C86701084F
:10A27000F4600108A46701089CCC002098CC002061
:10A28000E46701080C6801082DE9F8430546CC1C79
:10A29000A4B224F00304A4B20B2C04D9B4F5486F83
:10A2A00002D9002061E00C248C42C0F0A280544B03
:10A2B0001B68AB4203D8534B1B68AB4206D8524BCA
:10A2C00040F2D1225149524808F076F94C4B1B68B4
:10A2D000AB4245D84B4B1B68AB4241D9A5F10800B6
:10A2E000FFF772FE064635F8088CA8EB00081FFA47
:10A2F00088F8A8F108081FFA88F8444537D844457B
:10A3000079D87AD0434804F0D2FF35F8087C384633
:10A31000FFF754FE81460379002B3ED1B7F5486F15
:10A320002DD0B9F800703444A4B20834A4B23A4B2A
:10A330001B684B452BD02046FFF740FE00230371DE
:10A340000780468025F8084C0088B0F5486F02D099
:10A35000FFF734FE44802F4804F0B0FF284604E0A5
:10A3600004F0C8FF04F0D2FF2846BDE8F883264B6E
:10A370004FF439722949264808F01EF9BFE7224BED
:10A3800040F2F5222649224808F016F9C9E720468E
:10A39000FFF714FE204B1860CDE704F1140343458A
:10A3A000D9D83444A4B20834A4B2B7F5486F18D051
:10A3B0002046FFF703FE184B1B68834201D9164B5A
:10A3C00018600023037135F8083C0380468025F8A7
:10A3D000084C0088B0F5486FBDD0FFF7EFFD448012
:10A3E000B9E7094B40F216320D49094808F0E4F884
:10A3F000DEE70020B9E70020B7E72846B5E700BF51
:10A40000A4CC0020A0CC0020DC6601084068010834
:10A41000F46001089CCC002098CC0020586801080A
:10A4200078680108002800F0A3802DE9F041034678
:10A43000C61CB6B226F00306B6B20B2E04D9B6F58A
:10A44000486F02D9002091E00C269E42C0F0928015
:10A45000494804F02CFF494B1868FFF7B5FD054645
:10A460004FE0474B40F287324649474808F0A4F88E
:10A4700065E001230371414B1868A04212D03E48A9
:10A4800004F01CFF27440837404B1B689F421FD82D
:10A4900014F0030524D15DBB04F1080066E00088D8
:10A4A000FFF78CFD03791BB1384A12688242F6D15E
:10A4B000324A1060354A12688242E0D0002BDED06A
:10A4C0002F4B40F2B53232492F4808F075F8D6E7E5
:10A4D0002B4B40F2B9322F492B4808F06DF8D7E7E3
:10A4E000274B40F2BB322C49274808F065F8D2E7E9
:10A4F000234B40F2BD322949234808F05DF8CBE7F1
:10A500002588A8463746C6F548639D422AD2284684
:10A51000FFF754FD04460379002BF1D10388A3EB28
:10A520000803083BBB42EBD307F114029342A0D3CC
:10A530002E44B6B20836B6B2B6F5486F91D0304662
:10A54000FFF73CFD002303712388038045802680AC
:10A55000012323710088B0F5486F8CD0FFF72EFDE2
:10A56000468088E7044804F0A9FE0020BDE8F08199
:10A57000002070470020F9E79CCC002098CC0020F8
:10A58000DC66010878680108F4600108A0CC0020AE
:10A590008C680108A8680108D868010808690108E2
:10A5A00038B501FB00F4B4F5803F0AD2A0B2FFF742
:10A5B00039FF054618B12246002108F0A7F82846C1
:10A5C00038BD0025FBE7000038B5044604F092FED4
:10A5D0000546A3681C688CB122681A6014F0030F4A
:10A5E00004D1284604F092FE204638BD054B4FF4B6
:10A5F0008C720549054807F0DFFFF2E704F086FE9C
:10A60000F2E700BF2C6901085C690108F4600108E9
:10A6100038B505460C4611F0030F09D104F06AFE67
:10A62000AB681B682360AB681C6004F06FFE38BD2C
:10A63000034B4FF4B6720349034807F0BDFFEDE743
:10A640002C69010880690108F46001088368002210
:10A650001A604368033323F0030307E08168096845
:10A66000196081680B6001880B4401324188914276
:10A67000F4DC704710B5002406E0054B53F82400C5
:10A68000FFF7E4FF0134A4B2092CF6D910BD00BFD6
:10A69000F069010810B5044610B1FFF795FF10BD31
:10A6A000044B4FF49E720449044807F085FF20468E
:10A6B000F5E700BF2C690108A0690108F4600108F2
:10A6C00008B5092805D8074B53F82000FFF77CFF91
:10A6D00008BD054B40F257120449054807F06CFFCE
:10A6E0000020F5E7F06901082C690108B469010848
:10A6F000F460010808B518B109B1FFF789FF08BD7A
:10A70000034B40F295120349034807F055FFF6E763
:10A710002C690108A0690108F460010808B509283E
:10A7200006D821B1064B53F82000FFF771FF08BD92
:10A73000044B4FF4D5720449044807F03DFFF6E797
:10A74000F06901082C690108D4690108F460010866
:10A750006FF00B007047000070B516460A688368FA
:10A760009A4213D004460D4636B1A36833605DB1FA
:10A770002B68A360012070BD054B4FF4047205499E
:10A78000054807F019FFF0E70023F2E70020F2E7A1
:10A79000906A0108C46A0108F460010870B51646A1
:10A7A0000A68C3689A4213D004460D4636B1E3687E
:10A7B00033605DB12B68E360012070BD054B4FF441
:10A7C00014720549054807F0F7FEF0E70023F2E7A9
:10A7D0000020F2E7906A0108C46A0108F4600108E9
:10A7E00008B501F0B1FA08BD38B50C46054670B1A0
:10A7F00095F83D3003F00502052A07D114F0010F4A
:10A8000004D06A6812B113F0080F08D138BD064BA6
:10A8100040F26D320549064807F0CEFEE8E7291DF3
:10A82000284603F07BF9F1E7906A0108D46A010831
:10A83000F460010870B582B0044615460E4639B181
:10A8400075B1326863689A4212D1002002B070BDBF
:10A85000124B40F2CB121249124807F0ADFEEFE75F
:10A860000E4B4FF4E6720E490E4807F0A5FEE8E7DE
:10A8700001922B6001A92846FFF7B2FF5EB1336851
:10A88000636001212046FFF7AFFFE3690BB120466B
:10A8900098470120DAE70023F2E700BF906A010839
:10A8A000C46A0108F460010870470000014B186099
:10A8B000704700BF2405012000B1C161704700B19D
:10A8C00001627047024658B1064B186838B190F8DB
:10A8D00040300133DBB2934203D00068F6E77047A3
:10A8E000002070472805012010B50446B0B10230A1
:10A8F00006F0B6FDC2B20A4B186800E0006868B105
:10A9000090F840309342F9D1217890F83E30994246
:10A91000F4D1617890F83F309942EFD110BD00BF7B
:10A920002805012038B50C46054630B16CB12C60C5
:10A930000A4B1A686A601D6038BD094B40F2C96253
:10A940000849094807F038FEF0E7054B40F2CA62B3
:10A950000649054807F030FEE9E700BF2C05012055
:10A96000906A0108F86A0108F4600108146B010894
:10A97000F8B50D4616460A4B1C68074668B9094BE0
:10A9800040F2FC620849094807F016FE05E023681A
:10A9900032462946384698476468002CF7D1F8BDFE
:10A9A0002C050120906A0108286B0108F460010859
:10A9B0002DE9F04387B0044691461D468846A1B173
:10A9C000B9F1000F14D0B5B1B8F1000F02D0D8F82A
:10A9D000003093B96A4641462046FFF72BFF68B323
:10A9E000CDF80CD00127102609E0DFF87080E7E7EA
:10A9F000DFF86890E7E7194DE6E700273E4602AA30
:10AA000049462046FFF7A8FE18B146F0400602ABC3
:10AA1000049301AA29462046FFF7C0FE18B146F06C
:10AA2000200601AB059367B12EB103AA46F0800161
:10AA30002046FFF79DFF07B0BDE8F0830127002601
:10AA4000DDE76A4641462046FFF7F4FE0028EBD0DA
:10AA500046F01006CDF80CD0E7E700BFC47A010835
:10AA600070B5059C064628B3002C2CD0002933D0A5
:10AA7000002A33D0002B33D000207060B060F0602B
:10AA80003A4D7561B08686F83D00B062F062F061C3
:10AA90003062049870623648007886F84000069864
:10AAA00030613046FFF784FF3046A04700283ED093
:10AAB000002055E02F4B40F227122F492F4807F076
:10AAC0007BFD30464CE02B4B4FF494722C492B48C5
:10AAD00007F072FD002043E02A49C9E7294AC9E787
:10AAE000284BC9E7002386F8403024E0214B40F290
:10AAF0008B122549214807F05FFD09E094F84020BA
:10AB000096F840309A420ED024687CB1B442EDD021
:10AB10000135FF2DF2DD174B40F28D121B4917480E
:10AB200007F04AFDEAE7013386F840303CB196F879
:10AB30004030FF2BD6D0164B1C680025E5E796F871
:10AB40004030FE2B0DD00133094A1370104B1A68A8
:10AB500032601E60002201213046FFF709FF3046B7
:10AB600070BD034B00221A70F0E700BF51A7000828
:10AB700023050120906A0108406B0108F460010878
:10AB80005C6B0108C47A0108806B0108946B0108B2
:10AB90002805012010B584B0D0B1044690F83D30AE
:10ABA00013F0010F12D143F0010380F83D30C36967
:10ABB00003B1984701238DF8043001AA08212046EB
:10ABC000FFF7D6FE03212046FFF70EFE04B010BDAE
:10ABD000034B4FF454720349034807F0EDFCF5E7CB
:10ABE000906A0108C46B0108F460010810B584B0D4
:10ABF00038B1044690F83D3013F0010F09D104B08C
:10AC000010BD114B40F29B321049114807F0D4FCA3
:10AC1000F5E700238DF8043001AA0821FFF7A8FE0C
:10AC200094F83D3003F0FE0284F83D2013F0080F45
:10AC300005D1E369002BE2D020469847DFE72046A4
:10AC400002F0E8FEF5E700BF906A0108E06B01083A
:10AC5000F460010810B584B038B1044690F83D3076
:10AC600013F0040F09D004B010BD114B4FF47872EB
:10AC70001049114807F0A0FCF5E743F0040380F801
:10AC80003D3002F091FA204601F04EF903212046B2
:10AC9000FFF7AAFD236A0BB12046984701238DF8E0
:10ACA000043001AA04212046FFF762FEDBE700BF63
:10ACB000906A0108006C0108F460010810B584B0C6
:10ACC000B0B1044690F83D3013F0040F0ED003F0FD
:10ACD000FB0380F83D30036A03B1984700238DF8E9
:10ACE000043001AA04212046FFF742FE04B010BD43
:10ACF000034B40F206420349034807F05DFCF5E7C9
:10AD0000906A0108246C0108F460010810B4002462
:10AD100004604160028143819DF8043003739DF813
:10AD20000830437301238373C4735DF8044B704789
:10AD300008B5D0B10346B1F5803F1DD231B31FFA3B
:10AD400081FC0089604480B2604521D393F90CE016
:10AD5000BEF1000F12DBEAB15A68511A59605A89E4
:10AD600062445A811881002007E00B4B40F2DF1249
:10AD70000A490B4807F020FC012008BD5A68511A07
:10AD800003F110028A42E9D90120F6E70020F4E736
:10AD90000120F2E70120F0E7486C0108587501082E
:10ADA000F4600108F0B583B006460D461446412A0A
:10ADB00001D0012A0FD10820FFF782FC074638B1E5
:10ADC0000023019300942B462A463146FFF79EFF4D
:10ADD000384603B0F0BD044B4FF4A5720349044854
:10ADE00007F0EAFBE7E700BF486C0108786C010850
:10ADF000F460010810B582B084468E461846049966
:10AE00000CF1030C2CF0030C0EEB0C04BDF8143009
:10AE10009C420CD801B16144044602230193009284
:10AE200073467246FFF772FF204602B010BD002441
:10AE3000FAE708B50022FFF77BFF08BD10B590B117
:10AE40000346B1F5803F15D2F9B188B25A898242E2
:10AE500012D35C6821445960121A5A811A89121A55
:10AE60001A81002007E00A4B40F24B2209490A48A8
:10AE700007F0A2FB012010BD054B40F25522074907
:10AE8000054807F099FB0120F5E70020F3E700BF34
:10AE9000486C010858750108F46001088C6C0108C1
:10AEA00008B5002902DBFFF743FF08BD4942FFF761
:10AEB000C5FFFAE708B50122FFF7F2FF08BD000061
:10AEC000F8B510B10446002617E02B4B4FF437724B
:10AED0002A492B4807F070FB00263046F8BD264B68
:10AEE00040F2F1222749264807F066FB0DE023696E
:10AEF000204698470136F6B22C46002CEDD004F0DF
:10AF0000F9F90746A37B002BE9D0A57B013DEDB203
:10AF1000A573384604F0FAF9002DDED12568237BAD
:10AF200003F00F03627B12F0020F0AD02369002B9B
:10AF3000DDD1114B40F2FF221349114807F03CFBD1
:10AF4000D5E7022B06D0012B09D06BB92046FFF7BD
:10AF500023F9CFE721460920FFF7E0FBCAE72146A6
:10AF60000820FFF7DBFBC5E7034B40F20F32074930
:10AF7000034807F021FBBDE7486C0108587501083C
:10AF8000F4600108AC6C0108C46C0108E86C0108AD
:10AF90002DE9F04782B00E469046B2F5C17F45D00C
:10AFA00004460ED8012A02D0412A40F0828042464F
:10AFB00031460020FFF7F6FE8146484602B0BDE864
:10AFC000F087B2F5207F74D1C11C01F4FE71F21C30
:10AFD00093B223F003030B449BB203F1100080B241
:10AFE00022F0030293426ED382426FD8FFF71AFA1F
:10AFF00081460028E1D004F110010144033100230F
:10B000000193CDF800803346324621F00301FFF76B
:10B010007DFED9F8043013F0030FCED02D4B4FF442
:10B0200091722D492D4807F0C7FAC6E7054600275B
:10B03000B94611E0B9F1000F02D04846FFF740FFD2
:10B04000B946BAE7B9F1000F31D0CAF80070341B25
:10B05000A6B20025002EB0D0BA460920FFF730FB7B
:10B0600007460028E6D0EC1C24F00304A4B2C4F583
:10B070001474A4B2B44228BF344605F1100101444F
:10B08000033100230193CDF800802346324621F09E
:10B090000301FFF73BFE7B6813F0030FD2D00D4B8B
:10B0A0004FF480720E490D4807F086FACAE7B94698
:10B0B000CDE7084B40F227120A49084807F07CFA0E
:10B0C0004FF0000979E74FF0000976E74FF00009EB
:10B0D00073E700BF486C0108606D0108F460010867
:10B0E000FC6C01088C6D0108F8B50E460446B8B139
:10B0F0002789B7422ED935466389AB4218D2EB1A5D
:10B100009DB22389F21B134423812468002CF3D1C0
:10B110001A4B40F2AF121A491A4807F04DFAEBE702
:10B12000164B4FF4CC721849164807F045FADFE782
:10B13000227B12F00F0F05D1AB4203D0637B13F0DB
:10B14000020F08D065812581206808B1FFF7B8FE9D
:10B1500000232360F8BD63681B1BE91889B22046F1
:10B16000FFF792F804460028ECD1044B40F2BD12E0
:10B170000649044807F020FAE4E700BF486C0108DC
:10B18000C06D0108F4600108A86D0108D86D0108C0
:10B190000346002002E0013080B21B68002BFAD188
:10B1A0007047000098B110B5044604F0A3F8A37BE3
:10B1B0000133A37304F0AAF8A37B03B110BD044BC1
:10B1C00040F242320349044807F0F6F9F6E77047C7
:10B1D000486C0108F46D0108F460010838B510B13D
:10B1E0000D46044661B9154B40F2593214491548D1
:10B1F00007F0E2F919E023892889034423811446E2
:10B200002268002AF7D1228963899A420ED12368E5
:10B2100033B10A4B40F263320B490A4807F0CCF9CC
:10B2200023892A8913442381256038BD034B40F2CA
:10B2300062320649034807F0BFF9E8E7486C0108A5
:10B24000086E0108F4600108706E0108406E010884
:10B2500010B50C46FFF7C2FF2046FFF7A3FF10BD55
:10B260002DE9F04148B10C46054631B102890B8900
:10B270009A4202D30027B8463AE03A4B40F2C9322C
:10B2800039493A4807F098F96FF00F0068E0354BFC
:10B2900040F2D9323649354807F08EF93CE0314B5F
:10B2A00040F2DA323349314807F086F937E02D6849
:10B2B00015B14FF000083AE014B94FF0000836E03D
:10B2C000284B4FF479722C49284807F075F96FF034
:10B2D0000F0045E023687BB3224B40F2E932274957
:10B2E000224807F069F96FF0050039E0002C36D0EC
:10B2F0006E89A6EB08066389DB1B9E4200D31E46BF
:10B300006868616832463944404407F0F3FAB04453
:10B3100037446B894345BAD36389BB42BFD3638942
:10B32000BB4201D8246800276B894345BFD01CB1BC
:10B33000628923899A42CDD0002DD7D06A892B8982
:10B340009A42D3D12B68002BD0D0064B40F2EE327C
:10B350000A49064807F030F96FF0050000E00020C8
:10B36000BDE8F081486C0108806E0108F4600108B6
:10B37000B06E0108C86E0108E46E0108F46E0108A1
:10B380002DE9F84330B188469146054669B100275A
:10B390003E462AE01B4B40F20A421B491B4807F07D
:10B3A0000BF900273846BDE8F883164B40F20B42F4
:10B3B0001749164807F000F90027F3E76C89E41AEB
:10B3C000A4B2A14500D24C4669682246194408EB54
:10B3D000060007F08FFA2744BFB22644B6B2A9EBA5
:10B3E00004041FFA84F900232D68B9F1000FD9D0A5
:10B3F000002DD7D0002BE1D06A899A42DED89B1A63
:10B400009BB2F1E7486C0108206F0108F460010865
:10B41000406F010838B514460A462189FFF7B8FD88
:10B42000054618B12146FFF71BFF08B9284638BD6D
:10B43000034B40F224520349034807F0BDF8F5E7F7
:10B44000486C0108646F0108F4600108F8B504460F
:10B450000F4616460720FFF733F980B10546002353
:10B4600003608760C6604460104B1A6872B153680D
:10B47000E31A002B0FDA02600C4B1860F8BD0C4B7E
:10B48000BE220C490C4807F097F8F7E71860F5E77B
:10B490002B601560F2E7002AF0D01368002BF7D07C
:10B4A0005968611A0029F3DB1A46F4E734050120D4
:10B4B000786F0108AC6F0108F460010838B50446E4
:10B4C00043689847FBF708F884462568094B1868D5
:10B4D0002844A0EB0C03002B06DA2246064905EBB4
:10B4E0000C00FFF7B3FF38BD22460349FFF7AEFF5C
:10B4F000F9E700BF30050120BDB4000870B504466F
:10B500000D461646B0F1804F07D2FAF7E5FF3246F6
:10B5100029462044FFF79AFF70BD044B40F22912E0
:10B520000349044807F048F8EFE700BF786F0108C7
:10B53000EC6F0108F460010810B5002408E0064B28
:10B5400003EBC402054953F83400FFF7D7FF013479
:10B55000042CF4D910BD00BF38700108BDB4000838
:10B5600070B5FAF7B9FF05460B4B196891B14B68F6
:10B57000EA1A002A0EDB0868074A10608C68CE6859
:10B58000064A13600720FFF7C9F8002CECD03046BC
:10B59000A047E9E770BD00BF340501203005012058
:10B5A00010B50D4B1B6883B1FAF796FF0A4B1B6869
:10B5B0005C68241A0CD4002C0BDA084B4FF4DC72B4
:10B5C0000749084806F0F8FF03E04FF0FF3400E0B9
:10B5D0000024204610BD00BF34050120786F01080B
:10B5E00024700108F46001080020104A1388591CD7
:10B5F00011804FF6FF72934209D00D4B1B6893B137
:10B60000598A0A4A1288914206D0DB68F7E7074B4D
:10B610004FF440421A80F0E7013080B2B0F5804F1D
:10B62000E3D300207047014B1888704724000020A6
:10B6300038050120F8B50E4615460746C8B1FEB1DB
:10B640003C7A3CB11E4B5B6893F840300133DBB26F
:10B650009C4225D1DDB12FB33B682BB3184A526908
:10B66000B2F1FF3F22D0B16853400B4220D00020FE
:10B6700017E0144B87221449144806F09DFFDEE7BB
:10B68000104B88221249114806F096FFD8E78FB177
:10B690003B688BB10A4A526993420FD0284600E0BA
:10B6A0000020F8BD0120FCE70120FAE70120F8E7BF
:10B6B0000120F6E70120F4E70120F2E70120F0E79E
:10B6C00080CC00206070010890700108F4600108CF
:10B6D000B470010808B505F07DFF6FEA80406FEA9D
:10B6E0009040014B188008BD240000202DE9F04F48
:10B6F00083B00F468146D0B107B3B9F80A30072BA3
:10B7000023D9D9F80440534B1968586902F023FF34
:10B7100080462088FEF732FC82466088FEF72EFCC9
:10B7200005464D4B1C684FF0000B5E4619E04B4B35
:10B73000CF224B494B4806F03FFFDDE7474BD02275
:10B740004949484806F038FFD7E74846FFF7B8FBB5
:10B7500003B0BDE8F08FA346A38A534526D0264602
:10B76000E468002C30D0638AAB42F8D142463946B7
:10B770002046FFF75FFF0028F1D0237C13F0040F71
:10B78000EAD1BBF1000FE6D0B8F1000FE4D0314BA5
:10B790005B69B3F1FF3FDFD1DBF800207B689A42A1
:10B7A000DAD022689342D7D1A346D5E763681BB1AC
:10B7B000284A12699342D2D136B1E368F360264B2E
:10B7C0001A68E2601C6011E07CB108214846FFF76E
:10B7D00035FBB0B924B3A569F5B1E069CDF800A097
:10B7E000224B4A462146A847B2E75C46002CECD1E2
:10B7F0007A68184B5B699A42E7D04846FFF760FBCE
:10B80000A6E7164B4FF4B8721949164806F0D4FE55
:10B810004846FFF755FB9BE74846FFF751FB97E784
:10B82000B8F1000F05D10B4B5B6903F0F003E02B7F
:10B8300003D14846FFF744FB8AE7064B9989083154
:10B8400009B24846FFF736FB0321484602F096FC52
:10B85000EFE700BF80CC00203805012060700108B0
:10B86000DC700108F4600108F470010890CC00203D
:10B870001071010870B504460D4621B12CB1254B5D
:10B880001B6819460CE0244DF8E7244B40F2B73210
:10B890002349244806F090FE6FF00F0015E0C968B8
:10B8A00019B1A142FBD1012600E000267AB9FFF7C9
:10B8B0009BFE0246F8B1E5B12B682360628236BB7D
:10B8C000144B1A68E2601C60002070BDDB68002B1E
:10B8D000F1D0A342FAD0598A9142F7D11868296869
:10B8E00088420BD069B17BB10028EFD16FF007001F
:10B8F000EBE70023E1E76FF00700E6E76FF00700F2
:10B90000E3E76FF00700E0E76FF00700DDE70020F6
:10B91000DBE700BF38050120C47A01086070010828
:10B920002C710108F46001082DE9F04F85B0DDF8B5
:10B9300038B0DDF83CA0002845D00C46904699462A
:10B940000646002949D0002A51D0BAF1000F58D03C
:10B95000BBF1000F5FD0428A002A66D022894FF6E1
:10B96000F7739A427FD808212046FFF762FA002831
:10B9700062D125466B89072B6DD96F68708AFEF7F7
:10B98000FDFA38804846FEF7F9FA78800023BB714B
:10B99000FB712889FEF7F2FAB880CDF808B01123C0
:10B9A0000193B37A0093F37A42465146284602F057
:10B9B0003DFD0746A54202D02846FFF781FA3846EA
:10B9C00005B0BDE8F08F2B4B40F2D1222A492B481D
:10B9D00006F0F2FD6FF00F07F1E7264B40F2D2229E
:10B9E0002749264806F0E8FD6FF00F07E7E7214BEF
:10B9F00040F2D3222349214806F0DEFD6FF00F0705
:10BA0000DDE71C4B4FF435721F491C4806F0D4FD8E
:10BA10006FF00F07D3E7174B40F2D5221B491748A9
:10BA200006F0CAFD6FF00F07C9E70146FFF722FFD6
:10BA30000746002892D0C2E74FF420720821222046
:10BA4000FFF7A6FA054688B12389002B92D021463C
:10BA5000FFF7FEFB8EE7074B40F20D320C4907481B
:10BA600006F0AAFD89E74FF0FF37A8E74FF0FF3750
:10BA7000A5E700BF6070010844710108F460010887
:10BA80006471010884710108A8710108CC71010872
:10BA9000F0710108F0B583B0089D90B10446D1B1B2
:10BAA0001AB365B3002834D0066896B306F0F00CDC
:10BAB000BCF1E00F2DD06F68BE422BD06FF00300B9
:10BAC0002DE0184B4FF420721749184806F074FD0A
:10BAD0006FF00F0023E0134B40F28122144913480A
:10BAE00006F06AFD6FF00F0019E00E4B40F2822263
:10BAF00010490E4806F060FD6FF00F000FE0094B93
:10BB000040F283220C49094806F056FD6FF00F0001
:10BB100005E0281D019000952046FFF705FF03B0C2
:10BB2000F0BD00BF6070010820720108F4600108D8
:10BB30003C7201085872010878720108F0B583B0B0
:10BB400098B10D4614461E460746C1B10AB3007AA5
:10BB500048B3FEF7B7FE50B300903346224629465D
:10BB60003846FFF797FF03B0F0BD124B4FF4067253
:10BB70001149124806F020FD6FF00F00F3E70D4B5E
:10BB800040F219220E490D4806F016FD6FF00F0025
:10BB9000E9E7084B40F21A220A49084806F00CFD72
:10BBA0006FF00F00DFE7104602F016FBD3E76FF0EF
:10BBB0000300D8E76070010898720108F46001087A
:10BBC000B0720108CC72010808B528B171B1838A3E
:10BBD000021DFFF7B3FF08BD094B40F2D51209491A
:10BBE000094806F0E9FC6FF00F00F4E7044B4FF44E
:10BBF000EB720649044806F0DFFC6FF00F00EAE73D
:10BC000060700108E8720108F4600108007301081F
:10BC100021B191F840300133037270470023037261
:10BC20007047000070B5A0B10D4616460446D1B16C
:10BC3000428A12B32B686360A682237C43F004031C
:10BC40002374144B1A681346EBB1A34220D0DB686F
:10BC5000FAE7114B40F235421049114806F0ACFCAE
:10BC60006FF00F0013E00C4B40F236420D490C48C8
:10BC700006F0A2FC6FF00F0009E00146FFF7FAFDA5
:10BC80000028D7D003E0E260024B1C60002070BDAA
:10BC90000020FCE7380501206070010818730108D6
:10BCA000F46001083473010808B510B18161C26104
:10BCB00008BD044B40F28A420349044806F07CFC6C
:10BCC000F6E700BF6070010850730108F4600108D6
:10BCD00008B550B101460F4B1A68824211D1D268A3
:10BCE0001A600020FEF71AFD08BD0B4B40F2A1427E
:10BCF0000A490B4806F060FCF6E7CB68D360F0E732
:10BD00001A46002AEDD0D368002BF9D08B42F4D02C
:10BD10001A46F6E7380501206070010868730108CB
:10BD2000F460010810B50020FEF7CAFC044628B1F3
:10BD30002022002106F0EAFCFF23E372204610BD1A
:10BD400008B5FFF7EFFF08BDB8B102460368A3B11D
:10BD500099B10B688BB1094B1B686BB110B401E052
:10BD6000DB6833B110681C688442F9D10868186038
:10BD7000F6E75DF8044B70477047704738050120BF
:10BD8000C16A01230B7100234B7190F83B2090F89E
:10BD900039301B0443EA026390F8382043EA022357
:10BDA00090F83A201343C26A8AB1527A1344094A7E
:10BDB000A2FB0302D20802EB8202A3EB4202CA807A
:10BDC0004B7A0A2B02D94FF41673CB8070470022AE
:10BDD000ECE700BFCDCCCCCC10B582B04FF6FF73F2
:10BDE0000193002400946B4601AAC16AFEF7E0FDAE
:10BDF000204602B010BD000038B50D46C46A90F868
:10BE00003A3090F83B2043EA022314481844FEF7E6
:10BE1000BAF8FEF7B8F8647A0444A4B244F02944AE
:10BE200044F47E040E4B9C420BD804F57E440D4B2B
:10BE30002344B3F57E4F0AD22046FEF7A4F82860CB
:10BE400038BD094B9C42F2D9A4F57E44EFE7074B7D
:10BE5000BC220749074806F0AFFBEDE70001FEA949
:10BE6000FF00FEA900FF0156FFFEFEA98073010836
:10BE7000B8730108F460010808B5C16A01F04EFE0C
:10BE800008BD08B5011D01F049FE08BD38B5C56AF9
:10BE900090F83D3013F0010F15D0044614490B46BD
:10BEA0000A46FEF785FDC5B100232B71EB806B714F
:10BEB0002B602B7229462046FFF79EFF2046FFF796
:10BEC0005FFF002038BD0B4B40F205120A490B48BA
:10BED00006F072FB6FF00F00F4E70C210120FEF773
:10BEE0005FFB054608B1E062E4E74FF0FF30E9E7A9
:10BEF000C47A010880730108D4730108F460010852
:10BF000008B5C26A537A01335372FFF7BFFF08BD09
:10BF100010B5C46A237A13B1FFF7F2FF10BDFFF723
:10BF2000B0FF64232372F9E708B5C36A0BB11B792C
:10BF300003B908BDFFF724FFFBE7000008B5C36A9B
:10BF400033B100221A7182884FF6A9639A4201D058
:10BF5000002008BD02490B460A46FEF729FDF7E717
:10BF6000C47A010838B5344B1D6805E02379012BEC
:10BF700011D0022B4AD02D68002D5BD0EC6A002C2A
:10BF8000F9D0237A0BB1013B2372E388002BEDD06B
:10BF9000013BE380EAE7E388002BECD16379022BD5
:10BFA00009D9022323712846FFF716FF0123637185
:10BFB0001423E380DFE72846FFF75EFF6379013350
:10BFC000DBB26371032B1CD095F83B3095F8392018
:10BFD000120442EA036295F8383042EA032295F8E7
:10BFE0003A301A43EB6A7BB15B7A1A44134BA3FBDA
:10BFF0000213DB0803EB83035900531A0A33E3806F
:10C00000B9E71423E380B6E70023EEE7E388002BCB
:10C01000B1D12846FFF735FF1423E380637901335C
:10C02000DBB26371012BA6D9032323710023637153
:10C03000E380A0E738BD00BF28050120CDCCCCCCE3
:10C04000C36A002B33D010B582B004461A797AB196
:10C05000D0F836000090628FADF80420D1F80E20A1
:10C06000D1F818C01879012804D01B68934213D066
:10C0700002B010BD1B6893420AD0002AF8D1634574
:10C08000F6D106220831684606F016FB0028EFD0EC
:10C090002046FFF735FFEBE706220831684606F039
:10C0A0000BFB0028E4D02046FFF732FFE0E77047A3
:10C0B000C36A2BB10A681B689A4203D000207047FC
:10C0C000002070470120704743798B4203D04171B3
:10C0D000002383714381704770B504460D461646B0
:10C0E000831C442B07D8631C9BB2320A2A55A01C20
:10C0F000EE5480B270BD044B40F2AE520349044886
:10C1000006F05AFAEFE700BFF8730108307401082F
:10C11000F4600108F8B504460D4617461E46034470
:10C120000233442B06D8631C9BB22F55A01CEE543F
:10C1300080B2F8BD034B40F29A520349034806F01F
:10C140003BFAF0E7F87301086C740108F460010829
:10C1500070B504460D461646432803D8601C2E557C
:10C1600080B270BD034B40F2A6520349034806F06B
:10C1700023FAF3E7F8730108B0740108F4600108CA
:10C1800070B504460D461646031D442B11D8631C9A
:10C190009BB2320E2A55A21C92B2C6F30741E95453
:10C1A000E31C9BB2C6F30721A954201DEE5480B2B4
:10C1B00070BD044B40F2B7520349044806F0FCF945
:10C1C000E5E700BFF8730108E8740108F4600108AE
:10C1D0002DE9F8438046002841D0894615461E4681
:10C1E000002945D04FF420724FF49A713620FEF7A3
:10C1F000CFFE0746002879D04389B3F59A7F40D314
:10C20000032D46D099F80630002B47D0394B1B68D8
:10C21000C9F800307C684FF49A720021204606F07D
:10C2200075FA01232370637098F83C30A370D9F835
:10C230000000FDF7A8FE6060082D0BD0042D09D08A
:10C24000072D07D0032D08D199F80530043BDBB248
:10C25000012B02D8D8F80430E36000202BE0264BF5
:10C2600040F269722549264806F0A6F947463DE0A6
:10C27000214B40F26A722349214806F09DF94F464E
:10C2800034E01D4B40F271721F491D4806F094F9CD
:10C29000B6E799F80530032BBCD1B3E705F09AF95E
:10C2A000144B1860B2E708EB000393F836302118FE
:10C2B0000B77013080B20528F5D9632384F8EC3080
:10C2C0006FF07D0284F8ED20532284F8EE2084F88C
:10C2D000EF30F0340123352221460020FFF71AFF0A
:10C2E0002A462146FFF734FF06B130803846BDE8C4
:10C2F000F88300BF3C050120F8730108247501088C
:10C30000F4600108447501086475010810B5846A79
:10C310000023236263621A4BDB7813B1194BDB688D
:10C32000A362174B1B799BB1164B1B69E362144B3D
:10C330005B798BB1134B5B6923630B69E361104B32
:10C340009B797BB9002323720D4BDB7993B910BD28
:10C35000A36A5B08E362EAE7A36AC3EBC303DB08F3
:10C360002363EAE7074B9869FDF70DFE206201237E
:10C370002372E9E7034BD869FDF705FE6062E6E743
:10C3800048050120500501202DE9F0410646156BB6
:10C390008DB388462846F3F76BFF044658B3C6F1C1
:10C3A0004107B8420CD8BC4228BF3C46FF2C0FD8EE
:10C3B000E3B20C2241463046FFF7ACFE064617E0DA
:10C3C0000E4B40F2CB520E490E4806F0F5F8EAE764
:10C3D0000A4B40F2CD520A490A4806F0EDF8E7E769
:10C3E00015F8012B41463046FFF7B2FE06463C46A3
:10C3F000671E002CF4D13046BDE8F081F8730108C7
:10C40000A4750108F460010808B5844610460CF1D3
:10C4100001039BB2FF2201F80C2007E003F1010C9D
:10C420004FF0000E01F803E01FFA8CF3432BF5D90F
:10C4300003F1F00189B2FEF757FE08BD2DE9F04186
:10C4400084B00746856A04212846FFF73DFE0DF1BA
:10C450000E03032229463846FFF7BAFE00284ED0C5
:10C4600080464668F036022339223146BDF80E0078
:10C47000FFF750FEADF80E00BA8E3146FFF72CFEE6
:10C48000ADF80E00032337223146FFF743FEADF827
:10C490000E0000240AE0234B1A5D3146BDF80E0061
:10C4A000FFF756FEADF80E000134E4B2022CF2D9CB
:10C4B0003A463146BDF80E00FFF766FFADF80E00B4
:10C4C00042463146FFF7A0FF00974323164A4146F4
:10C4D00016480068FFF7DEFA04464046FEF7F0FC17
:10C4E000AB79FF2B01D00133AB71AB79092B09D8A4
:10C4F000C3EB431203EB8203DB009BB204E04FF07B
:10C50000FF34EDE742F2107303F2F313084A82FBA3
:10C510000312DB17C3EB62136B81204604B0BDE846
:10C52000F08100BF58770108C07A01084405012056
:10C53000D34D621010B5846A6379012B05D00A2BA4
:10C5400003D0052B01D0042B0BD1FFF777FFE38A33
:10C55000A28A9B1A012B04DD03EBD373C3F34F03B1
:10C56000638210BD2DE9F04184B00746856A03213E
:10C570002846FFF7A9FD0DF10E0303222946384690
:10C58000FFF726FE002861D080464668F036022379
:10C5900039223146BDF80E00FFF7BCFDADF80E00A4
:10C5A0004FF410723146FFF797FDADF80E000423EB
:10C5B00032223146FFF7AEFD0446ADF80E00E869C1
:10C5C000FDF7E1FC024631462046FFF7D9FDADF804
:10C5D0000E00032337223146FFF79CFDADF80E0015
:10C5E00000240AE0224B1A5D3146BDF80E00FFF729
:10C5F000AFFDADF80E000134E4B2022CF2D93A4698
:10C600003146BDF80E00FFF7BFFEADF80E00424602
:10C610003146FFF7F9FE00974323164A4146164874
:10C620000068FFF737FA04464046FEF749FCAB794D
:10C63000FF2B01D00133AB71AB79092B09D8C3EBC8
:10C64000431203EB8203DB009BB204E04FF0FF34A4
:10C65000EDE742F2107303F2F313084A82FB031270
:10C66000DB17C3EB62136B81204604B0BDE8F08199
:10C6700058770108C07A010844050120D34D6210A3
:10C680002DE9F04184B0002850D00746846A002C80
:10C6900056D001212046FFF717FD0DF10E030322AE
:10C6A00021463846FFF794FD8046002800F096802A
:10C6B0004668F036022339223146BDF80E00FFF7F6
:10C6C00029FDADF80E00BA8E3146FFF705FDADF835
:10C6D0000E00042332223146FFF71CFD0546ADF85B
:10C6E0000E00E069FDF74FFC024631462846FFF791
:10C6F00047FDADF80E00042336223146FFF70AFD50
:10C700000546ADF80E00A069FDF73DFC0246314636
:10C710002846FFF735FDADF80E00032337223146DA
:10C72000FFF7F8FCADF80E0000251EE02E4B40F29E
:10C7300077122E492E4805F03FFF6FF00F0549E0B4
:10C74000294B40F279122B49294805F035FF6FF04B
:10C7500005053FE0284B5A5D3146BDF80E00FFF756
:10C76000F7FCADF80E000135EDB2022DF2D93A46D4
:10C770003146BDF80E00FFF707FEADF80E00424649
:10C780003146FFF741FE1D4B0193009743231C4A9E
:10C7900041461C480068FFF7C7F805464046FEF7CB
:10C7A0008FFBA379FF2B01D00133A371A279052A56
:10C7B00017D801239340C3EB431203EB8203DB0042
:10C7C0009BB203F2F313104A82FB0312DB17C3EB95
:10C7D00062136381284604B0BDE8F0814FF0FF3555
:10C7E000DFE74EF66023ECE7F8730108C075010837
:10C7F000F4600108DC75010858770108C47A010863
:10C80000C07A010844050120D34D621070B5866AD4
:10C81000094B9B7803B970BD04460D460023738114
:10C82000064B9868FDF7AFFBB0612B69F3612046BA
:10C83000FFF726FFEFE700BF480501205005012064
:10C840002DE9F04184B00546846A0C212046FFF7AB
:10C850003BFC0DF10E03042221462846FFF7B8FCED
:10C8600098B307464668F036042332223146BDF8B5
:10C870000E00FFF74FFC8046ADF80E00E069FDF7B3
:10C8800082FB024631464046FFF77AFCADF80E00C7
:10C890003A463146FFF7B8FD0D4B0193009543230F
:10C8A0000C4A39460C480068FFF73EF80546384602
:10C8B000FEF706FBA379FF2B01D00133A3711423EC
:10C8C0006381284604B0BDE8F0814FF0FF35F1E701
:10C8D000C47A0108C07A01084405012038B505462C
:10C8E000846A08212046FFF7EFFB002204F11C01B7
:10C8F000284601F0CBF9A379FF2B01D00133A371B6
:10C900000123638138BD000030B583B0002868D0B2
:10C910000546846A002C6CD00023A382A26AB2F17F
:10C92000FF3F0FD01E32A3F17733A3FB02135B0945
:10C93000B2F5701F01D34FF6FF739BB2E3820BB9C0
:10C940000123E382E26AB2F1FF3F10D01E32394B7D
:10C95000A3FB02135B09B2F5701F01D34FF6FF73FF
:10C960009BB2A3810BB90123A381A3892382226BEC
:10C97000B2F1FF3F10D01E322E4BA3FB02135B0916
:10C98000B2F5701F01D34FF6FF739BB2E3810BB971
:10C990000123E381E3896382A289E3899A4202D376
:10C9A0000BB10023A381237A5BB3236A0193636AEB
:10C9B000009333B9E369019A1340009343F0807305
:10C9C0000093E379012B2ED00A212046FFF77CFB50
:10C9D0006B4601AA04F11C012846FDF7E9FF03B0EC
:10C9E00030BD154B40F215421449154805F0E4FDE1
:10C9F000F5E7114B40F217421249114805F0DCFDF2
:10CA0000EDE7227F94F91C30002B02DBFF2301931A
:10CA1000CDE7BF2A03D96FF07F430193C7E74FF6F5
:10CA2000FF730193C3E72846FFF788FA0023E371F9
:10CA3000CAE700BF89888888F8730108F87501087B
:10CA4000F4600108147601082DE9F04184B006462F
:10CA5000846A0023E36106212046FFF735FB0DF1D0
:10CA60000E03012221463046FFF7B2FB00283AD0E0
:10CA700080464768F037022339223946BDF80E0058
:10CA8000FFF748FBADF80E00B28E3946FFF724FBE6
:10CA9000ADF80E00032337223946FFF73BFBADF814
:10CAA0000E0000250AE0244B5A5D3946BDF80E0001
:10CAB000FFF74EFBADF80E000135EDB2022DF2D9B5
:10CAC00042463946BDF80E00FFF79EFC1B4B019312
:10CAD000009643231A4A41461A480068FEF724FF8D
:10CAE0004046FEF7EDF9A379FF2B01D00133A37186
:10CAF000E379BBB1A279052A1AD801239340C3EB8D
:10CB0000431203EB8203DB009BB203F2F3130E4AE2
:10CB100082FB0312DB17C3EB62136381002004B0B6
:10CB2000BDE8F0810123E3713046FFF7AFF9E1E79B
:10CB30004EF66023E9E700BF58770108C47A010880
:10CB4000C07A010844050120D34D621010B5044697
:10CB50000C21806AFFF7B8FA04490B460A462046C2
:10CB6000FDF726FF2046FFF76FFF10BDC47A0108CE
:10CB700010B50C4B1B7833B10A4A1378013BDBB27A
:10CB800013703BB110BD084BFF220849084805F05F
:10CB900013FDF1E7074C2068FFF79AF800232360A4
:10CBA000F0E700BF40050120F87301082C7601086A
:10CBB000F46001084405012038B5174B1B780BBB06
:10CBC000164B1B682BB1164BE5221649164805F08B
:10CBD000F3FCFFF7A7F8114B1860C8B1437A43F094
:10CBE00020034372114D44222946FEF743FE0B4CAD
:10CBF000432229462068FFF715F800220C492068D7
:10CC0000FFF752F8044A137801331370002038BD3F
:10CC10004FF0FF30FBE700BF400501204405012035
:10CC2000F873010850760108F4600108C47A01081D
:10CC3000BDD00008BF4B00221A605A6043892B2BDD
:10CC400040F21A822DE9F04F87B08246048990465F
:10CC5000F027554604E0FF1ABFB2E41AA4B22D68CB
:10CC6000002D00F00C826B89BB42F4D96B680193F4
:10CC70003E46BB46CDF80880B0E02A6812B1526843
:10CC80001278C7E00022C5E00F460A464FF0FF3990
:10CC90008FE0042A03D117464FF0060989E0A64B1E
:10CCA00040F22E62A549A64805F086FC6FF005000B
:10CCB000E7E1032A03D94FF00709042779E09E4BE7
:10CCC00040F233629F499E4805F076FC6FF0050004
:10CCD000D7E1042A03D117464FF0030969E0964BC8
:10CCE00040F241629549964805F066FC6FF00500F8
:10CCF000C7E1012A06D1BBF1F00F0DD117464FF065
:10CD0000000956E08C4B40F24F628F498C4805F089
:10CD100053FC6FF00500B4E1874B40F251628B4940
:10CD2000874805F049FC6FF00500AAE1012A03D10C
:10CD300017464FF001093CE07F4B40F255628249B3
:10CD40007F4805F039FC6FF005009AE1042A03D111
:10CD500017464FF002092CE0774B40F259627749B1
:10CD6000774805F029FC6FF005008AE1042A03D119
:10CD700017464FF004091CE06F4B40F25D626F49AB
:10CD80006F4805F019FC6FF005007AE1042A03D121
:10CD900017464FF005090CE0674B40F261626749A6
:10CDA000674805F009FC6FF005006AE14FF0FF39B4
:10CDB0000027002940F0AC800136B6B26B89B3423F
:10CDC0000CD8F61AB6B2E31A9CB2A64280F0628181
:10CDD0002D68002D00F024816B680193002D00F078
:10CDE0002981A64280F026813746019B995DFF2963
:10CDF00000F02081B31C1FFA83F8464500F24481FD
:10CE00003046721CB5F80AC06245BFF636AF01372E
:10CE1000019BDA5D3B29C9D801A757F821F000BF73
:10CE200089CC000893CC0008ADCD0008B3CC000835
:10CE3000ADCD0008ADCD0008ADCD0008ADCD0008EA
:10CE4000ADCD0008ADCD0008ADCD0008ADCD0008DA
:10CE5000ADCD0008ADCD0008ADCD0008ADCD0008CA
:10CE6000ADCD0008ADCD0008ADCD0008ADCD0008BA
:10CE7000ADCD0008ADCD0008ADCD0008ADCD0008AA
:10CE8000ADCD0008ADCD0008ADCD0008ADCD00089A
:10CE9000ADCD0008ADCD0008ADCD0008ADCD00088A
:10CEA000ADCD0008ADCD0008ADCD0008ADCD00087A
:10CEB000ADCD0008ADCD0008ADCD0008ADCD00086A
:10CEC000ADCD0008ADCD0008ADCD0008ADCD00085A
:10CED000ADCD0008ADCD0008ADCD0008ADCD00084A
:10CEE000ADCD0008ADCD0008ADCD0008D3CC000815
:10CEF000F3CC00082DCD00084DCD0008ADCD0008C5
:10CF0000ADCD0008ADCD00086DCD00088DCD000879
:10CF100010444FF6FD71884200F3B980324492B25A
:10CF2000023296B2002F3FF449AF002205920396D9
:10CF300039E000BF48050120F87301087876010840
:10CF4000F46001088476010898760108A476010847
:10CF5000524B13F80930002B60D13E46042F28BFF6
:10CF60000426F6B24346324605A92846FEF708FADB
:10CF7000B0424DD1042F2BD917F0030F1ED1474BD0
:10CF8000012203F809200598FCF7FDFF444B43F804
:10CF90002900043FFFB208F104039BB298453AD838
:10CFA00009F101099846B9F1070FD1D93D4B4FF46A
:10CFB000CF623D493D4805F0FFFAC9E7394B40F2E1
:10CFC00081623B49394805F0F7FA6FF0050058E0F7
:10CFD000039E042F0DD0012F10D19DF8143005931E
:10CFE0002E4B012203F809202D4B059A43F82920E6
:10CFF000E4E60598FCF7C7FF0590F1E7294B4FF4ED
:10D00000D2622C49294805F0D7FA6FF0050038E0C4
:10D010006FF0010035E06FF0010032E0039ECDE6D5
:10D02000204B40F29D622449204805F0C5FA6FF07C
:10D03000050026E0DDF80880184B1B7853B1184B2B
:10D040001B68164A00211170012B12D0022B09D047
:10D05000032B0CD0B8F1000F07D04FF000086C2460
:10D060002C27F6E54FF00108F4E7002009E04FF027
:10D070000108EC246C27ECE56FF0010070476FF0BD
:10D08000010007B0BDE8F08F6FF00100F9E76FF025
:10D090000100F6E76FF00100F3E700BF480501204B
:10D0A00050050120F8730108BC760108F4600108FE
:10D0B000D0760108E8760108FC76010870B51446C0
:10D0C000364B5D68AE6A5268F6B13379E3B1638975
:10D0D0002B2B19D91378022B16D1002395F83C106D
:10D0E00099420BD9052B09D8E91891F83600D118C7
:10D0F000097F884208D10133DBB2EFE75068FCF7C3
:10D1000042FF3368984203D02046FDF7D9FE70BD38
:10D1100031462046FFF78EFD0028F5D1204B5B7885
:10D12000002BF1D061681F4B1B79052B0AD0062B11
:10D1300026D0022BE8D17379062BE5D12846FFF7DC
:10D1400065FBE1E77379012B0AD0033BDBB2022BCD
:10D15000DAD82846FFF7DAF82846FFF7D5FBD3E7F9
:10D160002846FFF7D3F895F83D3013F0080F03D0A9
:10D170002846FFF7B3FBC7E72846FFF7C5FBC3E721
:10D180007279032A05D0012A03D0042A01D0052A86
:10D19000CFD12846FFF7DAFCB6E700BF80CC0020ED
:10D1A000480501205005012038B5856A35B104468F
:10D1B0006B79052B03D8032B03D243B938BD0A2B57
:10D1C00005D10023AB712046FFF7CCF9F6E70C2B15
:10D1D00008D8EB79012B0DD00023AB712046FFF767
:10D1E00033FCEBE7064B40F26D320649064805F08A
:10D1F000E3F9EEE72046FEF7A1FE0023EB71EBE733
:10D20000F873010844770108F460010808B530B1EB
:10D210000246836A13B15879082808D008BD084B24
:10D2200040F28B320749084805F0C6F9F6E709686D
:10D23000DB699942F2D11046FFF702FBEEE700BF2F
:10D24000F8730108E4600108F46001082DE9F04179
:10D2500084B00746856A05212846FEF735FF0DF1A3
:10D260000E03032229463846FEF7B2FF00284FD0AE
:10D2700080464668F036022339223146BDF80E005A
:10D28000FEF748FFADF80E00BA8E3146FEF724FFD8
:10D29000ADF80E00032337223146FEF73BFFADF811
:10D2A0000E0000240AE0234B1A5D3146BDF80E0043
:10D2B000FEF74EFFADF80E000134E4B2022CF2D9B5
:10D2C0003A463146BDF80E00FFF75EF8ADF80E00A5
:10D2D00042463146FFF798F80097432305F11802BC
:10D2E000414615480068FEF7D5FB04464046FDF769
:10D2F000E7FDAB79FF2B01D00133AB71AB79092B83
:10D3000009D8C3EB431203EB82031B019BB204E079
:10D310004FF0FF34EDE744F6206303F2F313074ABE
:10D3200082FB0312DB17C3EB62136B81204604B050
:10D33000BDE8F0815877010844050120D34D621003
:10D3400010B5846A6379012B03D00A2B01D0052B19
:10D350000BD1FFF77BFFE389A28A9B1A012B04DD27
:10D3600003EBD373C3F34F03238210BD88B1836AE9
:10D370008BB15B790A2B07D0052B08D0042B01D089
:10D38000002002E0012000E00120C0B2704701202F
:10D39000FBE7002070470020704700002DE9F041B6
:10D3A00084B0846A1CB30546637903B3A36903930D
:10D3B0000023A361E361236263622363E362A362E8
:10D3C000E382A38263822382FFF7D0FF90B92749CB
:10D3D0000B460A462846FDF7EBFAE379012B39D0D4
:10D3E00000212046FEF770FE2379002B38D104B0CF
:10D3F000BDE8F0810DF10A03072221462846FEF719
:10D40000E7FE07460028E2D04668F03604233622BD
:10D410003146BDF80A00FEF77DFE8046ADF80A00F1
:10D420000398FCF7B0FD024631464046FEF7A8FEE1
:10D43000ADF80A003A463146FEF7E6FF0095432371
:10D4400003AA39460A480068FEF724FB3846FDF770
:10D4500037FDBCE72846FEF771FD0023E371BFE707
:10D46000FFF786FB00232371C1E700BFC47A0108E0
:10D470004405012070B528B3044690F83D3013F000
:10D48000010F29D0856A838EB3F5107F43D36DB326
:10D490002B7993BB34220021284605F037F9FFF79A
:10D4A0008BFB064600283CD101232B7194F83D30BC
:10D4B00013F0040F24D02046FFF7C6FA064620BB1F
:10D4C000304670BD184B40F2E7221849184805F065
:10D4D00073F86FF00F06F3E7134B4FF43A721549E8
:10D4E000134805F069F86FF00F06E9E73420FCF700
:10D4F00099FF054690B1A062CCE7FFF739FBC9E779
:10D5000002212846FEF7E0FDDAE72046FFF746FF56
:10D510004FF0FF36D4E74FF0FF36D1E74FF0FF363C
:10D52000CEE74FF0FF36CBE7F8730108E46001085F
:10D53000F4600108D473010810B5174B1C6806E0AD
:10D540002046FFF72BFF2046FFF794FF246814B313
:10D55000A36A002BFAD05A79002AF7D0D98A29B1C8
:10D560009A8A013292B29A829142E9D05A8A1AB1C9
:10D57000511E5982012A0AD01A8A002AE6D0511E69
:10D580001982012AE2D12046FFF7DAFEDEE72046C3
:10D59000FEF7D0FFDAE710BD2805012010B50446DC
:10D5A000826A53790C2B08D0013B072B08D8DFE89F
:10D5B00003F008071D07070407142046FFF744FA85
:10D5C00010BD9379052B02D8FFF75AF8F8E7FFF75B
:10D5D000E5FE2046FFF74EFFF2E79379012B02D9D3
:10D5E000FFF792F9ECE7FFF779F9E9E79379012B77
:10D5F00002D9FFF729FAE3E7FEF7B4FFE0E70000FE
:10D6000010B50B4B1C6802E0012A0AD0246874B1E3
:10D61000A36A002BFAD05A89012AF5D9013A5A8116
:10D62000F4E7013A5A812046FFF7B8FFEEE710BD54
:10D630002805012008B5FFF7B1FE08BD10B5044666
:10D6400000EB4002094B53F8320038B1FDF738FCCB
:10D6500004EB4403DB00054A0021D15004EB4404F1
:10D66000024B03EBC40300221A7510BD74050120A0
:10D670002DE9F04F85B0064617464FF00009CDF86A
:10D680000890CB464FF00A0A4B465546D046CDF897
:10D690000CA0019103E078B91D4601331BB2092BA0
:10D6A0004BDC1C4603EB4300564A02EBC002107DE4
:10D6B0000A2DF0D00028F0D04EB104EB440E514AB0
:10D6C00002EBCE0CDCF80420316891420ED0012828
:10D6D00017D00128E1D904EB44044A4A02EBC40202
:10D6E000528A4A45D9D391469846D6E7002F00F092
:10D6F0008180444A02EBCE029268BA42E7D11D46CD
:10D7000052E004EB44023F4850F832204AB104EBA7
:10D71000440400EBC402528A5A45BED393469A464B
:10D72000BBE704EB4404374A02EBC402528A029975
:10D730008A42B2D302920393AFE7019911F0020F2C
:10D740005AD10A2D34D0092D16DDB8F1090F35DC78
:10D7500008EB48032B4A52F83330002B36D02A4BC3
:10D7600040F26D1229492A4804F026FF4546284612
:10D77000FFF764FF092D2DDC2C4605EB4502214BFC
:10D7800003EBC2031B7D6BBB36B1316804EB440273
:10D790001C4B03EBC20359601A4B04EB440203EB2E
:10D7A000C202002151829760284605B0BDE8F08F83
:10D7B00011F0010FC7D14FF0FF35F5E7039B092B9F
:10D7C00006DDBAF1090F1ADC5546D0E74546CEE72B
:10D7D000039DCCE70C4B40F283120E490C4804F039
:10D7E000EBFEC9E7084B4FF4C2720B49084804F03E
:10D7F000E3FEC9E71D46D7E74FF0FF35D4E74FF00A
:10D80000FF35D1E7740501205C77010894770108A2
:10D81000F4600108AC770108C0770108F0B583B067
:10D8200005460C4616461F4690F83C20062A3DD178
:10D83000002C43D02068002840D0294600F08BFE01
:10D8400000283BD1226802F0F002E02A36D02A46B6
:10D8500039462046FFF70CFFB0F1000C31DB1C4BC2
:10D860000CEB4C0003EBC002022111759560C10066
:10D870000831194434684C60B4880C81002151820D
:10D8800053F830700FB3C3000C46114AD1504FF417
:10D8900000630093334605F136023946284601F00D
:10D8A00015FC3846FDF70CFB20460CE0094B40F216
:10D8B000A9120949094804F07FFEB9E76FF00F008B
:10D8C00001E04FFA8CF003B0F0BD0020FBE700BF91
:10D8D000740501205C770108EC770108F460010809
:10D8E0002DE9F04F83B00F4690461D46DDF830A07D
:10D8F000DDF834B08146002848D04FF420721C2156
:10D900000E20FDF745FB0646002861D043891B2BFE
:10D9100044D97468BDF83C00FCF730FBE08099F80E
:10D920003C30062B42D12B68A360AB88A381DBF887
:10D930000030C4F81230BBF80430E382DAF800306B
:10D94000C4F80E300E9B1B68A361002323700122D4
:10D9500062700822A270E3700623237104236371AE
:10D96000BAF800204FF6A9639A4227D040F6060382
:10D97000009343463A463146484601F0A7FB3046FD
:10D98000FDF79EFA002003B0BDE8F08F124B40F285
:10D9900057421249124804F00FFEAEE70E4B40F218
:10D9A000624210490E4804F007FEB2E70A4B40F20B
:10D9B00069420D490A4804F0FFFDB4E740F606034A
:10D9C00000930A4B3A463146484601F07FFBD6E7C2
:10D9D0004FF0FF30D7E700BF5C770108E460010833
:10D9E000F46001081078010844780108247D0108DA
:10D9F00030B585B000F13603041D01250395029171
:10DA00000349019100941946FFF76AFF05B030BD44
:10DA10001C7D010838B50546002400E00134092CBE
:10DA200011DC04EB4402084B03EBC2031B7D002B0B
:10DA3000F4D0054B03EBC2039B68AB42EED120460A
:10DA4000FFF7FCFDEAE738BD740501202DE9F04140
:10DA500086B0A9B104460E4645682B88B3F5807F91
:10DA600008D12B79062B05D16B79042B02D16B8859
:10DA7000082B0DD02046FDF723FA06B0BDE8F08153
:10DA8000234B40F28A222349234804F095FDF4E712
:10DA900029463046FEF7D4FAD5F80E300593AA6928
:10DAA000776897B905F108080223424605A9304670
:10DAB000FFF7B4FEEB88B3F5807F11D0B3F5007F9C
:10DAC00020D02046FDF7FCF9D7E7974214BF002786
:10DAD000012705F108080FB10123E6E70223E4E777
:10DAE000002FEED006F13601331D0222039205AA63
:10DAF0000292CDF8048000930B4642463046FFF771
:10DB0000EFFEDEE705A93046FFF780FBD9E700BF4F
:10DB10005C770108E4600108F460010808B5024A76
:10DB2000FFF766FF08BD00BF247D010810B5002483
:10DB300005E0042B1BD92046FFF780FD0134092C9A
:10DB400035DC04EB4403DA00194B13441A7D002A38
:10DB5000F4D004EB4401CB00154919444B8A01333E
:10DB60009BB24B82B3F5967FE5D2012AE1D0032A1E
:10DB70000DD0042A13D0012AE0D104EB4402D300D3
:10DB80000B4A1344191D9868FFF7C8FFD6E704EB4A
:10DB90004403DA00064B134404221A75CEE704EB63
:10DBA0004403DA00024B134402221A75C6E710BD83
:10DBB0007405012070B582B005460E46144602EB8E
:10DBC00042022E4B03EBC2031B7D012B19D904EB40
:10DBD00044022A4B03EBC2031B7D022B19D004EB3A
:10DBE0004403DB000833254A13444FF400620092DB
:10DBF000043305F136023146284601F067FA02B0D7
:10DC000070BD1F4B40F2EE221E491F4804F0D4FCA9
:10DC1000DDE71A4B03EBC2035B8AB3F58E7F1BD89B
:10DC2000B3F5877FDBD304EB4401144B03EBC10155
:10DC300004EB4402D20008321A440432043128466C
:10DC4000FFF7D6FE0028CAD104EB44020B4B03EBCE
:10DC5000C20303221A75C2E7084901EBC20104316D
:10DC60002846FFF75BFF0028B9D104EB4402034BC1
:10DC700003EBC20303221A75B1E700BF740501204C
:10DC80005C770108A8780108F46001082DE9F043E9
:10DC900083B005468846164600F136070146D8F897
:10DCA000000000F058FC002840F09F80D8F80030B9
:10DCB00003F0F002E02A00F09B80002B00F09B8034
:10DCC0002A4601214046FFF7D3FC041E13DBA3B212
:10DCD0007E2B12D8E4B204EB44024A4B03EBC2039E
:10DCE0001B7D93B9474B03EBC2034FF0010983F847
:10DCF00014909D600BE060B240E0434B40F2C132B3
:10DD00004249434804F058FCE4E74FF0000904EBB3
:10DD100044023C4B03EBC2031B7D8BB1B9F1000FF6
:10DD200016D1AEB14FF0FF3004EB4402354B03EB9C
:10DD3000C2031B7D012B12D8012B1FD135462CE0CD
:10DD4000314B40F2CD323349314804F035FCE5E740
:10DD500041462846FFF7E2FE002EE5D10EE02E4BAD
:10DD60001C70D3000833274A13444FF4006200921A
:10DD700004333A463146284601F0A8F903B0BDE81D
:10DD8000F083214B40F2F1322449214804F014FC85
:10DD90002B7B13F0400F22D12D683DB16A892B896E
:10DDA0009A42F5D12B68002BEBD1F1E70023C3B1E8
:10DDB00032464FF420710E20FDF72CFB0646EEB1E3
:10DDC00004EB44030F4A52F8330008B1FDF778F82A
:10DDD00004EB44040B4B43F834600020CEE70123EE
:10DDE000E5E73046FDF7DEF9E9E76FF00F00C5E73C
:10DDF0006FF00F00C2E76FF00F00BFE74FF0FF308A
:10DE0000BCE700BF740501205C770108D8780108E1
:10DE1000F4600108E8780108700501201079010814
:10DE200070B584B00E4614460546002842D0002E38
:10DE300048D0002C4ED02946206800F08CFB0346C9
:10DE4000002840F08680226802F0F001E02949D0E5
:10DE50006968A868514001420ED092B24FF6A9619C
:10DE60008A4209D07268D26892B28A4204D0EA68C3
:10DE7000002A7AD005F10C043D4A127802EB4200E8
:10DE80003C4901EBC001097D012943D9394901EB26
:10DE9000C0018968A9423DD1206802EB420C354996
:10DEA00001EBCC014968884234D131462846FFF75E
:10DEB00081FE58E0304B40F21E323049304804F0C9
:10DEC0007BFBB4E72C4B40F21F322E492C4804F068
:10DED00073FBAEE7284B4FF448722B49284804F0F7
:10DEE0006BFBA8E701238DF8083000238DF809307B
:10DEF0005E238DF80A30637803F07F038DF80B30D2
:10DF0000A3788DF80C30E3788DF80D3002AB21E06A
:10DF10000133DBB2092B16D803EB430C154800EB99
:10DF2000CC00027D012AF3D98268AA42F0D121688F
:10DF300042689142ECD10E4A13701A463146284687
:10DF4000FFF738FE0FE0324621462846FFF79EFED7
:10DF500009E00E4B4FF40062009205F136023146A3
:10DF6000284601F0B3F804B070BD6FF00300FAE783
:10DF700070050120740501205C770108E460010848
:10DF8000F46001082C79010888780108247D0108D3
:10DF90002DE9F04186B00646884617464FF42072B8
:10DFA00024212220FCF7F4FFA0B305464389232B4C
:10DFB00033D9D6F804C06C6884F8008067700023F9
:10DFC00023716371A371E3716B687268166850689E
:10DFD0009168D7689E60D86019615F611669506961
:10DFE00091699E61D8611962DCF80C30059305A82F
:10DFF00000F0F2F858B10021A170E1700290012305
:10E0000001930091FF2305AA284600F08FFA2846C5
:10E01000FCF756FF06B0BDE8F081044B4FF4B47234
:10E020000349044804F0C8FAC3E700BF387901087F
:10E0300070790108F46001082DE9F04184B00546CB
:10E04000494B9E68347804F00F04A400132C15D9B2
:10E050000F464389032B11D943681B78082B61D1E4
:10E06000414B586900F0F003E02B1AD03E4B196881
:10E0700000F071FAA8B92B89072B05D82846FCF7C0
:10E080001FFF04B0BDE8F08104F10E0841462846A8
:10E09000FCF7CFFE00283AD02B89191989B28B42A0
:10E0A00003D92846FCF70CFFEBE74FF420720E2053
:10E0B000FCF76EFF80460028F3D0428904F1080384
:10E0C0009A4213D322463146406804F013FC21469D
:10E0D0004046FCF7B3FE60B929464046FDF7C0F85C
:10E0E00088B92846FCF7ECFE454615E0FCF7E8FE4B
:10E0F000D7E71E4BB6221E491E4804F05DFA404683
:10E10000FCF7DEFECDE74046FCF7DAFEC9E7414604
:10E110002846FCF793FE48B96E6821462846FCF76E
:10E1200088FE50B12846FCF7CBFEAAE70F4BC7226A
:10E130001149104804F040FAB3E768680A494B698E
:10E14000C3600B69036100223270B270F270FF236A
:10E1500003728272C2720297012001900092143100
:10E16000284600F0E3F9DDE780CC0020387901088B
:10E170009C790108F4600108D479010808B50A46C1
:10E180000321FFF705FF08BD08B50A460B21FFF77D
:10E19000FFFE08BD90F83D3013F0010F14D010B50C
:10E1A0000446436893B10A4A5069834203D021462A
:10E1B00000F0D1F908B1012009E006492046FDF739
:10E1C00077FF20B1012002E000207047002010BD41
:10E1D00080CC002094CC00208446284B18682DE089
:10E1E0000068B8B190F83D3013F0010FF8D013F08B
:10E1F000040FF5D04268002AF2D0DCF800104A4043
:10E200008468224216D013F0020FE9D1C368994204
:10E21000E6D10FE01A4B1B6863B193F83D2002F082
:10E220000502052A06D15A6822B19CF800207F2AEF
:10E2300000D018465DF8044B7047006860B190F854
:10E240003D3013F0010FF8D013F0040FF5D0426801
:10E25000002AF2D010B4D0E7094B1B686BB193F8D9
:10E260003D2002F00502052A07D15A682AB19CF820
:10E2700000207F2A01D018467047704728050120EA
:10E28000240501202DE9F041044647683B781A092E
:10E29000042A04D0FCF714FE0020BDE8F0810E46ED
:10E2A00003F00F039D007888FBF768FE8046238902
:10E2B00083421BD86389AB421DD3238943451AD3BC
:10E2C000132D18D93B69574A5361F968116103F05E
:10E2D000F003E02B13D196F83D3013F0010F2CD052
:10E2E0007368002B6BD14FF0000828E001462046F0
:10E2F000FCF7FAFEDEE72046FCF7E2FDCCE730460D
:10E30000FFF748FFA0B9474B1B7D7F2B4DD0464BF5
:10E31000D3F8008001E0D8F80080B8F1000F08D0F1
:10E32000B045F8D04046FFF735FF0028F3D000E0B5
:10E33000B046B8F1000F05D101E04FF000087B7A3C
:10E34000112B35D0374B186900283AD1B8F1000F9E
:10E3500045D0FB8823F0C0039BB233B1204600F0C8
:10E360005DFC0446002897D047682E4AC2F800801A
:10E37000566097603B7803F00F039B00938129461A
:10E380002046FCF75BFD7B7A012B2CD0112B2FD183
:10E3900031462046FDF7AAF9224B00221A605A6046
:10E3A0009A609A811A615A6176E74FF00008C6E7D1
:10E3B0007B195B88B3F5884FC4D1B046C6E7B04639
:10E3C000C0E7314600F0C7F828B9164B1B6903F0C7
:10E3D000F003E02BBAD12046FCF772FD5CE7204643
:10E3E000FCF76EFD58E731462046FFF725FED3E7E0
:10E3F00041460C4B586900F0AEF828B9094B5B69EF
:10E4000003F0F003E02B03D12046FCF759FDC3E7EE
:10E4100029462046FCF74EFD02212046FFF7AEFEBE
:10E42000F2E700BF80CC0020280501202DE9F04351
:10E4300083B004460F4616469946DDF83080827B4D
:10E44000012A3FD1002E51D014212046FCF7F1FCC7
:10E45000002859D165686389132B3BD985F808904A
:10E460009DF82C306B7233682B6145232B709DF81F
:10E4700028306B702089FBF781FD68800023AB7129
:10E48000EB71DFF8A490B9F80000FBF777FDA880E6
:10E49000B9F800300133A9F800301FB33B68EB60D6
:10E4A0000023AB72EB72B8F8343013B12289934277
:10E4B00024D3D8F81430324621464046984703B05A
:10E4C000BDE8F083134B4FF455721349134804F021
:10E4D00073F8B7E70F4B4FF4627211490F4804F01D
:10E4E0006BF8BBE70F4B1B68EB60D9E76389132B15
:10E4F0000DD963681B69019301AED4E732464146EA
:10E50000204600F093FCDAE76FF00100D7E76FF0E8
:10E510000100D4E7087A01083C7A0108F460010898
:10E52000487A0108C47A01086406012010B584B055
:10E53000089C94461AB109B10A6802B9211D0294D7
:10E540009DF81C2001929DF8182000926246FFF76A
:10E550006DFF04B010BD0346421E12F1030F12D826
:10E5600091F83D0010F0020014D04A689A420CD095
:10E5700089685A400A420AD1CA4323EA01039A42EF
:10E5800007D000207047012070470020704700200E
:10E59000704701207047000030B585B00D46037804
:10E5A000EC4635E0421C4378782B04D0582B02D03F
:10E5B0001046082134E083780230102130E0102921
:10E5C0001BD112F0440F18D024010A3302F00302C9
:10E5D000022A10D041229B1A1C4310F8013F424AE4
:10E5E000D25C12F0040FEAD004FB0133A3F1300433
:10E5F00010F8013FF3E76122EDE72E2B12D103ABB8
:10E600009C4558D2624642F8044B43789446013008
:10E61000354AD25C12F0040F4BD0302BC2D00A2105
:10E620000024DCE713B112F0080F47D06B46ACEBC7
:10E63000030080100130042834D8DFE800F03D0BDF
:10E6400003132100B4F1807F3AD2009BFF2B39D80D
:10E6500044EA0364002D45D02046FBF794FC286073
:10E66000012029E0B4F5803F2ED2009AFF2A2DD850
:10E67000019BFF2B2CD81B0443EA02631C43E9E7F0
:10E68000FF2C27D80099FF2926D8019BFF2B25D8DE
:10E69000029AFF2A24D81B0443EA016343EA0223B7
:10E6A0001C43D7E7114BF9221149124803F084FFAC
:10E6B000D0E7002000E0002005B030BD0020FBE7DF
:10E6C0000020F9E70020F7E70020F5E70020F3E756
:10E6D0000020F1E70020EFE70020EDE70020EBE766
:10E6E0000020E9E70120E7E706870108787A0108BA
:10E6F000B47A0108F460010800B583B001A9FFF7FE
:10E700004BFF20B94FF0FF3003B05DF804FB0198D8
:10E71000FAE700002DE9F04182B0884603680193D2
:10E720000C460026304601AF03283BD800233D7835
:10E730002049A1FB05CE4FEADE0E0EEB8E0CA5EBB9
:10E740004C0C5FFA8CFC87F800E09E460133DBB28C
:10E750000CF1300C0EF108010DEB010E0EF808CC97
:10E76000092DE4D809E005F108010DEB010616F8C2
:10E77000086C04F8016B1E462B465D1EEDB233B1EA
:10E78000731C9642EFDB002002B0BDE8F081731CE1
:10E7900096420CDA2E2504F8015B01370130C0B235
:10E7A0001E46C1E7002304F8013C4046ECE7002088
:10E7B000EAE700BFCDCCCCCC08B510220149FFF769
:10E7C000A9FF08BD6806012038B504460C4B1B683C
:10E7D000834208D00D4651B123682B6021460120A9
:10E7E000FBF79CFF38BD0268054B1A60F6E7054B46
:10E7F00040F245120449054803F0DEFEECE700BF95
:10E800007C060120C87A0108047B0108F460010835
:10E810002DE9F84380468946814215D0B9F1000FB1
:10E8200009D0D9F80030434505D0314BAD223149EC
:10E83000314803F0C1FED8F8044063689A8852B1A9
:10E840000026D8F804502BE0294BAB222B492A484C
:10E8500003F0B2FEE2E71B68C8F804306368D8F83A
:10E860000820D8F80C50D8F81000D8F814101A6006
:10E870005D609860D960D8F818201A61012120469F
:10E88000FFF782FC2046FCF783FC06462046FCF797
:10E8900017FBD6E73444A6B22846FCF711FB3D46E9
:10E8A00085B16B681F682846FCF772FC0446331874
:10E8B000B3F5803FEEDB0E4BCC2211490E4803F03E
:10E8C0007BFEE7E749464046FFF77EFF0D4B1B887E
:10E8D000B34206D30B4A13889B1B13803046BDE816
:10E8E000F883034BD2220849034803F065FEF1E7A1
:10E8F000C87A01082C7B0108F4600108207B01081C
:10E90000407B010878060120607B0108F8B50546C8
:10E910000F4600262BE09A69D5F810E0724511D118
:10E92000B3F80CE0AA8896450CD101E06146184680
:10E930001A6892B19C4613468BB15A69D5F80CE01F
:10E940007245E8D001340028F0D093F81FE0C27F70
:10E950009645EDD861461846EAE76346EAE710B106
:10E96000FFF756FF0644BE4208DA012C06DD044BD1
:10E970001B6800242146A4462046DDE73046F8BD4A
:10E980007C06012010B5044620B121460220FBF789
:10E99000C5FE10BD034B4FF431720349034803F029
:10E9A0000BFEF2E7C87A010858750108F460010807
:10E9B00010B5044638B1606908B1FCF781FA204609
:10E9C000FFF7E0FF10BD044B40F2CE22034904489C
:10E9D00003F0F2FDEFE700BFC87A0108847B01086D
:10E9E000F46001082DE9F84380460D4691464C68D5
:10E9F0006088FBF7C3FA237803F00F03B0EB830FB3
:10EA000003D24FF0FF30BDE8F8839A00801A87B236
:10EA1000E088FBF7B3FAC0F30C0C4FEACC0C6E683D
:10EA2000002333707370B370F370A6F804C007EB63
:10EA30000C001FFA80FEF080E645C0F08580D8F813
:10EA4000041001271C461FE03160ACB1E28862452A
:10EA50007DD89B889E457DD82560B3889A4200D09A
:10EA6000002719B3B9F1000F41D198F81E3013F007
:10EA7000010F3CD14846C6E79B889E456DD8C8F833
:10EA80000450EEE719681C460029EAD04B689A88C2
:10EA90006245D9D8624563D0D988614563D8002CD6
:10EAA000F0D0E1888A42EDD00027EBE794B1E2880C
:10EAB000B3889A4206D82560E288B3889A42D1D0BA
:10EAC0000027CFE7294B4FF4DB722949294803F08F
:10EAD00073FDF0E7D8F8043033B1244B4FF4DF7204
:10EAE0002549244803F068FDC8F80450BAE74FB33D
:10EAF000D8F804301BB35868838813BB32684AB116
:10EB00005368F1889A88914202D11A681E46F6E746
:10EB10001E460027B7B1B04209D0336893B1134BFA
:10EB20004FF4F1721549134803F046FD0AE00F4B0C
:10EB30004FF4F07212490F4803F03EFDEDE7002755
:10EB400000E0002738465EE74FF0FF305BE74FF00C
:10EB5000FF3058E74FF0FF3055E74FF0FF3052E7F6
:10EB60004FF0FF304FE74FF0FF304CE7C87A010815
:10EB7000907B0108F4600108B07B0108F87B010874
:10EB8000E87B010808B50220FBF79AFD08BD0000EC
:10EB900070B505460E460120FBF792FD0446B0B164
:10EBA00020220021204603F0B1FD0F23E3770F4B15
:10EBB0001A6822601C602B686868A968EA68A3600C
:10EBC000E060216162612B69A361204670BD31461E
:10EBD0002846FFF79BFEB04202DA002CE0D1F4E7B2
:10EBE0000120FBF76DFD0446F7E700BF7C0601201E
:10EBF00038B5094B1868002403E0013BC37704468D
:10EC0000006840B1C37F002BF7D105682146FFF7AC
:10EC1000FFFD2846F5E738BD7C0601202DE9F843C5
:10EC2000064645682B7803F00F03052B40F0D18092
:10EC3000E888FBF7A3F9C0F30C084FEAC808688816
:10EC4000FBF79CF92B7803F00F039A00B0EB830FCE
:10EC5000C0F0BF80801A87B23046FCF799FA81462F
:10EC60006B4B1B8803440A2B02DC6A4B1C680DE0CB
:10EC700001462846FFF74AFE002800F0AA80644BB0
:10EC80001B884B440A2BF0DDA3E024685CB1626969
:10EC9000EB689A42F9D1A2692B699A42F5D1A2890F
:10ECA000AB889A42F1D174B3E888FBF767F9C0F3F7
:10ECB0000C0080B3ED8805F02005002D0CBF01226B
:10ECC000002208D108EB07039BB298457ED84FF687
:10ECD000EB718B427AD831462046FFF783FEB0F1C4
:10ECE000FF3F73D04A4B1A889144A3F8009035B97E
:10ECF000B844A4F81C80A37F43F00103A377012844
:10ED00001BD0002569E049462846FFF741FF04462D
:10ED10000028CFD15DE0E089FBF730F9C0F30C00AB
:10ED20000028C7D02B686868A968EA68A360E0601B
:10ED3000216162612B69A361BCE7A08B1430636819
:10ED40005D682E68A368E768216962692B606F605F
:10ED5000A960EA60A3692B6180B2FBF70FF96880B4
:10ED60000023AB71EB71AB72EB72656809E07768F9
:10ED700014213046FCF762F831462846FCF72EFA9B
:10ED80003E68002EF3D1234B1968A14205D029B16A
:10ED90000B68A34202D01946F9E731462046FFF737
:10EDA00013FD2846FCF7F4F90446194B1B888342EF
:10EDB00004D3174A13881B1B13800EE0164B40F236
:10EDC0009B221649164803F0F7FBF2E744B163684B
:10EDD00073B13046FCF774F800252846BDE8F88387
:10EDE0000D4B4FF42A720F490D4803F0E5FBEEE797
:10EDF000084B1B68A34206D0074B40F2AB220A49DE
:10EE0000074803F0D9FB00212046FFF7DDFCE0E7CF
:10EE1000780601207C060120C87A01081C7C0108C4
:10EE2000F4600108387C0108447C01082DE9F04FAA
:10EE30008BB00646079108928B8E143B4ED4C3F3D9
:10EE4000CF030593D6F804B09BF8003003F00F030E
:10EE5000052B40F0D5807389132B41D9BBF80600F0
:10EE6000FBF78CF8C0F30C03069300F400530993EE
:10EE70003389143B1FFA83F814270024CDF80C8043
:10EE8000039B002B00F0BA80059BDB009BB2039A2A
:10EE9000934228BF134604934FF4207214210E208E
:10EEA000FCF776F88146002800F0AD804389132BEB
:10EEB00020D9D9F80430DBF80020DBF80450DBF867
:10EEC0000800DBF80C101A605D609860D960DBF810
:10EED00010201A61D9F804A0049D3CE00733AEE786
:10EEE0004A4B4FF43F724A494A4803F065FB6FF0C2
:10EEF000050043E0454B4FF449724749454803F04C
:10EF00005BFBD6E7414B40F22D324449414803F0C8
:10EF100053FB26E0FFF736FE804650B3736801943A
:10EF20003B4400930346412221460020FBF762FF49
:10EF3000029030B33046FCF735F9C8F81460384B0E
:10EF4000C8F8103002994846FCF748F92D1BADB2BD
:10EF50000DB136680027EDB17389DC1BA4B2BB424A
:10EF6000D0D3AC4228BF2C46002CD3D136682746DC
:10EF7000F1E74846FBF7A4FF4FF0FF300BB0BDE8C8
:10EF8000F08F4046FFF7FEFC4846FBF799FF4FF035
:10EF9000FF30F3E72744BFB2079B9B8E133B069AD3
:10EFA000C2F30C00039A934201DD099B0BB140F4BC
:10EFB0000050FAF7E3FFAAF80600049D05F11400DB
:10EFC00080B2FAF7DBFFAAF8020000238AF80A30C1
:10EFD0008AF80B3007984369089A4946984748468B
:10EFE000FBF76EFF039BA3EB050A1FFA8AF303935B
:10EFF000069B059A13449BB2069341E70020BDE7A8
:10F000006FF00500BAE74FF0FF30B7E7C87A0108A4
:10F01000647C0108F4600108807C0108A07C010880
:10F02000B1E9000870B5044643890E2B1CD90D4682
:10F03000C37B1BB991F840300133C3736068868984
:10F04000037813F0010F0AD0012B12D006221E49BB
:10F0500003F032FB18B9637B43F008036373082E97
:10F0600012D0B6F5C16F1FD02046FBF729FF002054
:10F0700070BD4378002BF2D183785E2BEFD1637B98
:10F0800043F010036373EAE795F83D3013F0080F7F
:10F09000EAD00E212046FBF7D1FE0028E4D1294614
:10F0A0002046FFF7EFF8E2E795F83D3013F0080F40
:10F0B000DAD00E212046FBF7C1FE0028D4D1294624
:10F0C0002046FEF7C3FCD2E7247D01082DE9F0417C
:10F0D00005460C4616461F46BDF81800FAF74EFFC7
:10F0E00080460E212046FBF7A4FEE8B96168A1F82E
:10F0F0000C803B680B60BB888B803368C1F806309E
:10F10000B3884B8195F83C30062B05D1AB6921467D
:10F1100028469847BDE8F081054B4FF499720549A0
:10F12000054803F049FAF1E76FF00100F2E700BF8C
:10F13000B07C0108E87C0108F460010810B584B0D7
:10F140000446009104230193002102910391684633
:10F15000F7F7B0FC206010B1002004B010BD4FF0F4
:10F16000FF30FAE710B504460068F7F72FFD206876
:10F17000F7F739FD10BD08B500220068F7F7AFFCBE
:10F1800000B908BD4FF0FF30FBE7F0B589B0054688
:10F190000F461446F7F7F0FA06468CB12246296866
:10F1A00005A8F7F7CFFC059B102B03D04FF0FF30DD
:10F1B00009B0F0BD069B3B60F7F7DEFA801BF7E76E
:10F1C0006C464FF0FF3229682046F7F7BBFC94E805
:10F1D000070008AB03E907003960F7F7CDFA801B99
:10F1E000E6E710B584B00C460022016801A8F7F7E5
:10F1F000A9FC019B102B03D04FF0FF3004B010BDD1
:10F20000029B23600020F9E703680BB101207047DF
:10F210000020704700230360704730B583B0044678
:10F220000D4600230093019301216846F7F7AEFBDA
:10F23000206040B115B1002003B030BD0021F7F7C8
:10F24000D1FB0020F8E74FF0FF30F5E708B5006884
:10F25000F7F7F7FB08BD08B50068F7F71FFC08BD16
:10F2600003680BB101207047002070470023036042
:10F270007047000008B50348F7F720FB024B186001
:10F2800008BD00BF2C7D01088006012010B582B0AA
:10F2900004460023009301936846F7F70FFB2060B4
:10F2A00010B1002002B010BD4FF0FF30FAE708B5F2
:10F2B0004FF0FF310068F7F70CFB08BD08B5006898
:10F2C000F7F737FB08BD10B588B00024019402940D
:10F2D0000394049405940694079401900291BDF957
:10F2E0002810ADF80C100593114601A8F7F74EFA57
:10F2F00008B010BD08B54FF0FF31034B1868F7F7A1
:10F30000E8FA012008BD00BF8006012008B5024BC5
:10F310001868F7F70EFB08BD8006012090F83D3015
:10F32000012B2CD10368174A0221934280F83D102B
:10F330001AD0B3F1804F17D0A2F57C42934213D07C
:10F3400002F5806293420FD002F5806293420BD0A7
:10F3500002F57842934207D002F57052934203D0EF
:10F36000A2F59432934204D19A6802F00702062A69
:10F3700003D01A6842F001021A6000207047012091
:10F38000704700BF000001400368196A41F2111282
:10F39000114208D1196A40F24442114203D11A685D
:10F3A00022F001021A60012380F83D3000207047EE
:10F3B00010B582B0044600230193094802685362E5
:10F3C000FFF7ACFF03E0064B1B685B6A0193019BF0
:10F3D000A342F8D30248FFF7D7FF02B010BD00BF29
:10F3E000D407002038B50546002404E04FF47A70B5
:10F3F000FFF7DEFF0134AC42F8DB38BD08B5F2F7A9
:10F400009DFD08BD10B50446F2F798FDA04201D35A
:10F41000001B10BD001B0138FBE700BF0048704710
:10F4200000000E0810B5174B1B784BB9164B1C6823
:10F4300022684DF6BA439A421FD1002319460EE0C6
:10F44000FFF7DCFF0146104B1B681B680F4A104892
:10F4500000F0C0FBEAE754F82320114401330D4AC1
:10F460001268501E9842F6D802F18042013A54F8D0
:10F4700022308B4203D1012000E0002010BD00208B
:10F48000FCE700BF260000208C060120347D010827
:10F490003C7D01088406012010B586B0002300934E
:10F4A00001930293039304930A230293012303938A
:10F4B00002230493F4F78CF80C4BF322DA6005A9CD
:10F4C0006846F4F7B3F9044610B1094B1B7823B929
:10F4D000F4F796F8204606B010BDFFF78FFF0146FF
:10F4E000044A054800F076FBF2E700BF003C02400A
:10F4F00026000020347D0108647D010808B5064B14
:10F500001860064B00221A60054B19608A000549F5
:10F5100003F0F0F908BD00BF8C0601208806012029
:10F520008406012000000C0808B5FFF77BFF08BD2A
:10F53000014B186001207047880601208446002393
:10F54000184603E05CF82320104401338B42F9D3C2
:10F550007047000038B51D4B1C684DF6BA43236058
:10F560001B4B196801F18045013D01392046FFF729
:10F57000E5FF44F82500FFF78FFFF4F729F8002492
:10F5800000E00134124B1B68A3421AD904F1007148
:10F5900001F540310D4B1B6853F8242000238900EE
:10F5A0000220F4F767F80028EBD00A4B1B78002BF9
:10F5B000E7D0FFF723FF0146074A084800F00AFB9F
:10F5C000DFE7F4F71DF8012038BD00BF8C060120ED
:10F5D0008406012026000020347D0108847D010876
:10F5E00008B5064B1A689200054B1968054B186858
:10F5F00003F080F9FFF7AEFF012008BD840601206B
:10F60000880601208C0601208AB04E4B984219D002
:10F610004D4B984225D04D4B984230D04C4B9842A0
:10F620003BD04C4B984246D04B4B984251D04B4B21
:10F6300098425CD04A4B984267D04A4B984272D06D
:10F6400000200CE000230193474B1A6B42F00102AB
:10F650001A631B6B03F001030193019B01200AB0A5
:10F66000704700230293404B1A6B42F002021A6368
:10F670001B6B03F002030293029B0120EFE70023C0
:10F680000393394B1A6B42F004021A631B6B03F0AD
:10F6900004030393039B0120E1E700230493324B0F
:10F6A0001A6B42F008021A631B6B03F00803049301
:10F6B000049B0120D3E7002305932B4B1A6B42F0E8
:10F6C00010021A631B6B03F010030593059B0120C6
:10F6D000C5E700230693244B1A6B42F020021A63FD
:10F6E0001B6B03F020030693069B0120B7E7002362
:10F6F00007931D4B1A6B42F040021A631B6B03F019
:10F7000040030793079B0120A9E700230893164BAA
:10F710001A6B42F080021A631B6B03F0800308939C
:10F72000089B01209BE7002309930F4B1A6B42F4BF
:10F7300080721A631B6B03F480730993099B012089
:10F740008DE700BF000002400004024000080240B4
:10F75000000C024000100240001402400018024059
:10F76000001C02400020024000380240000901381D
:10F77000062811D8DFE800F0041206080A0C0E0073
:10F780000748704707487047074870470748704761
:10F790000748704707487047002070470648704781
:10F7A0000000024000080240000C0240001002402D
:10F7B00000140240001802400004024000F00F0054
:10F7C0000F282FD8DFE800F008300A0C0E101214B2
:10F7D00016191C1F2225282B012070470420704772
:10F7E0000820704710207047202070474020704745
:10F7F000802070474FF4807070474FF4007070475E
:10F800004FF4806070474FF4006070474FF48050B1
:10F8100070474FF4005070474FF4804070474FF4EA
:10F8200000407047002070470220704708B520282C
:10F8300016DC002843DD01381F2840D8DFE800F03F
:10F840004A4C3F373F3F3F393F3F3F3F3F3F3F3BC2
:10F850003F3F3F3F3F3F3F3F3F3F3F3F3F3F3F3DBA
:10F86000B0F5806F3AD00BDDB0F5005F3CD016DD0F
:10F87000B0F5804F3CD0B0F5004F20D128200DE0EE
:10F88000B0F5807F2CD004DDB0F5007F17D11720B4
:10F8900004E0402826D0802811D1172008BDB0F5FB
:10F8A000006F23D0B0F5805F09D12820F6E708204B
:10F8B000F4E70920F2E70A20F0E71720EEE7B92382
:10F8C0000C4A0D490D4800F085F94FF47A70FFF7A6
:10F8D00089FDF4E70620E1E70720DFE72820DDE7E0
:10F8E0001720DBE71720D9E72820D7E72820D5E71E
:10F8F0002820D3E7A47D0108C06C0108C07D010861
:10F9000000296BD0F0B587B0044615460F469DF828
:10F9100030204273857203730123C372017008465D
:10F92000FFF724FF064660603846FFF747FF208157
:10F930002DB1012D1CD0022D1CD0002500E000258A
:10F940003046FFF761FE0023019302930393049373
:10F950000593237B83B923890193039501A96068EB
:10F96000F3F7C4FF237B63BB0123A37307B0F0BD90
:10F970000125E5E70225E3E7012B0AD0022B14D08D
:10F98000032BEBD1238901934FF444130293039586
:10F99000E4E723890193637B23B14FF404130293BB
:10F9A0000395DBE74FF48813F9E723890193637B21
:10F9B00023B94FF4041302930395CFE74FF4881350
:10F9C000F9E72089FFF732FF00220521F2F734FB27
:10F9D0002089FFF72BFFF2F753FBC5E770472DE9AE
:10F9E000F04186B09DF8308011B906B0BDE8F081D5
:10F9F00004460E4643738272002505730223C372C8
:10FA000001700846FFF7B2FE074660603046FFF718
:10FA1000D5FE20813846FFF7F7FD01950295039545
:10FA200004950595637B0BB188F001084246218956
:10FA30006068F4F7CFF8A37A6BB9238901930123A7
:10FA4000029300230393049301A96068F3F74EFF28
:10FA50000123A373C9E7012B0BD0022B11D0032B79
:10FA6000F2D123890193112302930023039304937A
:10FA7000EAE723890193012302930393002304936C
:10FA8000E2E72389019301230293022303930023D6
:10FA90000493D9E710B5044601894068F4F786F865
:10FAA000637B23B9012814BF0020012010BD013859
:10FAB00018BF0120FAE708B50A46437B0BB181F075
:10FAC000010201894068F4F785F808BD08B50120F6
:10FAD000F4F79CF808BD08B50220F4F797F808BDC4
:10FAE00008B50420F4F792F808BD08B50820F4F72B
:10FAF0008DF808BD08B51020F4F788F808BD08B5E2
:10FB00002020F4F783F84020F4F780F88020F4F701
:10FB10007DF84FF48070F4F779F84FF40070F4F743
:10FB200075F808BD08B54FF48060F4F76FF84FF42E
:10FB30000060F4F76BF84FF48050F4F767F84FF477
:10FB40000050F4F763F84FF48040F4F75FF84FF497
:10FB50000040F4F75BF808BD30B585B004460023DB
:10FB6000037080224270E12282700393029301931A
:10FB70000A4D03A92846F4F70FFD02A92846F4F719
:10FB80000BFD01A92846F4F707FD039BE370029BD8
:10FB90002371019B637105B030BD00BF00050020DB
:10FBA00070B582B00C46164600250BE014F8013BF8
:10FBB0008DF80730642301220DF107010448F6F7A0
:10FBC0001FFA0135B542F1DB304602B070BD00BF0F
:10FBD0000C0900200FB400B583B0074B1B7823B984
:10FBE00003B05DF804EB04B0704705A901910498D7
:10FBF00002F058FDF4E700BF2600002030B589B0C0
:10FC00000446114B1B78B3B91023039303AB019344
:10FC100004AB00930023E269A1692069F9F750FF62
:10FC20000028F1DD256A002DEED083B2A26904A977
:10FC30002046A847E8E7FFF7E1FB0146A36A034A2D
:10FC40000348FFF7C7FFDFE726000020D87D010843
:10FC5000E07D010810B588B004461023039303AB80
:10FC6000019304AB00930023E269A1692069F9F7CD
:10FC700027FFF2E7F0B58FB004460E4617461D4643
:10FC80002C22002102F042FD022363704448FEF75B
:10FC900033FD60603846FAF771F960802562159B84
:10FCA0006362A662149BCBB94FF48063E361E069A1
:10FCB00001F0DAFBA061A0B1112202210846F9F798
:10FCC000C7FF2061002817DB10222146F9F7B6FE96
:10FCD00048B3344B1B78EBB9002011E0149BE3616F
:10FCE000E5E73B23304A31493148FFF773FF4FF4D2
:10FCF0007A70FFF777FBF4E72A4B1B7813B90020E3
:10FD00000FB0F0BDFFF77AFB01462A4A2A48FFF7F9
:10FD100061FFF4E7FFF772FB0146284B254A2848AC
:10FD2000FFF758FFD8E701220023CDE90A2300237B
:10FD30000C93102300930AAB41F2060240F6FF71C8
:10FD40002069F9F7C9FF80B945B303AD1D4E0FCE49
:10FD50000FC596E8070085E80700214603A8F6F7D7
:10FD600015FD606178B10120CAE70E4B1B780BB915
:10FD70000020C5E7FFF742FB0146134B0D4A104830
:10FD8000FFF728FFF4E74E23074A10490848FFF71A
:10FD900021FF4FF47A70FFF725FBF4E70120AFE76E
:10FDA000187E010826000020207E01083C7E010804
:10FDB000C07D0108D87D0108607E0108887E0108A9
:10FDC000EC7E0108185D01080C7F0108647F0108C2
:10FDD00010B582B00C4611461A46006910230193F3
:10FDE00000940023F9F7B2FE02B010BD70B58EB0DA
:10FDF00004460D462022002102F088FC0223637095
:10FE00003E48FEF779FC60602846FAF7B7F8608054
:10FE10004FF48060E06101F027FBA061E0B11122A6
:10FE200002210846F9F714FF206100281FDB012298
:10FE30000023CDE90A2300230C93102300930AAB7F
:10FE400041F2060240F6FF71F9F746FF30B32C4B42
:10FE50001B78D3B900200EE066232A4A2A492B4892
:10FE6000FFF7B8FE4FF47A70FFF7BCFAF4E7244BC3
:10FE70001B7813B900200EB070BDFFF7BFFA014622
:10FE8000234A2448FFF7A6FEF4E7FFF7B7FA014636
:10FE9000214B1F4A2148FFF79DFEDBE71022214638
:10FEA0002069F9F7CBFD68B1154B1B780BB9002021
:10FEB000E1E7FFF7A3FA0146194B154A1748FFF788
:10FEC00089FEF4E703AD174E0FCE0FC596E8070085
:10FED00085E80700214603A8F6F758FC606108B1E1
:10FEE0000120C8E77623074A0F490848FFF772FE4A
:10FEF0004FF47A70FFF776FAF4E700BF187E010836
:10FF000026000020207E01088C7F0108C07D0108AA
:10FF1000D87D0108607E01080C7F0108EC7E010895
:10FF2000887E0108345D0108647F0108F0B587B060
:10FF300004460F4615461E4602238DF809304FF041
:10FF4000FF30FAF720F80390B8B2FAF717F8ADF8D7
:10FF50000A001023019302AB009300233246294686
:10FF60002069F9F7F3FD07B0F0BD0000F0B587B0E8
:10FF7000034614464DF6BA4222602E4AA26002F1B0
:10FF80007742E2606FF07F422261012262600322C9
:10FF9000626182690AB9818B89B1B2F1FF3F29D0D0
:10FFA000254A986910609B8B93800023A361E361CD
:10FFB000214B1868A0619B88A38307B0F0BD1E4841
:10FFC000FFF7CAFD1D4B1B78002BEED0FFF716FA8A
:10FFD0000146194B5A789878DD781E795F79049735
:10FFE00003960295019000921B78154A1548FFF779
:10FFF000F1FDDAE7998B4FF6FF729142D0D10E48AE
:020000040801F1
:10000000FFF7AAFD0D4B1B78002BCED0FFF7F6F9BA
:100010000146094B5A789878DD781E795F79049704
:1000200003960295019000921B78054A0548FFF758
:10003000D1FDBAE7C0A8080A9806012026000020D2
:10004000D47F0108DC7F010870B586B004463F4BC1
:100050001B78C3B93D4B1B78EBB93C4B1B78002B8D
:100060002ED13A4B1B78002B38D1384B1B78002B04
:1000700042D1364B1B78002B4CD1344B1B78002BD4
:100080005BD106B070BDFFF7B9F90146304A31487F
:10009000FFF7A0FDDEE7FFF7B1F901462379012B59
:1000A0000AD0022B0AD02BB12B4B294A2B48FFF741
:1000B00091FDD2E72A4BF8E72A4BF6E72A4BF4E703
:1000C000FFF79CF9054604F10800FEF775FB0346AF
:1000D0001F4A29462548FFF77DFDC2E7FFF78EF945
:1000E000054604F10C00FEF767FB0346184A294653
:1000F0001F48FFF76FFDB8E7FFF780F9054604F1E9
:100100001000FEF759FB0346114A29461948FFF72C
:1001100061FDAEE7FFF772F90146637EA27EE07EE5
:10012000257F667F04960395029001920093237EBB
:10013000074A1148FFF74EFD9FE7FFF75FF90146B9
:10014000034A0E48FFF746FD9BE700BF260000204C
:10015000D47F01083C8001083480010878800108C0
:10016000208001082880010830800108A88001084B
:10017000D8800108088101083881010884810108BC
:1001800070B5134B1B78BBB9124E09213046FFF7EF
:10019000B5F9FFF7C9F980F00104E4B20E4D2A4623
:1001A00021463046FFF7E2FE2846FFF7C1F95CB969
:1001B0000848FFF749FF70BDFFF720F90146074ADD
:1001C0000748FFF707FDDFE7FFF70AFAF0E700BF90
:1001D00026000020C4060120A0060120D47F0108CB
:1001E000C081010800487047C406012008B5FFF728
:1001F000B1F908BD08B5FFF7F3F908BD70B586B0D1
:100200001248FFF7A9FC124B1B7853B9114B00227F
:100210001A605A600D4A92E803001860998006B08F
:1002200070BDFFF7EBF80146084B5A789878DC78F8
:100230001D795E79049603950294019000921B78D3
:10024000054A0648FFF7C6FCE0E700BF900601201C
:1002500026000020DC060120D47F0108DC7F010895
:1002600030B585B004461D4600230293ADF80C302E
:100270008DF80E300093ADF804308DF806308DF80F
:100280000810C1F307218DF8091061F07F018DF886
:1002900009108DF80A20130A8DF80B30130C8DF815
:1002A0000C30120E8DF80D2007236A4602A9F4F7D0
:1002B0009FFD2046F4F784FF0128FAD19DF8023013
:1002C0009DF8032043EA02239DF8042043EA0243F9
:1002D0009DF8052043EA02632B6005B030BD30B5C0
:1002E00085B00446154600230293ADF80C308DF816
:1002F0000E300093ADF804308DF806308DF80810FC
:10030000090A8DF8091007236A4602A9F4F770FD5F
:100310002046F4F755FF0128FAD19DF802309DF8E8
:10032000032043EA02239DF8042043EA02439DF898
:10033000052043EA02632B6005B030BDF0B585B0FF
:100340000420F6F718FF284B1860284C284B236030
:100350000125009500232A4614212648FFF73FFB7C
:100360004FF47A732A4603A92068F4F781FC4623E8
:1003700084F8D030442184F8D110452384F8D23059
:10038000472384F8D330002600962B46022204F13E
:10039000E400FFF7B5FA00962B46022294F8D0103D
:1003A00004F1D400FFF7ACFA00960323022294F87C
:1003B000D21004F1F400FFF7A3FA04F58277009657
:1003C00033462A4694F8D3103846FFF708FB3146E7
:1003D0003846FFF770FB0A20FFF704F82946384635
:1003E000FFF769FB05B0F0BDE8060120FC0601201F
:1003F000E8060020EC0601202DE9F84305460F46EB
:100400001646DFF864804FF0FF31D8F80000F7F7A8
:100410002EF9144C00212046FFF74DFBDFF84C90DD
:1004200033463A462946D9F80000FFF719FF012163
:100430002046FFF740FB0120FEF7BAFF00212046CF
:10044000FFF739FB32462946D9F80000FFF747FF8E
:1004500001212046FFF72FFBD8F80000F6F7A5FE94
:10046000BDE8F883EC060120E8060120FC06012027
:10047000F8B504460D460C4E4FF0FF313068F7F7E3
:10048000F6F80A4F00213846FFF715FB2A462146A9
:10049000074B1868FFF723FF01213846FFF70BFBD6
:1004A0003068F6F782FEF8BDE8060120EC06012070
:1004B000FC06012000487047FC060120BFF34F8F67
:1004C0000549CA6802F4E062044B1343CB60BFF3F2
:1004D0004F8F00BFFDE700BF00ED00E00400FA050C
:1004E00010B582B00124009400231A462621094841
:1004F000FFF775FA009400231A4627210648FFF7F4
:100500006EFA009400231A4628210448FFF767FA80
:1005100002B010BD40080120300801202008012051
:1005200010B5044600210648FFF7C5FA21460548E4
:10053000FFF7C1FA21460448FFF7BDFA10BD00BF1E
:1005400040080120300801202008012008B500F0F3
:10055000EDFE08BD08B50F4B1868FEF753FF502895
:1005600000D808BD0C4B197881F0010119700B48B7
:10057000FFF7A1FA00F0D4FB38B10120FFF7D0FF5C
:10058000FEF73CFF034B1860EBE7034B1878FFF7CF
:10059000C7FFF5E71C0801201808012060080120AA
:1005A00008B5294B1B781BB1274B1B786BB908BDCD
:1005B0002648FFF76FFA0028F6D0FEF71FFF244BFE
:1005C0001860214B01221A70EEE72048FFF762FA0B
:1005D00018B91D4B00221A70E9E71D4B1868FEF789
:1005E00011FF40F6B8339842E1D91A4B1B7813B982
:1005F000FFF700FE15E0FEF701FF0146164A174817
:10060000FFF7E8FAF4E70020FFF78AFF4FF47A706B
:10061000F6F7EFF80120FFF783FF4FF47A70F6F753
:10062000E8F80A48FFF736FA0028ECD1094B1B78A6
:100630000BB9FFF743FFFEF7E1FE0146064A084803
:10064000FFF7C8FAF5E700BF1008012050080120A5
:100650001408012026000020E0810108E88101083B
:100660001882010870B584B0374B1B78002B3FD13E
:10067000354B1B78002B49D1002400942346224699
:1006800020213248FFF7ABF9FFF72AFF0122009241
:10069000234621212E48FFF733F9FFF771FD00F0C3
:1006A000F3F9FFF74BFEFFF705FF90F8D040FFF797
:1006B00001FF90F8D110204600F062FE00F050FBE0
:1006C0004FF47A70F6F795F800F0CCF8F0F7ACFD3F
:1006D0001D4B1B787BBB0A20F6F78BF8FFF73AFF20
:1006E000FFF75EFF00F0F2FA1A48F3F7E7FAF2E7D5
:1006F000FEF784FE01460023029301930623009334
:10070000154B164A1648FFF765FAB1E7FEF776FE75
:100710000446FEF783FE0578FEF780FE4678FEF776
:100720007DFE4388019300962B460C4A21460D48D6
:10073000FFF750FAA0E7FEF761FE0146074A0A48B4
:10074000FFF748FAC7E700BF260000206008012035
:1007500050080120F404002038820108E0810108DB
:1007600040820108608201088482010808B5FFF711
:1007700079FF000070B5064614460B4D01232B800F
:1007800083685A886A809B88AB80EC80A20005F160
:10079000080002F0AFF8A31C9B002A46716830687D
:1007A000FFF716FB70BD00BF740C012030B587B099
:1007B000144600220392049205920491039005943A
:1007C00022880AB107B030BD0B46224A01211170C0
:1007D000214D186859689A68DB680FC5A388012BFA
:1007E00016D0022B20D0032BECD1A068E1684FF487
:1007F00080730193194C2246002342F8043B01AB5D
:1008000000F094FB019A214603A8FFF7B3FFD9E754
:1008100000230193A06800F0A5FA0290022201A92A
:1008200003A8FFF7A7FFCDE700230193E168A068C5
:1008300000F014FB0290022201A903A8FFF79AFF1F
:10084000074B1B78002BBDD06420F5F7D2FFF1F7E2
:100850002DFCB7E7741401207814012070080120E2
:10086000B414012000B583B0002301934FF48063DA
:1008700000930B4B44F6BC520A490B48FFF7FAF9B8
:1008800050B98523094A0A490A48FFF7A3F94FF4EA
:100890007A70FEF7A7FDF4E703B05DF804FB00BF34
:1008A000AD070108A882010888140120B882010858
:1008B000DC820108C07D01087047704770B50C46A6
:1008C0001546614B5B683BBB11F0080F02D05F4BD4
:1008D0001B785BB914F0040F21D05C4B1B7873B903
:1008E0002B78ABB15A4B01221A7018E0FEF786FD47
:1008F00001462B78574A5848FFF76CF9EAE7FEF7AC
:100900007DFD01462B78534A5448FFF763F9E7E72A
:100910004F4B00221A7002E00646012B00D070BD3A
:1009200011F0080F02D0494B1B786BB914F0040F7B
:1009300025D0464B1B7883B92B78BBB17368F3B1D4
:10094000434B01221A701AE0FEF758FD01462B783E
:10095000404A4348FFF73EF9E8E7FEF74FFD0146FE
:100960002B783C4A3F48FFF735F9E5E7374B1B78D2
:10097000F3B93D4B1B781BBB354B00221A7014F0AA
:10098000F00FCCD0736813B3304B1B78002B2AD1F7
:100990002E4B1B78002B2ED12C4B1B78002B37D1E4
:1009A0002A4B1B78002B41D1294B01221A70B6E744
:1009B000FEF724FD0146274A2C48FFF70BF9D8E73C
:1009C0002B48FCF737FE284B00221A70D4E71F4B48
:1009D0001B78002BA3D0FEF711FD01461D4A2548C8
:1009E000FFF7F8F89BE7FEF709FD0146194A224890
:1009F000FFF7F0F8CCE7FEF701FD0446301DFDF7E8
:100A0000DBFE0346134A21461C48FFF7E3F8C3E721
:100A1000FEF7F4FC044606F10800FDF7CDFE0346A0
:100A20000C4A21461648FFF7D5F8B9E7FEF7E6FC71
:100A3000044606F10C00FDF7BFFE0346054A2146B9
:100A40001048FFF7C7F8AFE7C814012026000020C0
:100A5000EC14012038830108408301087C830108DD
:100A6000B8830108F4830108C6140120308401080A
:100A700008150120508401086C840108A88401082D
:100A8000CC840108F084010830B58DB0794B1B7817
:100A9000002B40F09F80FFF7A5FB774CA6468446CD
:100AA000BCE80F00AEE80F00BCE80F00AEE80F0096
:100AB000DCF80030CEF800306368A1686F4A11603E
:100AC0006F4A1060E1686F4A1160002B40F08E8021
:100AD0006D4B04F1180292E8030018609980002120
:100AE0000846F9F709FA654A117853781B0443EA76
:100AF0000163917843EA0123D1780B431A0202F48F
:100B00007F0242EA0162190A01F47F410A4342EA84
:100B100013635E490B605A4A107853781B0443EA0A
:100B20000063907843EA0023D07803431A0202F46A
:100B30007F0242EA0062180A00F47F40024342EA60
:100B40001363534A13604F48047843781B0443EA05
:100B50000463847843EA0423C4782343180200F42E
:100B60007F0040EA04601C0A04F47F44204340EA0A
:100B70001360484B1860484C484802904848019020
:100B8000002000902046F9F76BFF2046F9F78EFE13
:100B900044492046F9F793FE43492046F9F78CFE75
:100BA00042494348F9F7BEFE94F83D3013F0040F74
:100BB00018D02046F9F7EEFF05AC3E4D0FCD0FC41F
:100BC00095E8070084E80700334905A8F5F7DEFD3E
:100BD0000DB030BDFEF712FC0146374A3748FEF72C
:100BE000F9FF58E72C48FAF701F8E5E7264B344AB5
:100BF00092E803001860998000210846F9F77CF913
:100C0000224900200860224A1060224B1860224CC2
:100C10002C4D2563214D0295214D019500902046D4
:100C2000F9F71EFF2046F9F741FE1E492046F9F765
:100C300046FE1D492046F9F73FFE1C491C48F9F7BE
:100C400071FE94F83D3013F0040F0FD02046F9F7F1
:100C5000A1FF05AC1C4D0FCD0FC495E8070084E83B
:100C600007000D4905A8F5F791FDB1E70A48F9F726
:100C7000BDFFEEE726000020C8140120F814012073
:100C8000F4140120F0140120C014012004150120E7
:100C900000150120FC14012008150120B59E000854
:100CA00089640008B9080108BB080108BD080108EB
:100CB000B8140120505D010838830108148501082B
:100CC000E0140120388201086C5D010808B50F4B63
:100CD0001B782BB90E4B93F83D3013F0010F00D168
:100CE00008BD0B48FCF7C6FB0028F9D1074B0122D1
:100CF0001A70084B1B78002BF2D0FEF77FFB0146E1
:100D0000054A0648FEF766FFEAE700BFC614012061
:100D10000815012026000020388301083C850108C1
:100D2000014B1878704700BFEC14012008B501385A
:100D3000032807D8DFE800F002080B0FFFF75EFA80
:100D4000FFF754FA002008BDFFF754FAFAE7034B07
:100D500001221A70F6E7FFF749FAF3E7B41401200D
:100D60007047000000B583B00023019330B94FF401
:100D7000C0230193019803B05DF804FB012821D042
:100D8000022822D0032823D0042824D0052827D0E5
:100D900006282AD007282DD0082830D0102833D094
:100DA000112836D0122839D013283CD014283FD02F
:100DB0001E2842D01F2844D01F28DBD901A9FFF7E5
:100DC00057FBD7E7214B0193D4E7214B0193D1E7A0
:100DD00001230193CEE7FEF721FB03780193C9E7D6
:100DE000FEF71CFB43780193C4E7FEF717FB43882B
:100DF0000193BFE7FFF7F6F983690193BAE7FFF7BD
:100E0000F1F9C3690193B5E7FFF7ECF94368019382
:100E1000B0E7FFF7E7F983680193ABE7FFF7E2F983
:100E2000C3680193A6E7FFF7DDF903690193A1E722
:100E3000FFF7D8F9436901939CE7064B1B680193C0
:100E400098E7054B1B68019394E700BF69666C79CE
:100E5000746F70004C1501205015012010B582B040
:100E600000230193D0B10C4601281DD002281FD0C9
:100E7000032821D0102823D0112829D012282FD0C0
:100E8000132835D014283BD01E283ED01F2845D02B
:100E90001F2806D901AAFFF7AFFA02E0FFF762FFA9
:100EA0000190019802B010BDFFF75CFF0190F8E7D8
:100EB000FFF758FF0190F4E7FFF754FF0190F0E7C8
:100EC000FFF790F94460FFF78DF943680193E8E775
:100ED000FFF788F98460FFF785F983680193E0E7FD
:100EE000FFF780F9C460FFF77DF9C3680193D8E785
:100EF000FFF778F90461FFF775F903690193D0E70B
:100F0000FFF770F943690193CBE7064B1968204658
:100F1000FFF70CFF0190044B1860C2E7014B19600A
:100F20000191BEE7501501204C150120F8B504468B
:100F300016461F460B18B3F5807F01D9C0F58071A6
:100F40003D688D4207D30D4605E02046FFF70AFFB6
:100F500046F824000134A542F7D83D60F8BD10B42E
:100F600003690C699C4207D3002313700B69006965
:100F7000181A5DF8044B7047012313700B69006960
:100F8000181A00F5A83000F5C070F2E708B5074A56
:100F9000D071030A9371030C5371000E1071342346
:100FA00043F2D6210248FEF7C1FF08BD2800002009
:100FB000CC18012038B50B4C002525606060A1607D
:100FC000E260FEF71BFA206165611823224644F6B1
:100FD000BF510548FEF7AAFF182814BF00200120C2
:100FE00038BD00BF54170120AC18012010B51346BE
:100FF000064A0124146050609160D360102344F6C7
:10100000BF510348FEF792FF10BD00BF54160120E8
:10101000AC18012008B5064A02231360012353606F
:10102000082344F6BF510348FEF780FF08BD00BF08
:1010300054150120AC1801202DE9F04387B0044677
:101040000D469046F5F798FB06464246294620464F
:10105000FFF7B0FF0746F5F78FFB334B1B78002BEC
:101060003AD1002F35D0314A1360314A13602E4BEC
:1010700001221A702F4A136801331360871B2E4B0D
:101080001B68A6EB03092D4B1B68A9EB0303002B80
:10109000B8BF5B42032B03DD244A1368013313609E
:1010A000012F03DD224A136801331360244B1B68B0
:1010B000A34217D0234B1B780BBB1F4B1E601F4B4B
:1010C000C3F800901E4B1C601F4B1D601F4BC3F8E4
:1010D000008007B0BDE8F083002FCFD1124B002273
:1010E0001A70F6E7184B1B68AB42E3D1174B1B682D
:1010F0004345DFD1164A136801331360DAE7FEF780
:101100007DF90146124B1B680493094B1B6803933E
:10111000064B1B6802930197CDF8009033460D4AA9
:101120000D48FEF757FDC8E7781801207418012014
:10113000701801206C180120681801206418012023
:1011400060180120260000205C180120581801209A
:1011500054180120648501087085010808B5074B03
:101160001868FEF74FF9B0F5967F00D208BDFEF77C
:1011700045F9024B1860FFF74DFFF7E77C18012097
:10118000F0B501F00F04C1F30125C1F3034EC1F323
:10119000026102F00F03C2F30227C2F30346C2F357
:1011A000016202EB820206EB4206066007EB87074C
:1011B00003EB4703436001EB81010EEB41028260C8
:1011C00005EB850104EB4104C460C3EB03139B00F2
:1011D0004FF4616101FB06331A440261F0BD000067
:1011E00070B58CB084E001A940F26220FFF740F9AD
:1011F00002A940F26320FFF73BF903A94FF41970ED
:10120000FFF736F9039B0BB1013B039300238DF8E5
:101210000330029A019907A8FFF7B2FF3D4D0DF187
:10122000030207A92846FFF79AFE0646AE460DF1CF
:101230001C0CBCE80F00AEE80F00DCF80030CEF864
:101240000030022E0BD89DF803301BB1324A1368D0
:101250000133136036B9314B1B7883B102E02E4B5A
:1012600000221A602D4B00221A702B4B1B680B9822
:101270002B4A02FB03002B4B1860FFF787FE039AF3
:1012800002990198FFF7D8FEFEF7B8F8264B1860D0
:1012900038E000230393079303A940F20D50FFF7B2
:1012A000E7F807A940F20E50FFF7E2F8079A039912
:1012B0000120FFF79BFEFEF7A1F81B4B186024E00E
:1012C00000240394079403A940F20D50FFF7D0F8CF
:1012D00007A940F20E50FFF7CBF8079A0399204672
:1012E000FFF784FEFEF78AF80F4B1860FFF736FF12
:1012F0003222072104A8F5F7B5FA059C14F0010F76
:101300007FF471AF14F0020FC3D114F0040FD7D1E2
:10131000ECE700BF88180120841801205C00002041
:1013200080510100801801207C18012010B504466E
:10133000104B1B68984204D00F4B1B689C4212D084
:1013400010BDFFF7B7F8F430FEF7A4FB28B1022177
:101350000A4B1868F5F754FAEEE70421074B1868B2
:10136000F5F74EFAE8E70121044B1868F5F748FA5B
:10137000E6E700BFA41801209C180120A81801204E
:1013800010B588B043F2D5212948FEF72FFD58B992
:101390004FF49073274A28492848FEF71BFC4FF466
:1013A0007A70FEF71FF8F3E744F6BE512448FEF7C3
:1013B0001DFD58B940F221131E4A22491F48FEF76D
:1013C00009FC4FF47A70FEF70DF8F3E70DF1040C09
:1013D0001D4C0FCCACE80F0094E807008CE8070028
:1013E000002101A8F5F7D2F9184A106098B1FFF76B
:1013F00061F8B0F8DC20164B1A60FFF75BF8B0F824
:10140000EC20144B1A60FFF755F8B0F8FC20124B93
:101410001A6008B010BD4FF49373064A0F4907488D
:10142000FEF7D8FB4FF47A70FDF7DCFFF3E700BF5F
:10143000CC180120B0850108DC850108C07D0108B9
:10144000AC18012014860108885D0108A818012045
:10145000A01801209C180120A41801205086010822
:101460000A22002100F070B9024B0146186800F012
:1014700025B800BF6C00002070B50F4E0C463168D7
:10148000054611B901F0EAF930602146284601F01D
:10149000E5F9431C03D14FF0FF34204670BDC41C56
:1014A00024F00304A042F8D0211A284601F0D6F90E
:1014B0000130F2D1EFE700BFEC1801202DE9F8432D
:1014C000CD1C25F0030508350C2D38BF0C25002D4B
:1014D000064601DBA94204D90C2333600020BDE895
:1014E000F883DFF8D48000F069F8D8F800301C46A3
:1014F00044BB29463046FFF7BFFF431C044658D182
:10150000D8F800402746002F43D1002C4BD0236849
:101510003946304604EB030901F0A0F9814542D178
:1015200021686D1A29463046FFF7A6FF01303AD0F0
:1015300023682B442360D8F800305A6862BBC8F88F
:1015400000700FE02268521B20D40B2A17D96119B2
:10155000A342256018BF5960636808BFC8F800102F
:1015600062514B60304600F02FF804F10B00231D50
:1015700020F00700C21A1CBF1B1AA350AFE7626815
:10158000A3420CBFC8F800205A60EBE7234664680A
:10159000AEE73C467F68B6E71A465B68A342FBD1DC
:1015A00000235360DEE70C233360304600F00CF874
:1015B00094E70560D6E700BFF01801200148F0F776
:1015C0009DBB00BF500900200148F0F7A0BB00BF41
:1015D00050090020164B10B51C68236BB3B91820B6
:1015E000FFF742FF0246206320B9124B12485221F6
:1015F00001F094F91149124BC0E90013114B8360BB
:101600000B23838100210120C2E90401216B0E48D4
:101610000B694C690D4A584302FB0400A3FB0232DC
:10162000013340EB0200C1E9043020F0004010BD5E
:101630006C00002096860108AD8601080E33CDAB04
:1016400034126DE6ECDE05002DF451582D7F954CDB
:10165000242B2DE9F0478646904601D8012B06D170
:1016600001F01EF9162303600020BDE8F08734481E
:101670000D462A4615F8014B065D16F00806F8D10E
:101680002D2C2DD12C780126951C33F0100209D178
:10169000302C2AD12A7802F0DF02582A25D16C7822
:1016A0001023023506F1004C0CF1FF3C0022BCFB7C
:1016B000F3F9104603FB19CAA4F13007092F1BD810
:1016C0003C46A34227DD571C07D0814520D301D1DA
:1016D000A2451DDB00FB0340012215F8014BEBE79F
:1016E0002B2C04BF2C78951CCFE7002BDAD1302CA3
:1016F0000CBF08230A23D5E7A4F14107192F01D80D
:10170000373CDEE7A4F16107192F04D8573CD8E72E
:101710004FF0FF32E1E7531C08D12223CEF800300E
:101720006046B8F1000FA0D0691E06E006B1404245
:10173000B8F1000F99D0002AF6D1C8F8001094E74C
:1017400006870108FFF784BF13460A460146024890
:101750000068FFF77DBF00BF6C0000202DE9FF4748
:1017600057EC106B002F0C4619463B46BBBF07F1E8
:1017700000431F4600232D230B700D9BDDF830A086
:10178000914623F02008BCBF32461646B8F1460FFA
:1017900005D0B8F1450F00D10134022100E003214A
:1017A00003AB019302AB009347EC106B5346224608
:1017B00001F05AF9B8F1470F054619D119F0010F98
:1017C0000ED000EB04090022002330463946EFF723
:1017D0007BF908B1CDF80C903022039B4B451ED30A
:1017E000039B0E9A5B1B2846136004B0BDE8F0878C
:1017F000B8F1460F00EB0409E5D10378302B0AD18C
:101800000022002330463946EFF75EF918B9C4F1DB
:101810000104CAF80040DAF800309944D3E7591CB3
:1018200003911A70D9E7F7B50029BABF49422D23B1
:101830002B2309290270437029DD0DF107031D4692
:101840000A271A46B1FBF7F607FB1614303402F8E4
:10185000014C0C46632C03F1FF333146F1DC30318F
:10186000941E03F8011C411C2346AB420AD30DF120
:1018700009039B1AAC4288BF002302330344181AA1
:1018800003B0F0BD13F8016B01F8016FEDE73023F1
:1018900030318370C170031DF1E700002DE9F04F76
:1018A0008DB00C46DDF8588016461F46054600F000
:1018B00047FF036804931846EEF7DAFC00230A9307
:1018C000D8F800300590073323F0070303F108022E
:1018D00094F818A0D4F800B0C8F80020D3E9008923
:1018E00029F000430793CDF81880C4E91289DDE997
:1018F00006019C4B4FF0FF32EFF718F970BBDDE9A2
:101900000601984B4FF0FF32EFF7F2F830BB0022A0
:10191000002340464946EFF7E1F810B12D2384F843
:101920004330914A914BBAF1470F94BF9046984685
:10193000032323612BF0040323604FF00009009779
:1019400033460BAA2146284600F0D2F9013040F078
:101950008D804FF0FF300DB0BDE8F08F42464B4612
:1019600040464946EFF7E2F840B14B46002BBCBF7A
:101970002D2384F843307E4A7E4BD4E763680AF017
:10198000DF0206925A1C3BD1062363604BF480624F
:101990000023226003930AABCDE901A309AB0093B6
:1019A000616849EC108B0DF123032846FFF7D6FE42
:1019B000069B0999472B804629D1C81C02DB636826
:1019C000994241DDAAF1020A5FFA8AFA01395246C8
:1019D00004F150000991FFF726FF0A9A1318012A13
:1019E0008146236102DC2268D20701D501332361DD
:1019F0009DF82330002BA2D02D2384F843309EE79E
:101A0000069A472AC2D1002BC0D10123BDE7BAF103
:101A1000650FDBD9BAF1660F18D1002963680BDDB9
:101A2000216113B92268D00702D501330B44236129
:101A3000A1654FF00009DBE713B92268D20701D591
:101A40000233F4E70123F2E74FF0670A0A9B994259
:101A500005DB23682161D807EAD54B1CE7E700299D
:101A6000D4BFC1F1020201221344E0E723685A0502
:101A700007D42369424631462846B84701302BD166
:101A800067E7BAF1650F40F2DD80D4E91201002268
:101A90000023EFF719F8002833D0374A01233146E5
:101AA0002846B84701303FF454AFDDE909384345D3
:101AB00002DB2368D8070FD5DDE904233146284629
:101AC000B84701303FF445AF4FF0000908F1FF3847
:101AD00004F11A0AC84509DC23689B0700F1038159
:101AE000E0680B9B9842B8BF184634E70123524682
:101AF00031462846B84701303FF42BAF09F10109C0
:101B0000E8E7099B002B39DC1B4A012331462846B4
:101B1000B84701303FF41DAFDDE9093959EA030345
:101B200002D12368D907D7D5DDE9042331462846F9
:101B3000B84701303FF40DAF4FF0000A04F11A0B23
:101B4000099B5B42534501DC4B4693E701235A4610
:101B500031462846B84701303FF4FBAE0AF1010A8E
:101B6000EEE700BFFFFFEF7F068801080A88010843
:101B70000E8801081288010816880108A36DDDF897
:101B800028A05345A8BF5346002B994636DC4FF09A
:101B9000000B29EAE97904F11A02A36D0693A3EB7D
:101BA00009035B4531DC099B9A453ADC2368DA0777
:101BB00037D4099BAAEB0309069BAAEB03039945BB
:101BC000A8BF9946B9F1000F33DC4FF0000829EAAD
:101BD000E97904F11A0B099BAAEB0303A3EB0903B0
:101BE00043457FF779AF01235A4631462846B84727
:101BF00001303FF4AEAE08F10108ECE74246314651
:101C00002846B8470130C2D1A3E601233146284611
